:100000000C947F050C94AA050C94AA050C94AA05DF
:100010000C94E30B0C94AA050C94AA050C94AA0565
:100020000C94AA050C9480390C94AA050C94AA058A
:100030000C94AA050C94776A0C94AA050C94AA0552
:100040000C94AA050C94AA050C94F4720C94AA05BD
:100050000C94AF740C9445750C94AA050C94AA05E5
:100060000C94AA050C94AA050C942E710C94AA0564
:100070000C94E8740C9492750C94AA050C94AA053F
:100080000C94AA050C94AA050C94AA052D33002DF6
:1000900032002D31002030002B31002B32002B3369
:1000A000002B340020430020432300204400204440
:1000B0002300204500204600204623002047002042
:1000C000472300204100204123002042004D53548B
:1000D000004D494400434C4B00322F3100312F3149
:1000E00000312F3200312F3400312F3800312F31C1
:1000F0003600312F34380053494E005452490053D2
:1001000041570053515500532F4800445732004483
:100110005733004457340044573500445736005491
:100120005731005457320054573300545734004568
:10013000585000485244005346540046555A005304
:10014000504B0053545000313025003235250035D6
:1001500030250037352500393025004348524F4DB2
:100160004154494320004D414A4F52202020202035
:10017000006D696E6F7220202020200050454E5483
:1001800041544F4E494300444F5249414E20202094
:100190002000504852594749414E2020004C5944B4
:1001A00049414E20202020004D49584F4C59444988
:1001B000414E004C4F435249414E20202000464FB3
:1001C00052574152442020004241434B5741524430
:1001D000200050494E472D504F4E470052414E444B
:1001E0004F4D2020200053594E0042504D00545294
:1001F00058004356525800434C4B004E4300414375
:1002000000505452004C454E0053434C0054524948
:1002100047004C464F005741560046525100414D51
:100220005000535450004E5445004F4354004C4529
:100230004E470055544D0050524F00525452470003
:1002400050554C0042415200435059004155540012
:100250004D414E004F464600204F4E005253540031
:10026000504F5300534E4700424400534400533113
:10027000005332004C54004D540048540043500089
:100280004348004F48004352005244003576200056
:1002900031307600E601EA014002F70148025C02D3
:1002A000FB01FE010102050209020D021202160203
:1002B0001A021E02440226022A022E020902FB0131
:1002C000FB01FB014402330237023B0244023302CA
:1002D00037022E024402050209020D026402600286
:1002E00001020502BE01C801D201DC015B01660109
:1002F00071017C01870192019D01A801B3014701B1
:100300004B014F0153015701F700FB00FF000301B0
:1003100007010B010F01130117011B011F0123012D
:1003200027012B012F01330137013B013F0143011D
:10033000D900DD00E100E500E900ED00F200CD00AC
:10034000D100D5008C008F009200950098009B0092
:100350009E00A100A400A700AB00AE00B200B50053
:10036000B800BC00BF00C300C600CA0068026B0230
:100370006E027102740277027A027D0280028302A9
:100380008602890250024C02540258028C029002EA
:100390000102030405060708090A0B0C0101030307
:1003A00005060608080A0A0C0101030304060608EC
:1003B0000809090B0101030303050508080A0A0AD5
:1003C0000101030304060608080A0A0B01010202E0
:1003D000040606080809090B0101030305070708BD
:1003E000080A0A0C0101030305060608080A0A0B9D
:1003F00001010202040606070709090B00002B0091
:1004000055008000AB00D50000012B015501800193
:10041000AB01D501807C797673706D6A6763605D2E
:100420005A5754514F4C494643403E3B383633317E
:100430002E2C2A272523211F1D1B191715131210D7
:100440000F0D0C0A09080706050403030201010049
:10045000000000000000000000000101020303048E
:1004600005060708090A0C0D0F1012131517191BA2
:100470001D1F212325272A2C2E313336383B3E40A1
:100480004346494C4F5154575A5D6063676A6D70DB
:100490007376797C808386898C8F9295989C9FA2B5
:1004A000A5A8ABAEB0B3B6B9BCBFC1C4C7C9CCCEAA
:1004B000D1D3D5D8DADCDEE0E2E4E6E8EAECEDEF31
:1004C000F0F2F3F5F6F7F8F9FAFBFCFCFDFEFEFF9F
:1004D000FFFFFFFFFFFFFFFFFFFFFEFEFDFCFCFB3A
:1004E000FAF9F8F7F6F5F3F2F0EFEDECEAE8E6E406
:1004F000E2E0DEDCDAD8D5D3D1CECCC9C7C4C1BFE7
:10050000BCB9B6B3B0AEABA8A5A29F9C9895928F8C
:100510008C8986837C7A78767472706E6C6A686671
:100520006462605E5C5A58565452504E4C4A48467B
:100530004442403E3C3A38363432302E2C2A28266B
:100540002422201E1C1A18161412100E0C0A08065B
:100550000402010000020406080A0C0E1012141610
:10056000181A1C1E20222426282A2C2E303234361B
:10057000383A3C3E40424446484A4C4E505254560B
:10058000585A5C5E60626466686A6C6E70727476FB
:10059000787A7C7E80828486888A8C8E90929496EB
:1005A000989A9C9EA0A2A4A6A8AAACAEB0B2B4B6DB
:1005B000B8BABCBEC0C2C4C6C8CACCCED0D2D4D6CB
:1005C000D8DADCDEE0E2E4E6E8EAECEEF0F2F4F6BB
:1005D000F8FAFCFEFEFCFAF8F6F4F2F0EEECEAE8CB
:1005E000E6E4E2E0DEDCDAD8D6D4D2D0CECCCAC89B
:1005F000C6C4C2C0BEBCBAB8B6B4B2B0AEACAAA88B
:10060000A6A4A2A09E9C9A98969492908E8C8A887A
:10061000868482807E0102030405060708090A0B0E
:100620000C0D0E0F101112131415161718191A1B92
:100630001C1D1E1F202122232425262728292A2B82
:100640002C2D2E2F303132333435363738393A3B72
:100650003C3D3E3F404142434445464748494A4B62
:100660004C4D4E4F505152535455565758595A5B52
:100670005C5D5E5F606162636465666768696A6B42
:100680006C6D6E6F707172737475767778797A7B32
:100690007C7D7E7F808182838485868788898A8B22
:1006A0008C8D8E8F909192939495969798999A9B12
:1006B0009C9D9E9FA0A1A2A3A4A5A6A7A8A9AAAB02
:1006C000ACADAEAFB0B1B2B3B4B5B6B7B8B9BABBF2
:1006D000BCBDBEBFC0C1C2C3C4C5C6C7C8C9CACBE2
:1006E000CCCDCECFD0D1D2D3D4D5D6D7D8D9DADBD2
:1006F000DCDDDEDFE0E1E2E3E4E5E6E7E8E9EAEBC2
:10070000ECEDEEEFF0F1F2F3F4F5F6F7F8F9FAFBB1
:10071000FCFDFEFF000000000000000000000000E3
:1007200000000000000000000000000000000000C9
:1007300000000000000000000000000000000000B9
:1007400000000000000000000000000000000000A9
:100750000000000000000000000000000000000099
:100760000000000000000000000000000000000089
:100770000000000000000000000000000000000079
:100780000000000000000000000000000000000069
:100790000000000000FFFFFFFFFFFFFFFFFFFFFF64
:1007A000FFFFFFFFFFFFFFFFFFFFFFFFFFFFFFFF59
:1007B000FFFFFFFFFFFFFFFFFFFFFFFFFFFFFFFF49
:1007C000FFFFFFFFFFFFFFFFFFFFFFFFFFFFFFFF39
:1007D000FFFFFFFFFFFFFFFFFFFFFFFFFFFFFFFF29
:1007E000FFFFFFFFFFFFFFFFFFFFFFFFFFFFFFFF19
:1007F000FFFFFFFFFFFFFFFFFFFFFFFFFFFFFFFF09
:10080000FFFFFFFFFFFFFFFFFFFFFFFFFFFFFFFFF8
:10081000FFFFFFFFFF202837465564738291202099
:100820002020002E2E2E2E2E2E2E2E2E2E2E2E2E32
:100830002E2E2E00444143732063616C6962726105
:1008400074696F6E0020696E697469616C697A61A0
:1008500074696F6E20002020202020454550524FA3
:100860004D2020202020002B002D00546F74616C3F
:10087000204163632076616C756520005B534156AF
:100880004544215D00455854002020202020202090
:100890002020202020202020200020202020002098
:1008A00020202000202020200020202020001018C0
:1008B00020304060805074726E2000506F732000B2
:1008C00020536F6E6720506C6179205300736E6700
:1008D00020706F7320707472206C656E20004F6EF4
:1008E000004F6666004F6E004F66660020204C4643
:1008F0004F73202043562F476174652000730062B8
:1009000061722075746D2070726F2072747267004E
:100910006261722075746D2070726F206C656E67F5
:10092000006C666F207761762066727120616D7051
:100930002000435620547261636B205363616C65E1
:100940003A20007300626172206E7465206F6374D8
:10095000206C656E670020202000312F0046494C36
:100960004C00626172206C656E2073636C2074723F
:100970006967004558540020205061747465726E98
:1009800020506C61792020002020204261722020BC
:10099000202053746570202000200063707920723D
:1009A0007374206E632020616320200073796E20B1
:1009B00062706D2070756C20636C6B200020547227
:1009C000636B20646972656374696F6E20002050E8
:1009D00074726E20646972656374696F6E20002B97
:1009E000002D00202053687566666C652076616C6A
:1009F000756520000002040507090B0002050709C0
:100A000000030408121313111F000000000000006F
:100A1000001804020919191110080601000000004D
:100A20000004001F0000000001020C100000000084
:100A300010101112040810000000171417151700E9
:100A40000000101810100C0000000E0A0E0A0E0014
:100A500000001B091B0A1B0001010101010F1F0EF1
:100A600000000A0A0E02020000000E020E080E002C
:100A700076312E3034330000002100240027002A74
:100A80000000002200250028002B00000020002389
:100A900000260029000202020202020202040404EB
:100AA0000404040404030303030303030301010117
:100AB000010101010101020408102040800102042B
:100AC0000810204080010204081020408001020428
:100AD000081020408000000001020008090000000A
:100AE00000040307060000000000000000000000F2
:100AF000000000000000C033C66F0D77B933112429
:100B00001FBECFEFD0E4DEBFCDBF11E0A0E0B1E06B
:100B1000E4E1FEEF00E00BBF02C007900D92A23FA0
:100B2000B107D9F71BBE1FE2A2EFB1E001C01D92D1
:100B3000A932B107E1F71AE0CCEFDAE004C022975E
:100B4000FE010E94C27EC63FD107C9F70E94A3776B
:100B50000C94FD7E0C940000CF93DF93BC01823097
:100B6000910510F462E070E0A091272FB091282F3A
:100B7000ED01E0E0F0E040E050E021C088819981A3
:100B80008617970769F48A819B81309719F09383C0
:100B9000828304C09093282F8093272FFE0134C0B6
:100BA0006817790738F44115510519F0841795072E
:100BB00008F4AC01FE018A819B819C01E901209728
:100BC000E9F641155105A9F1CA01861B970B049757
:100BD00008F4BA01E0E0F0E02AC08D919C911197F1
:100BE00084179507F9F46417750781F412968D91AF
:100BF0009C911397309719F09383828304C090934C
:100C0000282F8093272FFD0132964CC0CA01861BE6
:100C1000970BFD01E80FF91F6193719302978D9374
:100C20009C9340C0FD01828193819C01D901109762
:100C3000A1F68091252F9091262F892B41F4809148
:100C40003101909132019093262F8093252F40916E
:100C50003301509134014115510541F44DB75EB750
:100C600080912F0190913001481B590B2091252F25
:100C70003091262FCA01821B930B8617970780F0AD
:100C8000AB014E5F5F4F8417950750F0420F531F23
:100C90005093262F4093252FF9016193719302C041
:100CA000E0E0F0E0CF01DF91CF910895CF93DF93A3
:100CB000009709F450C0EC0122971B821A82A09180
:100CC000272FB091282F109709F140E050E0AC1782
:100CD000BD0708F1BB83AA83FE0121913191E20F88
:100CE000F31FAE17BF0779F48D919C911197280FD0
:100CF000391F2E5F3F4F3983288312968D919C9127
:100D000013979B838A834115510571F4D093282F43
:100D1000C093272F20C012968D919C911397AD01FF
:100D2000009711F0DC01D3CFFA01D383C283219164
:100D30003191E20FF31FCE17DF0769F488819981A3
:100D4000280F391F2E5F3F4FFA01318320838A819C
:100D50009B8193838283DF91CF910895A0E0B0E0DF
:100D6000E4EBF6E00C94CE7EEC01A880B980CA805A
:100D7000DB80A114B104C104D10441F484E2A82EA3
:100D800089EDB82E8BE5C82E87E0D82EC601B501B7
:100D90002DE133EF41E050E00E94A57E27EA31E4E7
:100DA00040E050E00E94317E7B018C01C601B5011C
:100DB0002DE133EF41E050E00E94A57ECA01B90168
:100DC0002CEE34EF4FEF5FEF0E94317E6E0D7F1DF2
:100DD000801F911F97FF04C0615070408040904871
:100DE000688379838A839B839B01AC015F77B90118
:100DF000CA01CDB7DEB7EAE00C94EA7E0E94AE06E7
:100E0000089585E391E00E94AE0608956093350150
:100E10007093360180933701909338010895A0E0D4
:100E2000B0E0E5E1F7E00C94C87E6C01009729F48E
:100E3000CB010E94AC056C01C1C08EEF882E8FEFF4
:100E4000982E8C0C9D1C8601060F171F081519057E
:100E500008F4B2C0F401A081B181A617B707B8F0B9
:100E6000A530B10508F4AAC0CD01049786179707ED
:100E700008F4A4C01297A61BB70BF801A193B19375
:100E8000D4016D937C93CF010E94560697C07B01DD
:100E9000EA1AFB0AEEEFFFEFEE0EFF1E36016A0EB6
:100EA0007B1EC091272FD091282F44245524AA249B
:100EB000BB244AC0C615D705E1F5488159814E15B6
:100EC0005F05B8F1CA0104978E159F05B0F412961C
:100ED000A40FB51FF401B183A0832A813B81411483
:100EE000510431F0D20113963C932E93129766C0B1
:100EF0003093282F2093272F61C08A819B81F8018E
:100F000093838283425050404E195F09518340833E
:100F10004114510431F0D20113961C930E93129791
:100F200004C01093282F0093272FF401718360834E
:100F300045C088819981A816B90608F45C012E0184
:100F40008A819B819C01E901209709F0B3CF8091B0
:100F5000252F9091262F86159705E9F4A616B7063A
:100F6000D0F420913301309134012115310541F441
:100F70002DB73EB780912F0190913001281B390B7E
:100F800002171307C8F41093262F0093252FD401BE
:100F90006D937C9313C0CB010E94AC05EC010097CC
:100FA00059F0F40140815181B6010E94EB07C6015E
:100FB0000E9456066E0102C0CC24DD24C601CDB7C6
:100FC000DEB7E0E10C94E47EFB01DC0105900D92BC
:100FD0000020E1F70895FB01DC0102C001900D92B1
:100FE00041505040D8F70895FB01DC018D910190EC
:100FF00080190110D9F3990B0895FB01DC010190D0
:101000000D920020E1F70895FB019F01E894423022
:10101000C4F04532B4F44A3029F497FB1EF490959D
:1010200081959F4F642F77270E945C7E805D8A3375
:101030000CF0895D8193CB010097A1F716F45DE276
:1010400051931082C9010C943B08FB019F0142306F
:1010500074F0453264F4642F77270E945C7E805DD3
:101060008A330CF0895D8193CB010097A1F7108240
:10107000C9010C943B08DC01FC01672F71917723B7
:10108000E1F7329704C07C916D9370836291AE1743
:10109000BF07C8F30895FC018081877E808320E02C
:1010A000672B09F021E090819E7F922B9083892FFE
:1010B000869581702817A9F092FD04C0213011F4A3
:1010C00098609083808182FF04C080FD02C08061AF
:1010D00080838081982F9170990F990F8B7F892B36
:1010E00080838081982F9170990F8D7F892B8083C9
:1010F0000895CF92DF92EF92FF920F931F93CF93B9
:10110000DF93382F9091F30180E02091F201022FBC
:1011100010E0082B192B332321F0313009F068C07F
:1011200068C060911E2B70911F2BCCE0D2E040E094
:1011300050E021E0C22ED12CE12CF12CFA01EE0F6F
:10114000FF1FE55FFD4F3081C801042E02C0969558
:1011500087950A94E2F7A82FA170367F932F9A2BD8
:101160009083892F86958170A81751F192FD28C030
:10117000A13031F53960308388818F5F8883813079
:1011800019F08230E9F40DC0D701C601042E04C065
:10119000880F991FAA1FBB1F0A94D2F7682B792BBF
:1011A0000FC01882D701C601042E04C0880F991FF2
:1011B000AA1FBB1F0A94D2F78095909568237923C4
:1011C000FA01EE0FFF1FE55FFD4F8081982F9170B0
:1011D000990F8D7F892B80834F5F5F4F229640311F
:1011E000510509F0ABCF60931E2B70931F2B02C0EB
:1011F00002C0B801CB01DF91CF911F910F91FF90F9
:10120000EF90DF90CF9008952F923F924F925F9290
:101210006F927F928F929F92AF92BF92CF92DF9206
:10122000EF92FF920F931F93CF93DF931C01609077
:10123000E602462D50E0FA01E957F04E70807294B4
:10124000B0EF7B2220916E1F30E00091EF03ACE005
:10125000CA2EA2E0DA2E60E070E0EA01CC0FDD1FBA
:10126000CA01E6E0880F991FEA95E1F7C80FD91F78
:1012700083E994E0FC012E9FC0012F9F900D3E9FBB
:10128000900D1124C80FD91F84E7882E8FE1982E66
:10129000840E951E86E299E0289F5001299FB00C8C
:1012A000389FB00C11247A01EA0CFB1C8FEF93E0FD
:1012B000E80EF91E872D860F482E5524FE01E40DF9
:1012C000F51DEE0FFF1FEE5EFB4F8081282F217072
:1012D000382F36953170C101062E02C0969587953C
:1012E0000A94E2F7182F1170AB01440F551FFA0151
:1012F000E55FFD4F90819E7F912B9083892F86958E
:101300008170181709F472C092FD57C0113009F0AE
:1013100054C0F4011083222309F446C0332329F476
:10132000F7018081882309F044C0F6011082F0E1C2
:101330006F16D9F0FE01E60FF71FEE0FFF1FDF015A
:10134000AE5EBB4F8C9183708C9311968C911197EC
:10135000887F846011968C93ED5EFB4F808187704F
:101360008083F401108320E028C0FA01E60FF71F04
:10137000EA0DFB1DDF01A45AB34F8C918E7F8C9335
:10138000E35AF34F8081877080839C9111968C91F2
:101390001197887F846011968C9311979170986152
:1013A0009C9320E001E009C0F7018081882319F4B3
:1013B00021E031E002C021E030E0FE01E40DF51D46
:1013C000EE0FFF1FEE5EFB4F80818C7F330F822B71
:1013D000832B8083FB01EE0FFF1FE55FFD4F8081B4
:1013E000982F9170990F8D7F892B80836F5F7F4F2E
:1013F00082E090E0C80ED91E6031710509F05ACF25
:101400000093EF03DF91CF911F910F91FF90EF9029
:10141000DF90CF90BF90AF909F908F907F906F9014
:101420005F904F903F902F9008959F92AF92BF9200
:10143000CF92DF92EF92FF920F931F93CF93DF93A0
:101440005C01E090E6024E2D50E020916E1F30E0EE
:10145000FA01E957F04EF080F294A0EFFA22A09141
:10146000EF0360E070E086E299E0289F8001299F09
:10147000100D389F100D112499249394EA01CC0F7C
:10148000DD1FCA01E6E0880F991FEA95E1F7C80F52
:10149000D91F83E994E0FC012E9FC0012F9F900D7E
:1014A0003E9F900D1124C80FD91F84E7C82E8FE1ED
:1014B000D82EC40ED51EC501062E02C0969587955E
:1014C0000A94E2F7482F4170FB01EE0FFF1FE55F22
:1014D000FD4F90819E7F942B9083892F86958170FC
:1014E000481709F46BC092FD5FC0413009F05CC041
:1014F0008F2D860F282F30E090E0F901EE0FFF1FAF
:10150000E20FF31FE00FF11FE45AF34F808180FFD9
:1015100091E0F901EE0FFF1FE20FF31FE00FF11F43
:10152000E45AF34F80818E7F892B80839923D9F5EC
:10153000F0E1EF16D1F0FE01E60FF71FEE0FFF1FEF
:10154000DF01AE5EBB4F8C9183708C9311968C91B2
:101550001197887F846011968C93ED5EFB4F80819C
:1015600087708083F60190821EC0FB01EE0FFF1F83
:10157000E60FF71FE00FF11FDF01A45AB34F8C9164
:101580008E7F8C93E35AF34F8081877080839C9188
:1015900011968C911197887F846011968C93119786
:1015A000917098619C93A1E0FB01EE0FFF1FE55F36
:1015B000FD4F440F80818D7F842B80836F5F7F4F31
:1015C0006031710509F077CFA093EF03DF91CF91E0
:1015D0001F910F91FF90EF90DF90CF90BF90AF9051
:1015E0009F900895AF92BF92CF92DF92EF92FF92B9
:1015F0000F931F93CF93DF93EC01D0902B02D694DF
:10160000D69481E0D822A0909901C090721FB0902A
:1016100028034091292850912A2820E030E091E0C9
:10162000E92EF12C012D112DF901EE0FFF1FE55FC1
:10163000FD4F6081CE01022E02C0969587950A94D7
:10164000E2F7782F7170667F962F972B9083892F02
:1016500086958170781709F453C092FD51C071309E
:1016600009F04EC069606083DD2031F1CC2081F04B
:10167000CA01022E02C0969587950A94E2F780FD72
:1016800024C0AA24A394CC24BB2440E050E038C05A
:10169000D801C701022E04C0880F991FAA1FBB1FC3
:1016A0000A94D2F7AC0140955095AA24A394CC2477
:1016B000C394BB24B39424C0CA01022E02C09695E1
:1016C00087950A94E2F780FF0FC0D801C701022E68
:1016D00004C0880F991FAA1FBB1F0A94D2F78095D8
:1016E0009095482359230CC0D801C701022E04C08D
:1016F000880F991FAA1FBB1F0A94D2F7482B592B9A
:10170000F901EE0FFF1FE55FFD4F8081982F91706B
:10171000990F8D7F892B80832F5F3F4F20313105BB
:1017200009F082CFA0929901C092721FB092280353
:1017300050932A2840932928DF91CF911F910F9130
:10174000FF90EF90DF90CF90BF90AF90089581E031
:101750000E947908AC0190931D2B80931C2B20E0F4
:1017600030E0CA01022E02C0969587950A94E2F7EE
:1017700080FF02C0822F08952F5F3F4F2031310537
:1017800081F78FEF089581E00E947908AC01909372
:101790001B2B80931A2B60E020E030E0CA01022E60
:1017A00002C0969587950A94E2F780FF05C06130E4
:1017B00011F4822F089561E02F5F3F4F20313105F2
:1017C00069F780E008951F920F920FB60F920BB643
:1017D0000F9211242F933F934F935F938F939F9377
:1017E000AF93BF93EF93FF9380B181708093DB2A17
:1017F0009091DB2A8091DC2A9817B9F18091DB2A3D
:10180000882379F581E08093DD2A10928302E6EB4C
:10181000FAE281932AE2E73CF207D9F72C9A2C9856
:1018200010927F0210924C0110924B0180E090E0E8
:1018300021E0FC01EB56FD4F1082FC01E25FFC4F02
:101840001082FC01E551FD4F2083FC01E954FD4F5E
:101850001082FC01E853FD4F2083019681319105F0
:1018600041F78091DB2A8093DC2A80917E0283708D
:10187000823009F0B8C080B190E09595879581706D
:101880008093D12A9091D12A8091A701981709F4C9
:1018900074C08091A701882311F02C9A01C02C9864
:1018A0008091D12A882309F065C08091C72A909140
:1018B000C82AA091C92AB091CA2A2091CD2A309174
:1018C000CE2A4091CF2A5091D02A821B930BA40B91
:1018D000B50B80939F019093A001A093A101B093B9
:1018E000A20180919F019091A001A091A101B091CE
:1018F000A201885E9340A040B04080F480919F0197
:101900009091A001A091A101B091A2018093A301A7
:101910009093A401A093A501B093A60121E0209388
:10192000D22A8091C72A9091C82AA091C92AB09141
:10193000CA2A8093CD2A9093CE2AA093CF2AB0931F
:10194000D02A8091E0028823C1F42093D32A2093E7
:10195000A8018091A3019091A401A091A501B0914B
:10196000A60180939F019093A001A093A101B09341
:10197000A20103C081E08093D52A8091D12A80936F
:10198000A70180919F019091A001A091A101B09128
:10199000A201885E9340A040B04060F088EE93E0E2
:1019A000A0E0B0E080939F019093A001A093A101DB
:1019B000B093A20180919F019091A001A091A101FB
:1019C000B091A201893C9105A105B10560F488ECB4
:1019D00090E0A0E0B0E080939F019093A001A093DD
:1019E000A101B093A201FF91EF91BF91AF919F919F
:1019F0008F915F914F913F912F910F900BBE0F9060
:101A00000FBE0F901F901895E82F592F40915C2A18
:101A100030915D2A2091202B222381F0213051F436
:101A20008DB38093222B9DB38091212B80958923A8
:101A30008DBB04C08FB7F8948093222B4CBD3DBD65
:101A40005D985EBD00000DB407FEFDCF8EB5EEBD06
:101A500000000DB407FEFDCF8EB57EBD00000DB4B5
:101A600007FEFDCF8EB56EBD00000DB407FEFDCFA5
:101A70008EB55D9A222339F08091222B213011F40A
:101A80008DBB01C08FBF5093FC01E093FB017093AD
:101A9000FA016093F9010895682F592F40915C2A4B
:101AA00030915D2A2091202B222381F0213051F4A6
:101AB0008DB38093222B9DB38091212B8095892318
:101AC0008DBB04C08FB7F8948093222B4CBD3DBDD5
:101AD0005C985EBD00000DB407FEFDCF8EB56EBDF7
:101AE00000000DB407FEFDCF8EB55C9A222339F0BD
:101AF0008091222B213011F48DBB01C08FBF5093F8
:101B0000F8016093F701089540915C2A30915D2AB5
:101B10002091202B222381F0213051F48DB380932A
:101B2000222B9DB38091212B809589238DBB04C0EE
:101B30008FB7F8948093222B4CBD3DBD5C981EBCA2
:101B400000000DB407FEFDCF8EB51EBC00000DB425
:101B500007FEFDCF8EB55C9A222339F08091222BAF
:101B6000213011F48DBB08958FBF08959C013F7003
:101B7000306160915C2A50915D2A4091202B442372
:101B800081F0413051F48DB38093222B9DB380912D
:101B9000212B809589238DBB04C08FB7F894809347
:101BA000222B6CBD5DBD12983EBD00000DB407FE3A
:101BB000FDCF8EB52EBD00000DB407FEFDCF8EB556
:101BC000129A442339F08091222B413011F48DBBBD
:101BD00008958FBF08958F3708F08FE7282F30E0E2
:101BE00045E0220F331F4A95E1F73F70306960915D
:101BF0005C2A50915D2A4091202B442381F0413092
:101C000051F48DB38093222B9DB38091212B80952D
:101C100089238DBB04C08FB7F8948093222B6CBDB1
:101C20005DBD12983EBD00000DB407FEFDCF8EB520
:101C30002EBD00000DB407FEFDCF8EB5129A4423D1
:101C400039F08091222B413011F48DBB08958FBF64
:101C500008959C013F70306160915C2A50915D2A2B
:101C60004091202B442381F0413051F48DB3809377
:101C7000222B9DB38091212B809589238DBB04C09D
:101C80008FB7F8948093222B6CBD5DBD13983EBD39
:101C900000000DB407FEFDCF8EB52EBD00000DB4C3
:101CA00007FEFDCF8EB5139A442339F08091222B85
:101CB000413011F48DBB08958FBF08959C013F7092
:101CC000306960915C2A50915D2A4091202B442319
:101CD00081F0413051F48DB38093222B9DB38091DC
:101CE000212B809589238DBB04C08FB7F8948093F6
:101CF000222B6CBD5DBD13983EBD00000DB407FEE8
:101D0000FDCF8EB52EBD00000DB407FEFDCF8EB504
:101D1000139A442339F08091222B413011F48DBB6A
:101D200008958FBF089540915C2A30915D2A2091DB
:101D3000202B222381F0213051F48DB38093222B6C
:101D40009DB38091212B809589238DBB04C08FB7D3
:101D5000F8948093222B4CBD3DBD5E9A1EBC0000C2
:101D60000DB407FEFDCF8EB51EBC00000DB407FEFE
:101D7000FDCF8EB58093B42A1EBC00000DB407FEC3
:101D8000FDCF8EB51EBC00000DB407FEFDCF8EB595
:101D90001EBC00000DB407FEFDCF8EB58093B22AA5
:101DA0008093B32A5E98222339F08091222B213030
:101DB00011F48DBB08958FBF08959C0143B1487005
:101DC00040935E2A93B1947090935F2A442311F557
:101DD0008091602A8823F1F0992319F0260F371F8C
:101DE00019C080912D0282FF10C080916B2A813032
:101DF00041F0813010F0823069F42A30310554F01E
:101E000007C02031310534F003C02115310511F030
:101E1000261B370B4093602AC9010895482F53B100
:101E200052705093642A93B191709093652A552310
:101E3000D9F48091662A8823B9F0992369F08FEF4D
:101E400090E0841B9109262F30E08217930714F449
:101E50004FEF0AC0460F08C0461720F4442321F074
:101E6000462F02C04111461B5093662A842F90E0F2
:101E70000895CF92DF92EF92FF920F931F93CF932B
:101E8000DF93EC01F42EE22E680118811093092BE8
:101E9000812F0E940E0F8883F81608F0F88288813F
:101EA0008E1508F0E8828881811739F08093092B1C
:101EB00081E0F601808380939901DF91CF911F919A
:101EC0000F91FF90EF90DF90CF9008950F931F93A5
:101ED000DF93CF930F92CDB7DEB7898380916E1FCA
:101EE00090E026E239E0829FF001839FF00D929FFF
:101EF000F00D1124E95AF34F2081203311F02036E0
:101F000009F428E12150CE01019661E040E00FEE96
:101F100013E00E94390F698160932003809135029C
:101F200083FF26C080916E1F90E040E050E026E2E3
:101F300039E0829FD001839FB00D929FB00D112494
:101F4000962F9F71990FFA01EE0FFF1FE40FF51FF7
:101F5000EA0FFB1FE45AF34F8081817C892B808339
:101F60004F5F5F4F4034510571F781E08093EF037D
:101F7000862F0F90CF91DF911F910F9108951F939E
:101F8000FC0113B112701093642A93B19170909375
:101F9000652A112361F58091662A882341F19923EE
:101FA000D1F0CF01A0E0B0E02FEF3FEF40E050E0F4
:101FB000281B390B4A0B5B0B862F90E0A0E0B0E0AA
:101FC000281739074A075B071CF4EFEFFFEF0FC034
:101FD000E60FF11D0CC070E0E617F70720F430970C
:101FE00031F0FB0104C0309711F0E61BF70B1093A2
:101FF000662ACF011F910895AF92BF92CF92DF92D0
:10200000EF92FF920F931F93CF93DF93EC01F42E87
:10201000E52EB22EA32E6801088119811093062B9C
:102020000093052BC8010E94BF0F9C0199838883F0
:102030008F2D9E2D8217930710F0998388832B2D67
:102040003A2D888199818217930710F0398328836C
:10205000888199818017910749F09093062B80938E
:10206000052B81E0F601808380939901DF91CF9168
:102070001F910F91FF90EF90DF90CF90BF90AF90A6
:1020800008959C0143B142704093642A93B19170CA
:102090009093652A442309F58091662A8823E9F004
:1020A00070E0992369F08FEF9FE7821B930B8617EF
:1020B00097071CF42FEF3FE710C0260F371F0DC006
:1020C000261737072CF42115310539F09B0105C07F
:1020D0002115310511F0261B370B4093662AC901E3
:1020E0000895AF92BF92CF92DF92EF92FF920F933B
:1020F0001F93CF93DF93EC017A01690158010881A6
:1021000019811093082B0093072BC8010E944110DE
:1021100099838883E816F90614F0F982E8828881A9
:1021200099818C159D0514F0D982C8828881998186
:102130008017910749F09093082B8093072B81E03B
:10214000F501808380939901DF91CF911F910F91C9
:10215000FF90EF90DF90CF90BF90AF9008959F9247
:10216000AF92BF92CF92DF92EF92FF920F931F93A5
:102170007B018C0159016A0193B082E09822909210
:10218000642A93B191709093652A9920D9F5809132
:10219000662A8823B9F1992329F0C801B7010E9462
:1021A0001C7C2EC080912D0282FF1AC080916B2A68
:1021B000813059F0813010F0823021F5C801B7012B
:1021C00020E030E040E251E406C0C801B70120E061
:1021D00030E040E851E40E94CA7D88239CF00AC0A8
:1021E000C801B70120E030E040E050E00E94807C70
:1021F000882341F0C801B701A60195010E941B7C0C
:102200007B018C019092662AB701C8011F910F9142
:10221000FF90EF90DF90CF90BF90AF909F90089588
:1022200023B122702093642A93B191709093652A10
:102230001092042B1092032B222379F48091662AAA
:10224000882359F0992319F081E090E002C08FEFC4
:102250009FEF9093042B8093032B2093662A809109
:10226000032B9091042B0895EF92FF920F931F93ED
:10227000CF93DF93582F20916E1F803109F04DC00E
:1022800030E0A0E0B0E086E299E0289F7001299F4D
:10229000F00C389FF00C1124062F10E0C42FD0E072
:1022A000742F7295770F770F707C4695469547701F
:1022B000562F5295550F550F507C66956695677051
:1022C000FD01EE0FFF1FEA0FFB1FEE0DFF1DE45A8D
:1022D000F34F2081922F9295969596959370318128
:1022E000832F8770880F880F892B90E080179107C4
:1022F00034F42F73252B2083387F362B08C08C179E
:102300009D0734F02F73272B2083387F342B3183A4
:102310001196A034B105A1F686C030E0A0E0B0E08F
:1023200083E994E0289FE001299FD00D389FD00DCC
:102330001124062F10E0242F30E0F42EF294FF0C2D
:10234000FF0C80ECF822469546954770762F7295E3
:10235000770F770F707C669566956770852F90E094
:10236000FC01689415F8EE0FFF1F1694E1F7880F33
:10237000991FE80FF91FEC0FFD1FEA0FFB1FEE0F6F
:10238000FF1FEE5EFB4F9081929596959695937008
:1023900081818770880F880F892B90E080179107C3
:1023A000ECF4852F90E0FC01689415F8EE0FFF1F08
:1023B0001694E1F7880F991FE80FF91FEC0FFD1F26
:1023C000EA0FFB1FEE0FFF1FEE5EFB4F80818F7346
:1023D000872B80838181887F862B1FC0821793077C
:1023E000ECF0852F90E0FC01689415F8EE0FFF1FCC
:1023F0001694E1F7880F991FE80FF91FEC0FFD1FE6
:10240000EA0FFB1FEE0FFF1FEE5EFB4F80818F7305
:102410008F2980838181887F842B81831196A034CA
:10242000B10509F09BCFDF91CF911F910F91FF90E4
:10243000EF9008953F924F925F926F927F928F92AA
:102440009F92AF92BF92CF92DF92EF92FF920F9343
:102450001F93DF93CF93CDB7DEB760970FB6F89495
:10246000DEBF0FBECDBF80913B0283FF0AC08091CB
:1024700077018F5F80937701883018F087E0809331
:1024800077018091390283FF09C0809177018150E3
:1024900080937701883010F010927701DE01119659
:1024A000E1EBF1E080E101900D928150E1F7809144
:1024B0006E1F482F50E086E299E0489FF001499F47
:1024C000F00D589FF00D1124EA5AF34FE081E330EC
:1024D00018F4E13048F405C0E33049F0E93048F43D
:1024E00003C0ACE0EA2E05C0F7E0EF2E02C0E5E045
:1024F000EE2E8091E002882309F444C08091E50229
:10250000813009F03FC08091EE038823D9F180919A
:10251000B60290E0FC01EE0FFF1FE80FF91F86E204
:1025200099E0489F9001499F300D589F300D11242C
:10253000E20FF31FE25AF34F9091022B9F708081BC
:10254000807F892B80838091B60290E0FC01EE0FA2
:10255000FF1FE80FF91FE20FF31FE45AF34F8081CA
:10256000817C8E6280838091B60290E0FC01EE0F48
:10257000FF1FE80FF91FE20FF31FE45AF34F8081AA
:1025800081608083F090022B00E010E03E0108940F
:10259000611C711CAE2CBB2446E2842E49E0942EB3
:1025A0003CE0532E4424439427E0322EF801EE0FF2
:1025B000FF1FE55FFD4F30818091560290915702D9
:1025C000002E02C0969587950A94E2F7282F217075
:1025D000367F932F922B9083892F869581702817B1
:1025E00009F4D0C092FDC2C0213009F0BFC03960EB
:1025F0003083F301E00FF11FE0818E2F90E06E2D0C
:1026000070E00E945C7E9B0180917701860F809331
:102610007801883010F0309278012A9DC0012B9DFE
:10262000900D3A9D900D11242E2F281B80916E1F26
:1026300090E0889DF001899DF00D989DF00D11248A
:10264000EA5AF34F8081833018F4813068F405C072
:10265000833081F0893098F407C0E22FF0E0E05732
:10266000FC4FF490FA940BC0E22FF0E0EC50F64FE0
:10267000F49005C0E22FF0E0E550F64FF490859D10
:10268000F0011124EF0DF11DE057FC4FE491E150F2
:10269000F0E0EE0FFF1FE450FC4F859194912091E4
:1026A0007801D22EDD0CCC248C0D9D1D0E94B60D20
:1026B0005F9A4092EE038091E002882309F456C0AD
:1026C0008091E502813009F051C020916E1F30E009
:1026D0008091B60290E0FC01EE0FFF1FE80FF91F9A
:1026E000A901489D9001499D300D589D300D112440
:1026F000E20FF31FE25AF34F9F2D9F708081807F7E
:10270000892B80838091B60290E0FC01EE0FFF1FC1
:10271000E80FF91FE20FF31FE25AF34F909178018F
:1027200097709295907F80818F78892B808380919C
:10273000B60290E0FC01EE0FFF1FE80FF91FE20F59
:10274000F31FE45AF34F8081817C886180838091FC
:10275000B60290E0FC01EE0FFF1FE80FF91FE20F39
:10276000F31FE45AF34F808181608083F801EE0FFC
:10277000FF1FE55FFD4F8081982F9170990F8D7F2E
:10278000892B80830F5F1F4F0031110509F00ECF99
:10279000F092022B8091560290915702892B21F5DD
:1027A0008091EE03882301F15F981092EE038091EF
:1027B000B60290E020916E1F30E0FC01EE0FFF1F8B
:1027C000E80FF91F86E299E0AC01249FC001259F24
:1027D000900D349F900D1124E80FF91FE45AF34F28
:1027E0008081817C8861808360960FB6F894DEBF1B
:1027F0000FBECDBFCF91DF911F910F91FF90EF9052
:10280000DF90CF90BF90AF909F908F907F906F9010
:102810005F904F903F900895BF92CF92DF92EF92DA
:10282000FF920F931F93082FE0915A2AF0E0E45D86
:10283000F54DB48881E0B81609F47AC0B81628F0CE
:10284000E3E0BE1609F0FDC0C2C0209176023091CF
:102850007702C9014E970C9718F424EE3FEF02C19E
:10286000C9018A970A9718F42DEE3FEFFBC0C90102
:10287000C4970A9718F423EF3FEFF4C0C901CE972D
:102880000A9708F464C0C901885490400A9718F464
:102890002BEF3FEFE7C0C901825590400A9718F42B
:1028A0002DEF3FEFDFC0C9018C5590400D9708F424
:1028B000ACC0C90189569040059708F4C2C0C9014F
:1028C0008F569040099708F4C8C0C90188579040B6
:1028D0000A9708F4BFC0C901825890400A9708F4CB
:1028E000B6C0C9018C5890400A9708F4ADC0C90120
:1028F000865990400A9718F426E030E0B3C0C90129
:10290000805A9040889718F427E030E0ABC0C901A6
:10291000885C9040449718F428E030E0A3C02C5D18
:1029200030402F31310508F08CC029E030E09AC0EA
:102930002091760230917702C9014E970C9718F4D6
:1029400022EF3FEF8FC0C9018A970D9718F427EF48
:102950003FEF88C0C901C797079718F42AEF3FEFE8
:1029600081C0C901CE970D9708F440C0C9018B54AE
:1029700090400F9708F441C0C9018A5590400A97CA
:1029800008F443C0C901845690400A9708F459C01E
:10299000C9018E5690400D9708F45FC0C9018B574E
:1029A0009040489708F456C0C901835990408397D6
:1029B00008F456C0C901865B9040859708F447C06B
:1029C0002B5D30402032310508F43EC03AC02091E2
:1029D000760230917702C9014E970C9718F428EFD0
:1029E0003FEF40C0C9018A97409718F42CEF3FEFA2
:1029F00039C0C901CA970D9718F42EEF3FEF32C0C6
:102A0000C90187549040419718F42FEF3FEF2AC037
:102A1000C901885590404D97A0F0C9018557904055
:102A2000C097D8F0C901855A9040CC9798F0C90159
:102A3000815E90400E97A0F02F5E30402C30310523
:102A400048F020E030E00EC025E030E00BC024E08C
:102A500030E008C022E030E005C021E030E002C0F4
:102A600023E030E010E0045D154D20503F4FB901E8
:102A7000882777FD8095982F0E941A7D6B017C0135
:102A8000609176027091770280E090E00E94187D5C
:102A9000EB2DF0E0EE0FFF1FEE0FFF1FE758FE4F8C
:102AA00020813181428153810E94CE7D9B01AC0106
:102AB00060E070E080E792E40E94847C21E338E0EB
:102AC0004CEA5CEB0E94847C9B01AC01C701B6011F
:102AD0000E941C7C0E94EC7CF80162831F910F9184
:102AE000FF90EF90DF90CF90BF9008953F924F926C
:102AF0005F926F927F928F929F92AF92BF92CF928E
:102B0000DF92EF92FF920F931F93CF93DF93A090EA
:102B10002B02A694A694BB24B394AB209A2D990FB4
:102B2000809166028C7FB0912D02B695B695B170FA
:102B3000892B8B2BB0904302B694B694CC24C394CB
:102B4000BC202B2D220F220F837FC0904502C694FC
:102B5000C694DD24D394CD209C2D990F990F990F05
:102B6000822B892B40913102469546954170342F36
:102B70003295307F8F7C20913902269526952170E1
:102B8000922F9295990F907E832B892B90913B02E7
:102B9000969596959170392F3295330F330F307C7F
:102BA0008F7B832B80936602022F10E0000F111F92
:102BB000000F111F692F70E093E0660F771F9A9541
:102BC000E1F7C42FD0E085E0CC0FDD1F8A95E1F757
:102BD00020916502922F96959270902B822F82956C
:102BE00086958170982B962B269526952071292BFA
:102BF0002C2B20935E02E0907C02F0907D0221E07D
:102C0000E216F10419F45091390109C0E114F104FC
:102C100011F451E005C0509135025695569551700A
:102C2000852F81708295880F807E909165029F7DAF
:102C3000982B90936502C7010397029720F04CE010
:102C4000E416F10429F4D090390181E0D82207C0BC
:102C5000DD2492E0E916F10411F4DD24D3949D2DD6
:102C6000990F990F809165028B7F892B8093650264
:102C7000E4E0EE16F10421F0FCE0EF16F10421F49B
:102C800030913901317007C030914B02369536953D
:102C9000317009F031E0932F9170990F990F990FCE
:102CA00080916502877EA0914902A695A695A170A4
:102CB0002A2F2295207F892B822B80936502809179
:102CC000E502882359F08091670281608093670252
:102CD000909167029170E4E7FFE120C08091711F3D
:102CE000882381F480916F02882361F48091EF033F
:102CF000882341F480915B2A882321F48091282A3B
:102D0000882341F0909139019170809167028E7F04
:102D1000892BDCCF809167028E7FD8CF808188237A
:102D200019F090913901917031962FE1E438F20752
:102D3000A9F7809167028E7F892B8093670245E017
:102D4000E416F10421F480916502806403C080914F
:102D500065028F7B809365028090292890902A28B5
:102D600090926C0280926B0288E0E816F104D1F434
:102D700080916D2A823091F480916B2A833071F4B6
:102D800081E090E00090E90202C0880F991F0A9448
:102D9000E2F7909359028093580204C010925902AE
:102DA000109258024091E002E0E0442309F4E1E08F
:102DB000809165028E7F8E2B80936502442321F0E3
:102DC00080916602806809C0909139019795992792
:102DD0009795809166028F77892B80936602602B8E
:102DE000712B6C2B7D2B8091650282958695869543
:102DF000817090E004E0880F991F0A95E1F7682B35
:102E0000792B8C2D90E016E0880F991F1A95E1F729
:102E1000682B792B8A2F90E09695982F8827979585
:102E20008795682B792B9B2D80E0682B792B9A2D29
:102E3000990F990F80E0682B792B9B2F990F990F91
:102E4000990F80E0682B792B20916602221F2227A0
:102E5000221F922F9295907F80E0682B792B2091F2
:102E600067022170922F9295990F990F907C80E0C4
:102E7000682B792B9E2F9295990F907E80E0682B7E
:102E8000792B852F90E0682B792B8D2D90E0880F82
:102E9000991F682B792B932F990F80E0682B792B42
:102EA0007093600260935F026090E602C62DD0E0EE
:102EB00021E030E0C901062C02C0880F991F0A9456
:102EC000E2F79093690280936802E4E0EE16F10461
:102ED00009F42EC2F5E0EF16F10464F452E0E516B1
:102EE000F10411F163E0E616F1040CF0E7C0F7FE1F
:102EF00046C25BC277E0E716F10409F4DFC0E8E000
:102F0000EE16F10434F4F5E0EF16F10409F04DC2C9
:102F100042C229E0E216F10409F4D0C04CE0E41604
:102F2000F10409F042C204C28091350282FF08C058
:102F30000090E70202C0220F331F0A94E2F726C274
:102F4000442309F46CC090916A1F992309F44BC083
:102F500080916B1F482F50E04F70507060E070E020
:102F600020E030E0E92FF0E001E0E02EF12C012D2F
:102F7000112D10C0C901840F951F5701680104C0AD
:102F8000AA0CBB1CCC1CDD1C8A95D2F76A297B29B4
:102F90002F5F3F4FE217F3076CF780913901FE0175
:102FA000E65CFE4FE081CC57DD4F288140E050E0E9
:102FB000882311F441E050E08091E8028F7002C054
:102FC000440F551F8A95E2F7409550956423752369
:102FD0008E2F90E02F7002C0880F991F2A95E2F77C
:102FE000682779275AC040913901FE01E65CFE4FFF
:102FF0008081CC57DD4F288190E02F7002C0880F70
:10300000991F2A95E2F750E02091E8022F7002C044
:10301000440F551F2A95E2F784279527C2C1909146
:103020006A1F992309F43EC080916B1F482F50E01E
:103030004F70507060E070E020E030E0E92FF0E089
:1030400011E0E12EF12C012D112D10C0C901840FCA
:10305000951F5701680104C0AA0CBB1CCC1CDD1CC9
:103060008A95D2F76A297B292F5F3F4FE217F30732
:103070006CF78091390120E030E0882311F421E0E1
:1030800030E08091E8028F7002C0220F331F8A95D2
:10309000E2F7209530956223732370935902609371
:1030A000580283C18091390190E02091E8022F708D
:1030B00002C0880F991F2A95E2F773C1BB2309F05C
:1030C00070C1FE01E957F04E7080372C3294B0EF9A
:1030D0003B2220916E1F30E040E050E000E010E025
:1030E00060E070E04E01880C991CCE01F6E0880F7C
:1030F000991FFA95E1F7880E991E83E994E06C0117
:103100002C9DC0012D9D900D3C9D900D1124880E8D
:10311000991EE1E0AE2EB12CC12CD12C86E299E0B3
:10312000289F2001299F500C389F500C1124832D7B
:10313000840FA82FB0E020E1621669F4FD01EE0FC4
:10314000FF1FEA0FFB1FE40DF51DE45AF34F8081CA
:1031500080FF3AC00DC0A80DB91DAA0FBB1FAE5EFF
:10316000BB4F8C91982F917081FF0FC09923E1F094
:10317000D601C501042E04C0880F991FAA1FBB1FCA
:103180000A94D2F7682B792B1FC0992369F0D601D6
:10319000C501042E04C0880F991FAA1FBB1F0A94E3
:1031A000D2F7082B192B10C0D601C501042E04C07C
:1031B000880F991FAA1FBB1F0A94D2F7809590957C
:1031C00068237923082319234F5F5F4F403451054B
:1031D00009F0ADCF00935C0210935D0260935A0238
:1031E00070935B02FE01E856F04E30817316B1F425
:1031F000FE01E65CFE4F8081FE01EC57FD4F208111
:1032000090E02F7002C0880F991F2A95E2F7862759
:103210009727909359028093580204C070935902E3
:103220006093580280916A02883C08F17316B9F4E1
:10323000FE01E65CFE4F8081CC57DD4F288190E097
:103240002F7002C0880F991F2A95E2F780279127D7
:10325000862B972B909359028093580206C0062B19
:10326000172B109359020093580210926A0247E0FC
:10327000E416F10429F059E0E516F10409F095C0CF
:103280007720A1F480918202803108F08EC02091D5
:10329000390130E002C0220F331F8A95E2F7809196
:1032A000580290915902822793277BC061E07616DD
:1032B00079F420918202203208F077C0203108F49E
:1032C00074C08091390190E030E02051304024C03A
:1032D00072E0771679F420918202203308F065C0FD
:1032E000203208F462C08091390190E030E0205231
:1032F000304012C083E0781609F057C02091820256
:10330000203408F052C0203308F44FC080913901B6
:1033100090E030E02053304002C0880F991F2A957A
:10332000E2F72091580230915902282739272EC000
:1033300080917E028370A9F081E00E94790820913B
:10334000DD023091DE024091620250E0F9014E9FB1
:1033500090014F9F300D5E9F300D1124282B392B8B
:1033600015C0009163021091640281E00E94790807
:10337000082B192B109359020093580216C0009085
:103380002C2802C0220F331F0A94E2F7309359020F
:10339000209358020AC080916302909164028829A8
:1033A0009929909359028093580260915F0270911D
:1033B0006002809158029091590240915E020E94F1
:1033C000040DDF91CF911F910F91FF90EF90DF904F
:1033D000CF90BF90AF909F908F907F906F905F90B5
:1033E0004F903F900895DF92EF92FF920F931F93BB
:1033F000CF93DF9320916E1F803109F48CC0622F30
:1034000070E0282F30E084E890E0289FD001299FC9
:10341000B00D389FB00D112486E299E0689FA0019D
:10342000699F500D789F500D1124FD01E40FF51F89
:10343000E850FC4FE656FF4FE190AC5BB94EA65604
:10344000BF4FED9280818C931296329680818C933F
:1034500082918E93F901EC5BF94E48505C4F420F1C
:10346000531FDA0117968C91878350E0E90106E03B
:10347000CC0FDD1F0A95E1F7220F331FC20FD31FB8
:1034800083E994E0689F8001699F100D789F100D7B
:1034900011240C0F1D1F852F90E09E01280F391F4E
:1034A000220F331FB901625A794EF801E80FF91F54
:1034B000EE0FFF1FDF01AE5EBB4F8C91482F429590
:1034C00046954695437011969C919770990F990F68
:1034D000942B492F4295440F440F407C8F73842BCB
:1034E000DB018C9396959695977011968C91119718
:1034F000887F892B11968C93215A394EED5EFB4FB4
:103500009081987FF90180818770892B80835F5F2C
:10351000E51608F679C030E086E299E0A901489FF7
:103520009001499F300D589F300D1124F901E8504A
:10353000FC4FE05AF74FD080D092A41E8291809326
:10354000A31E329681918093A51E80818093A61E32
:10355000349780818093A21E00E0E901802F90E0E3
:10356000DC01AA0FBB1FA80FB91F9D012855314EC2
:10357000BD016C0F7D1F4CE5E42E4CE0F42EE60EF1
:10358000F71EF7011081912F9170F90180818E7FD4
:10359000892B8083AD014655514EFB01E25AF34F12
:1035A0008081FA018083912F9E73F9018081817C53
:1035B000892B8083A755B14E635A734FFB019081CD
:1035C000987F8C918770892B8C9312951695169500
:1035D0001370D70111969C919770990F990F912BA9
:1035E000492F4295440F440F407CF90180818F732D
:1035F000842B8083969596958181887F892B818302
:103600000F5FD01608F0AACFDF91CF911F910F91D5
:10361000FF90EF90DF900895CF92DF92EF92FF92AC
:103620000F931F93CF93DF93462F20916E1F80310E
:1036300009F4A3C0622F70E0C82FD0E050E084E806
:1036400090E0489FD001499FB00D589FB00D1124C4
:10365000AC5BB94EA656BF4FCD90C89FF001C99F35
:10366000F00DD89FF00D112486E299E0689F90013B
:10367000699F300D789F300D1124E20FF31FE85041
:10368000FC4FE656FF4FC1928C9180833296129682
:103690008C9180838E91829328503C4F2C0F3D1F3C
:1036A000FA01EC5BF94E8781D90117968C93DD24E2
:1036B0008E01000F111FCE0126E0880F991F2A9559
:1036C000E1F7080F191F83E994E0FC016E9FC00128
:1036D0006F9F900D7E9F900D1124080F191F7A0186
:1036E00096E0EE0CFF1C9A95E1F7440F551FE40E8F
:1036F000F51E8D2D90E09801280F391F220F331FE2
:10370000B9016E5E7B4FF701E80FF91FEE0FFF1F47
:10371000DF01A25AB94E8C91482F429546954695A5
:10372000437011969C919770990F990F942B492F84
:103730004295440F440F407C8F73842BDB018C93A4
:1037400096959695977011968C911197887F892BF5
:1037500011968C932D5E3B4FE15AF94E9081987FE4
:10376000F90180818770892B8083D394CD1408F66A
:10377000CC58D04E81E088837EC030E0D090A41E2B
:1037800086E299E0A901489F9001499F300D589F1A
:10379000300D1124F901E850FC4FE05AF74FD08268
:1037A0008091A31E829332968091A51E8193809171
:1037B000A61E808334978091A21E808300E0E901D9
:1037C000802F90E0DC01AA0FBB1FA80FB91FBD011D
:1037D0006C0F7D1F9B01245A334F88EAE82E8EE13F
:1037E000F82EEA0EFB1EF7011081912F9170F9015E
:1037F00080818E7F892B8083AB01425A534FFD011C
:10380000E655F14E8081FA018083912F9E73F90174
:103810008081817C892B8083635A734FA755B14E79
:103820009C91987FDB018C918770892B8C931295EA
:10383000169516951370F70191819770990F990F4E
:10384000912B492F4295440F440F407CD9018C9114
:103850008F73842B8C939695969511968C911197D6
:10386000887F892B11968C930F5FD01608F0A8CF14
:1038700081E08093EF0381E080939901DF91CF9104
:103880001F910F91FF90EF90DF90CF900895CF930D
:10389000DF9320916E1F30E0C82FD0E084E890E0E5
:1038A000C89FF001C99FF00DD89FF00D112486E24A
:1038B00099E0AC01249FC001259F900D349F900D8D
:1038C0001124E80FF91FE850FC4FE656FF4F8FE038
:1038D000819388E18083329681E08083129260E058
:1038E00070E0AE01440F551FCE01E6E0880F991F2E
:1038F000EA95E1F7480F591F83E994E0FC012E9FF8
:10390000C0012F9F900D3E9F900D1124480F591F0D
:10391000FA01E60FF71FEE0FFF1FDF01AE5EBB4F90
:1039200082E08C9311968C911197887F8460119618
:103930008C93ED5EFB4F8081877080836F5F7F4F3C
:103940006034710529F7CC58D04E81E0888380938C
:103950009901DF91CF910895CF93DF9380916E1FEE
:1039600090E026E239E0A901849F9001859F300D07
:10397000949F300D1124F901E850FC4FE05AF74FA5
:103980008FE0808388E18293329681E08193108278
:103990003497108240E050E0B901FA01EE0FFF1FAA
:1039A000E40FF51FE60FF71FDF01A45AB34F8C9108
:1039B0008E7F8C93CF01825A934F20E3EC012883B2
:1039C0008C91817C88618C93E35AF34F808187705E
:1039D00080838C918F738C9311968C911197887F33
:1039E000846011968C934F5F5F4F40345105A9F668
:1039F00081E08093EF0380939901DF91CF91089547
:103A00001F9310E0812F0E94F3191F5F1131D1F72E
:103A100080912C2A8093432A80912E2A8093452AD4
:103A20008091302A9091312AA091322AB091332A84
:103A30008093472A9093482AA093492AB0934A2A10
:103A400080913E2A8093552A8091402A8093572A5C
:103A500080912D2A8093442A80912F2A8093462A90
:103A60008091342A9091352AA091362AB091372A34
:103A700080934B2A90934C2AA0934D2AB0934E2AC0
:103A800080913F2A8093562A8091412A8093582A18
:103A90001F9108951F9310E0812F612F0E940C1B2E
:103AA0001F5F1131C9F78091432A80932C2A80919E
:103AB000452A80932E2A8091472A9091482AA091E6
:103AC000492AB0914A2A8093302A9093312AA093B0
:103AD000322AB093332A8091552A80933E2A8091CE
:103AE000572A8093402A8091442A80932D2A8091DE
:103AF000462A80932F2A80914B2A90914C2AA0919C
:103B00004D2AB0914E2A8093342A9093352AA0935F
:103B1000362AB093372A8091562A80933F2A809183
:103B2000582A8093412A1F9108951F9310E0812FF6
:103B30000E94471C1F5F1031D1F70E94AC1C1F91DF
:103B40000895CF92DF92EF92FF920F931F93CF933E
:103B5000DF93082FE42E20916E1F803161F430E056
:103B6000F62E86E299E0289F6001299FD00C389FAD
:103B7000D00C112482C130E0162F83E994E0289FF5
:103B8000E001299FD00D389FD00D112402C1612F73
:103B900070E0412F4F7050E0802F90E0DC0126E074
:103BA000AA0FBB1F2A95E1F7880F991FA80FB91F0D
:103BB000AC0FBD1FA60FB71FAA0FBB1FAE5EBB4F3A
:103BC000802F90E0FC0136E0EE0FFF1F3A95E1F701
:103BD000880F991FE80FF91FEC0FFD1FE40FF51F69
:103BE000EE0FFF1FEE5EFB4F908191708C918E7FE8
:103BF000892B8C93802F90E0DC0126E0AA0FBB1F5D
:103C00002A95E1F7880F991FA80FB91FAC0FBD1FA8
:103C1000A60FB71FAA0FBB1FAE5EBB4F802F90E051
:103C2000FC0136E0EE0FFF1F3A95E1F7880F991F70
:103C3000E80FF91FEC0FFD1FE40FF51FEE0FFF1F3C
:103C4000EE5EFB4F908192708C918D7F892B8C93CF
:103C5000802F90E0DC0126E0AA0FBB1F2A95E1F738
:103C6000880F991FA80FB91FAC0FBD1FA60FB71F54
:103C7000AA0FBB1FAE5EBB4F802F90E0FC0136E069
:103C8000EE0FFF1F3A95E1F7880F991FE80FF91F14
:103C9000EC0FFD1FE40FF51FEE0FFF1FEE5EFB4F55
:103CA00090819C738C91837C892B8C93802F90E0E6
:103CB000DC0126E0AA0FBB1F2A95E1F7880F991FA8
:103CC000A80FB91FAC0FBD1FA60FB71FAA0FBB1FB0
:103CD000AE5EBB4F802F90E0FC0136E0EE0FFF1F81
:103CE0003A95E1F7880F991FE80FF91FEC0FFD1FB8
:103CF000E40FF51FEE0FFF1FEE5EFB4F80818295F4
:103D000086958695837091819770990F990F982B5E
:103D1000292F2295220F220F207C8C918F73822BCA
:103D20008C939695969511968C911197887F892BF7
:103D300011968C93802F90E0DC01F6E0AA0FBB1F58
:103D4000FA95E1F7880F991FA80FB91FAC0FBD1F97
:103D5000A60FB71FAA0FBB1FAD5EBB4F802F90E011
:103D6000FC0136E0EE0FFF1F3A95E1F7880F991F2F
:103D7000E80FF91FEC0FFD1FE40FF51FEE0FFF1FFB
:103D8000ED5EFB4F9081987F8C918770892B8C938F
:103D90001F5FE11608F0FBCEE02FF0E0EC58F04E8C
:103DA00081E0808370C02F2D30E08F2D8F7090E0E8
:103DB000D901AA0FBB1FA20FB31FAC0DBD1DBD01C2
:103DC000645A734FFC01EE0FFF1FE80FF91FEC0D53
:103DD000FD1D8F01045A134FE80198819170EB018A
:103DE00088818E7F892B8883AD01425A534F9F0172
:103DF000225A334FE90198819F70EA018881807FC0
:103E0000892B8883E901988190778F78892BEA0143
:103E10008883E901988190788F77892BEA018883DC
:103E2000E80198819E73EB018881817C892B8883CE
:103E3000A35AB34FE35AF34F9081987F8C918770C8
:103E4000892B8C93F8018081829586958695837065
:103E500091819770990F990F982B292F2295220FF6
:103E6000220F207C88818F73822B8883969596956C
:103E70008981887F892B8983F394EF1408F093CF8D
:103E800081E08093EF0381E080939901DF91CF91EE
:103E90001F910F91FF90EF90DF90CF9008952F9298
:103EA0003F924F925F926F927F928F929F92AF92CA
:103EB000BF92CF92DF92EF92FF920F931F93DF9307
:103EC000CF9300D000D0CDB7DEB720916E1F8031E8
:103ED00009F0FEC0822E992486E299E0889E900126
:103EE000899E300D989E300D1124F901E85AF34F48
:103EF000A080D901A45AB34F9C917724739479225E
:103F0000F901E25AF34F80810FE0602E6822F82E0B
:103F1000F2941FE0F12247E0F422B82EBB1CBB2430
:103F2000BB1CE92EE6945FE1E522F901E35AF34F69
:103F3000C080C694C694C6949295969596959370B3
:103F400011961C911770110F110F192BDD24D394AA
:103F5000190172C02D2D30E0C9010197AC01440F49
:103F6000551F480F591F420D531DBA01645A734F14
:103F7000D901AA0FBB1FA20FB31FA20DB31DCD0104
:103F8000845A934F9A838983FC0190819170FB013D
:103F900080818E7F892B80839A01225A334FEEE5F0
:103FA0004E2EECE05E2E4A0E5B1EF20190819F7059
:103FB000F9018081807F892B8083F2019081907745
:103FC0008F78892BF9018083F201908190788F7727
:103FD000892BF9018083E981FA8180818295869518
:103FE0008695837091819770990F990F982B292F3F
:103FF0002295220F220F207CFB0180818F73822B60
:104000008083969596958181887F892B8183435AF9
:10401000534FA35AB34F9C91987FDA018C918770CC
:10402000892B8C93E981FA8190819E73DB018C91BD
:10403000817C892B8C93D394AD1408F08BCF8A2D7F
:1040400090E0FC01EE0FFF1FE80FF91F86E299E0F8
:104050009C01829EC001839E900D929E900D112422
:10406000E80FF91FAF01445A534FDA018C918E7F4C
:1040700087298C93CF01825A934FB7E0FB22F294A9
:1040800030EFF322B794BB24B794F628FB28DC0169
:10409000FC92912F9295990F990F907CDA018C9157
:1040A0008F73892B8C93E35AF34FCC0CCC0CCC0C34
:1040B000169516951C291083BFE1EB22EE0CFA0130
:1040C0008081817C8E29808381E08093EF03F1C021
:1040D000C22EDD24E82EFF2484E890E0E89ED00183
:1040E000E99EB00DF89EB00D112486E299E09C0186
:1040F000C29EC001C39E900DD29E900D1124A80FA8
:10410000B91FFD01EE56FB4F5080FD01EE5EFB4FE7
:104110008081442443944822082F06950170382F4B
:10412000369536953F708295869586958370118178
:104130001770110F110F182BAD5EBB4FAC90A694EA
:10414000A694A694BB24B3943701660C771C470150
:1041500096E0880C991C9A95E1F7A301480D591D2A
:1041600083E994E0DC01CA9EC001CB9E900DDA9EEB
:10417000900D1124480F591F5C834B8359C0EB2DC0
:10418000F0E031974B815C814E0F5F1F3196440FF9
:10419000551FB2E12B2EB4E03B2E240E351E8B8131
:1041A0009C81E80FF91FEE0FFF1FBF016E5E7B4F72
:1041B000DB019C919170D1018C918E7F892B8C9326
:1041C000DB019C9192708D7F892BD1018C93DB0157
:1041D0009C919C73837C892BD1018C93DB012C9166
:1041E000229526952695237011969C919770990F8C
:1041F000990F922B292F2295220F220F207C8F734B
:10420000822BD1018C939695969511968C9111974E
:10421000887F892B11968C934D5E5B4FED5EFB4F33
:104220009081987FFA0180818770892B8083B39475
:104230005B1408F0A4CFF301E80DF91D83E994E0C5
:10424000AC01C49EC001C59E900DD49E900D11245A
:10425000E80FF91FE50DF11DEE0FFF1FDF01AE5E48
:10426000BB4F0170000F02703F70330F330F0429F2
:10427000812F8295880F880F807C032B082B0C934D
:104280001695169511968C911197887F812B119612
:104290008C93ED5EFB4FAA0CAA0CAA0C8081877050
:1042A0008A29808384E79FE1E80EF91E81E0D70127
:1042B0008C9380917C0290917D028930910511F060
:1042C000079719F481E0809399010F900F900F9058
:1042D0000F90CF91DF911F910F91FF90EF90DF90A2
:1042E000CF90BF90AF909F908F907F906F905F9096
:1042F0004F903F902F9008952F923F924F925F9250
:104300006F927F928F929F92AF92BF92CF92DF92E5
:10431000EF92FF920F931F93DF93CF9300D000D0C3
:104320000F92CDB7DEB740916E1F803109F009C101
:10433000442E552486E299E0489EA001499E500DE6
:10434000589E500D1124FA01E85AF34F208130E0B5
:10435000F901EE0FFF1FE20FF31FE40FF51FBF017E
:10436000645A734FDB019C91662463946922DF01D8
:10437000A25AB34F8C91B82FBF70B983782E771C97
:104380007724771CE82EE294AFE0EA2217E0E122DE
:10439000B92EB6948FE1B822E35AF34FA080A694C9
:1043A000A694A6949295969596959370DB01119696
:1043B000FC90F122FF0CFF0CF92A1B821A82690182
:1043C00016010894210831084A0174C0C601EA8127
:1043D000FB818E1B9F0B9C01220F331F280F391F5F
:1043E000280D391DB901645A734FDA01AA0FBB1F9A
:1043F000A40FB51FA80DB91D8D01045A134FF80164
:1044000090819170FB0180818E7F892B8083A9012F
:10441000425A534FCD01825A934F9D838C83FC01A6
:1044200090819F70FA018081807F892B8083EC814D
:10443000FD81908190778F78892BFA018083EC81C0
:10444000FD81908190788F77892BFA018083F80124
:104450008081829586958695837091819770990F5A
:10446000990F982B492F4295440F440F407CFB0134
:1044700080818F73842B8083969596958181887F28
:10448000892B8183235A334FA35AB34F9C91987F32
:10449000D9018C918770892B8C93F80190819E7340
:1044A000DB018C91817C892B8C93EA81FB81319695
:1044B000FB83EA83A1012A813B81421B530B2C150C
:1044C0003D0509F083CF86E299E0489EA001499E10
:1044D000500D589E500D1124DA01A45AB34F8C91FF
:1044E0008E7F86298C93CA01825A934F37E0E3224C
:1044F000E29410EFE1227794772477946981E62A99
:10450000E728FC01E0829F2D9295990F990F907CEE
:104510008C918F73892B8C93435A534FAA0CAA0CFE
:10452000AA0CF694F694FA28FA01F082FFE1BF2271
:10453000BB0C8C91817C8B298C9381E08093EF0361
:10454000F5C0842E9924282F30E03B832A8384E809
:1045500090E0289FF001299FF00D389FF00D112465
:1045600086E299E0BC01869EC001879E900D969ED2
:10457000900D1124E80FF91FEE56FB4F408150E0DB
:10458000220F331F8A819B81E6E0880F991FEA95ED
:10459000E1F7280F391F83E994E0DC018A9EC0010E
:1045A0008B9E900D9A9E900D1124280F391FF901B2
:1045B000E40FF51FEE0FFF1FDF01AE5EBB4F8C91C6
:1045C000332433943822082F06950170B82EB69400
:1045D000B6941FE0B12282958695869583701196D8
:1045E0001C911770110F110F182BED5EFB4FA0805F
:1045F000A694A694A694EE24FF246A0126010894AA
:1046000041085108390153C096012E193F09260D62
:10461000371D220F331F3D832C83A9014E5E5B4F54
:10462000D301A80FB91FAA0FBB1FBD016E5E7B4F40
:10463000FB0190819170FA0180818E7F892B8083AC
:10464000FB01908192708D7F892BFA018083FB01A1
:1046500090819C73837C892BFA018083FB012081EC
:10466000229526952695237091819770990F990F21
:10467000922B292F2295220F220F207C8F73822BC1
:10468000FA018083969596958181887F892B818315
:10469000EC81FD81ED5EFB4FAD5EBB4F9C91987F41
:1046A00080818770892B80830894E11CF11CC201F2
:1046B0008E199F09EC14FD0409F0A6CF84E890E060
:1046C0002A813B81289FF001299FF00D389FF00D32
:1046D000112486E299E0BC01869EC001879E900D60
:1046E000969E900D1124E80FF91FDF01AE5EBB4FBF
:1046F0000170000F02707FE0B722BB0CBB0C0329D6
:10470000812F8295880F880F807C0B29082B0C93B2
:10471000ED5EFB4FAA0CAA0CAA0C169516951A2949
:1047200010832C58304E81E0D9018C9380917C020B
:1047300090917D028930910511F0079719F481E07D
:10474000809399010F900F900F900F900F90CF9141
:10475000DF911F910F91FF90EF90DF90CF90BF906E
:10476000AF909F908F907F906F905F904F903F9011
:104770002F900895CF93DF93782F6F5F20916E1F56
:104780008031B9F530E086E299E0289FA001299FA9
:10479000500D389F500D112429C0862F90E0FC0148
:1047A000EE0FFF1FE80FF91FE40FF51FDF01A45AFA
:1047B000B34F8C918E7F8C93CF01825A934F20E31D
:1047C000EC0128838C91817C88618C93E35AF34FB0
:1047D0008081877080838C918F738C9311968C91DC
:1047E0001197887F846011968C936F5F6034A8F274
:1047F00088C030E083E994E0289FA001299F500DF4
:10480000389F500D11247AC0262F30E0872F90E07A
:10481000FC01B6E0EE0FFF1FBA95E1F7880F991F74
:10482000E80FF91FE40FF51FE20FF31FEE0FFF1F54
:10483000EE5EFB4F80818E7F8083872F90E0FC01AE
:10484000B6E0EE0FFF1FBA95E1F7880F991FE80F4A
:10485000F91FE40FF51FE20FF31FEE0FFF1FEE5ECF
:10486000FB4F808182608083872F90E0FC01B6E05F
:10487000EE0FFF1FBA95E1F7880F991FE80FF91F98
:10488000E40FF51FE20FF31FEE0FFF1FEE5EFB4F6D
:104890008081837C8083872F90E0FC01B6E0EE0F5F
:1048A000FF1FBA95E1F7880F991FE80FF91FE40F72
:1048B000F51FE20FF31FEE0FFF1FEE5EFB4F80812F
:1048C0008F7380838181887F84608183872F90E0CC
:1048D000FC01B6E0EE0FFF1FBA95E1F7880F991FB4
:1048E000E80FF91FE40FF51FE20FF31FEE0FFF1F94
:1048F000ED5EFB4F8081877080836F5F603408F4CA
:1049000083CFDF91CF910895DF92EF92FF920F93C3
:104910001F93CF93DF9380916E1F90E026E239E0E2
:10492000829FF001839FF00D929FF00D1124E850BB
:10493000FC4F10821182C0E0D0E034E8E32EF12C6D
:1049400006E219E0DD24D3944C2F80916E1F282FAE
:1049500030E0CE9DF001CF9DF00DDE9DF00D1124D5
:10496000209FC001219F900D309F900D1124E80FD2
:10497000F91FEE56FB4FE081DC01A850BC4F8C9133
:104980008E1718F4EC93C093861FCE9DF001CF9D37
:10499000F00DDE9DF00D1124209FC001219F900D90
:1049A000309F900D1124E80FF91FED56FB4FE08169
:1049B000DC01A850BC4F11968C9111978E1710F402
:1049C0001196EC93FE01E551FD4FD082CE9DF00192
:1049D000CF9DF00DDE9DF00D1124209FC001219F81
:1049E000900D309F900D1124E80FF91FEE56FB4FEC
:1049F000842F60810E94BA232196C031D10509F02D
:104A0000A3CF80916E1F282F30E086E299E0289F87
:104A1000F001299FF00D389FF00D1124E850FC4F54
:104A2000E05AF74F9081E056F8408081891720F4D2
:104A3000908380E18093861F86E299E0289FF001B1
:104A4000299FF00D389FF00D1124E850FC4FE15ADA
:104A5000F74F9081EF55F8408181891708F49183D1
:104A600081E08093FB0286E299E0289FF001299F74
:104A7000F00D389FF00D1124E85AF34F80E160816A
:104A80000E94BA23DF91CF911F910F91FF90EF9079
:104A9000DF9008951F938091370283FF0FC010911C
:104AA0002C281093F62A0E94A70B80932C2881179C
:104AB00029F081E08093272A809399011F9108951E
:104AC00080917E02837090E0009719F0039754F56F
:104AD00023C0609176027091770280E090E00E949E
:104AE000187D20E030E040EC52E40E94CE7D20E0D2
:104AF00030E040E752E40E94847C9B01AC0160E01E
:104B000074E284EF99E40E94847C0E94EC7C7093B0
:104B1000890060938800089584EF91E09093890064
:104B2000809388000895E1E8F0E01082808180930E
:104B3000800080818A6080830E946025EFE6F0E03B
:104B400080818260808308959F92AF92BF92CF92BE
:104B5000DF92EF92FF920F931F93DF93CF9300D0DA
:104B600000D0CDB7DEB780917C0290917D0282307B
:104B70009105D1F00C97C1F080916B2A90E061E033
:104B800070E00E94DD0E982F843008F093E090933F
:104B90006B2A8091162B981739F09093162B81E091
:104BA00080939A01809399018091712A882309F456
:104BB000B7C00091E60260916E1F0031A1F4862F0C
:104BC00090E026E239E07C01E29EC001E39E900D78
:104BD000F29E900D1124875A934F61E041E027E047
:104BE0000FEE13E020C010E084E890E09C01029FEB
:104BF000C001039F900D129F900D1124462F50E08D
:104C000026E239E0B901469F9001479F300D569F3B
:104C1000300D1124820F931F0C58104E8B569B4F52
:104C200061E041E027E00E94390F80912B0282FD74
:104C300007C080917C0290917D02029709F070C0BC
:104C40004091E60260916E1F4031A1F4262F30E0C2
:104C500086E299E0289FF001299FF00D389FF00D22
:104C60001124E850FC4FEF59F74F8081E156F8408E
:104C700083831FC0262F30E086E299E0289FD00171
:104C8000299FB00D389FB00D1124242F30E084E807
:104C900090E0289FF001299FF00D389FF00D11241E
:104CA000EA0FFB1FEB56FB4F8081A850BC4F1396B9
:104CB0008C9320E030E004E810E066E279E0FF2425
:104CC000F39480916E1F90E0209FF001219FF00DE2
:104CD000309FF00D1124DC01A69FC001A79F900D0D
:104CE000B69F900D1124E80FF91FEB56FB4FDC0126
:104CF000A850BC4FAD014D5F5F4F13968C91139739
:104D00008083F901EC58F04EF0822F5F3F4F203145
:104D10003105B9F6FD01EF59F74FDA018C91808327
:104D20008091702A882309F4C1C00091E602609145
:104D30006E1F0031A1F4862F90E026E239E0FC01DD
:104D4000E29FC001E39F900DF29F900D1124865ABF
:104D5000934F61E040E023E00FEE13E020C010E04D
:104D600084E890E07C010E9DC0010F9D900D1E9D7A
:104D7000900D1124462F50E026E239E0B901469FFC
:104D80009001479F300D569F300D1124820F931FC5
:104D90000C58104E8C569B4F61E040E023E00E947F
:104DA000390F80912B0282FD07C080917C02909187
:104DB0007D02029709F07AC02091E60260916E1F91
:104DC000203171F4462F50E086E299E0489FF001CF
:104DD000499FF00D589FF00D1124E65AF34F1AC069
:104DE000462F50E030E084E890E0289FF001299FB2
:104DF000F00D389FF00D112486E299E0DC014A9F06
:104E0000C0014B9F900D5A9F900D1124E80FF91F80
:104E1000EC56FB4F208183E994E0489FF001499FC5
:104E2000F00D589FF00D1124EE0FFF1FE650FC4FC0
:104E3000208320E030E094E8E92EF12C06E219E02E
:104E400063E974E0DD24D39480916E1F90E02E9D81
:104E5000F0012F9DF00D3E9DF00D1124809FA001CB
:104E6000819F500D909F500D1124E40FF51FEC56BB
:104E7000FB4F869FD001879FB00D969FB00D1124E8
:104E8000AA0FBB1FA650BC4F8C918083F901EC5830
:104E9000F04ED0822F5F3F4F20313105A9F6FA0145
:104EA000E65AF34F8C918083D092EF0380917C027D
:104EB00090917D028630910509F4CDC4873091052B
:104EC00084F482309105F9F0833091052CF4019738
:104ED00011F00C9429337AC3059714F00C942933FC
:104EE000CAC08830910509F4EBC3883091050CF4F1
:104EF000C9C58930910509F48CC70C9711F00C9441
:104F000029330C9413338091310282FF6AC080915F
:104F10006E1F90E076E2E72E79E0F72E8E9DF0018D
:104F20008F9DF00D9E9DF00D1124E850FC4FD08018
:104F3000CF0161E040E02FE301E71FE10E94390F5C
:104F400080916E1F90E08E9DF0018F9DF00D9E9DD3
:104F5000F00D1124E850FC4F80818D1591F120E077
:104F600030E064E870E046E259E011E080916E1FA5
:104F700090E0269FF001279FF00D369FF00D112441
:104F80007C01E49EC001E59E900DF49E900D1124DD
:104F9000E80FF91FEE56FB4FDC01A850BC4F8C9177
:104FA0008083F901EC58F04E10832F5F3F4F203182
:104FB0003105E1F6FD01E05AF74F8C9180831093A3
:104FC000EF038091E602082F10E00957104ED80138
:104FD000FC908F2D90E061E070E00E94DD0E0C945B
:104FE000F52F809176029091770261E00E94BF0FC9
:104FF00090937702809376028F31910530F48EE1A1
:1050000090E090937702809376028091760290915F
:1050100077028A3F910530F08AEF90E09093770213
:105020008093760220917602309177028091132B43
:105030009091142B2817390749F03093142B2093A3
:10504000132B0E94602581E08093990180917E025C
:10505000837011F00C94293380913E2A882319F033
:1050600080E00E940C1480913F2A882311F40C9454
:10507000293381E04FC480916B2A813099F08130CF
:1050800040F0823009F4A2C0833011F00C9429332F
:1050900038C280913F0283FF97C780912D0282FD25
:1050A00093C77BC70091E60260916E1F0031A1F4A7
:1050B000862F90E026E239E07C01E29EC001E39E6B
:1050C000900DF29E900D1124885A934F61E040E0BC
:1050D0002FE30FEE13E020C010E084E890E09C0185
:1050E000029FC001039F900D129F900D1124462F27
:1050F00050E026E239E0B901469F9001479F300D0C
:10510000569F300D1124820F931F0C58104E8E564F
:105110009B4F61E040E02FE30E94390F80916E1FAA
:1051200090E026E239E0829FF001839FF00D929F8C
:10513000F00D1124E850FC4F108220E030E064E8CC
:1051400070E046E259E080916E1F90E0269FF001EA
:10515000279FF00D369FF00D1124DC01A49FC001A4
:10516000A59F900DB49F900D1124E80FF91FEE56E6
:10517000FB4FE081DC01A850BC4F8C918E1718F4D6
:10518000EC932093861F2F5F3F4F20313105D9F6D6
:1051900080916E1F90E026E239E0829FF001839FAC
:1051A000F00D929FF00D1124E850FC4FE05AF74F9C
:1051B0009081E056F8408081891710F00C942933D3
:1051C000908380E18093861F0C9429332091E6021E
:1051D00060916E1F203171F4262F30E086E299E055
:1051E000289FF001299FF00D389FF00D1124E95AF6
:1051F000F34F1AC030E0462F50E084E890E0289F3B
:10520000F001299FF00D389FF00D112486E299E0FE
:105210007C014E9DC0014F9D900D5E9D900D11240F
:10522000E80FF91FED56FB4F10811831A9F0193125
:1052300028F41C30A9F01031B1F410C0103341F043
:10524000103619F0103279F405C0109248020BC0E4
:1052500081E007C082E005C083E003C084E001C0B4
:1052600085E0809348028091480261E00E940E0F21
:10527000982F863008F095E0909348028091122B89
:10528000981711F40C9429339093122B81E080939A
:105290009901E091E602E03119F48093EF0304C034
:1052A000F0E0EC58F04E8083809148028230A9F003
:1052B000833028F4882351F0813011F509C08430FF
:1052C000A1F0843060F08530D9F415C010E601C03B
:1052D00010E3EE246FE1F62E13C010E2FACF18E1CE
:1052E00054E0E52E4BE1F42E0BC010E138E0E32E44
:1052F00027E1F22E05C01CE09AE0E92E85E1F82EA8
:105300008091E6026E2D4F2D0E9434118091E602AD
:105310008031E1F5103321F0103611F0812F01C0FA
:1053200088E150E0A6E2B9E0682F70E0482F4150D4
:105330004F71440F17C0852F90E0FC01EE0FFF1F47
:10534000E80FF91FE20FF31FE45AF34F2081822F79
:1053500086958F7190E0861797071CF0217C242B8F
:1053600020835F5F80916E1F90E08A9F90018B9FEA
:10537000300D9A9F300D1124F901E85AF34F8081C6
:105380008517C8F61092EC031092EB032091E60209
:1053900060916E1F203171F4262F30E086E299E093
:1053A000289FF001299FF00D389FF00D1124E95A34
:1053B000F34F1AC030E0462F50E084E890E0289F79
:1053C000F001299FF00D389FF00D112486E299E03D
:1053D0009C01429FC001439F900D529F900D11244C
:1053E000E80FF91FED56FB4F10838091350282FDC7
:1053F00002C00C9429334091E60260916E1F403147
:10540000A1F4262F30E086E299E0289FF001299F41
:10541000F00D389FF00D1124E850FC4FE15AF74F82
:105420008081EF55F84081831FC0262F30E086E24F
:1054300099E0289FD001299FB00D389FB00D11240D
:10544000242F30E084E890E0289FF001299FF00DA0
:10545000389FF00D1124EA0FFB1FED56FB4F8081A2
:10546000A850BC4F11968C9300E010E094E8A92E50
:10547000B12C86E2C82E89E0D82E9924939480918D
:105480006E1F90E00A9DD0010B9DB00D1A9DB00DCE
:1054900011248C9DF0018D9DF00D9C9DF00D11242B
:1054A000AE0FBF1FAD56BB4FE850FC4F81818C93B0
:1054B000802F6E2D4F2D0E943411F801EC58F04EC4
:1054C00090820F5F1F4F00311105C9F680E16E2DEC
:1054D0004F2D0E94341180916E1F90E026E239E03A
:1054E000829FF001839FF00D929FF00D1124E850F0
:1054F000FC4F8181E15AF74F80839092EF030C9427
:10550000293380913F0283FF5BC04091E602809186
:105510006E1F90E026E239E0829FF001839FF00D3C
:10552000929FF00D1124E850FC4FE40FF11D87818C
:10553000882359F140E050E063E974E020916E1F48
:1055400030E08091E60290E0FC0116E0EE0FFF1FD4
:105550001A95E1F7880F991FE80FF91F269FC001E0
:10556000279F900D369F900D1124E80FF91FE40F2F
:10557000F51FEE0FFF1FEE5EFB4F80818260808380
:105580004F5F5F4F40345105C9F680916E1F90E028
:105590004091E60226E239E0829FF001839FF00D00
:1055A000929FF00D1124E850FC4FE40FF11D90E0A4
:1055B0008781882309F491E0978381E080939901A2
:1055C00086EE92E061E040E020E156C1E0912D28B6
:1055D000F0912E28E55DF74D91858091E8029817AE
:1055E00041F081E08093692A80917C0280936A2A4D
:1055F00002C01092692A80916B2A8130A1F081301B
:1056000038F0823039F1833011F00C94293342C0E4
:105610008CE298E261E040E02FE007E21AE20E94AB
:10562000390F0C94293380913F0282FF05C08DE22F
:1056300098E26AE070E004C08DE298E261E070E018
:1056400040E050E023EF31E000E010E00E947110F4
:105650000C94293380912D2890912E288C5C974DA5
:1056600061E040E02FE708E21AE20E94390F8091E2
:105670003F0282FD02C00C942933E0912D28F09165
:105680002E28E55DF74D81858093EA0281E08093C5
:105690006F1FDFC780913F0282FF05C081E398E260
:1056A0006AE070E004C081E398E261E070E040E00D
:1056B00050E023EF31E000E010E00E94FC0FC9C78A
:1056C00080916D2A813021F0823009F0C2C76BC011
:1056D00080916B2A813059F1813038F0823009F4A1
:1056E00054C0833009F0B5C756C080917E028370E4
:1056F00061E00E940E0F582F5370533009F452E0AE
:10570000852F837040917E024C7F482B40937E0210
:10571000252F30E08091112B90E02817390709F4EC
:1057200098C75093112B446040937E022AC0809109
:1057300078029091790261E00E94BF0F9C018E3146
:10574000910518F42EE130E005C08B3F910510F073
:105750002AEF30E030937902209378028091102B69
:1057600090E02817390709F474C72093102B0E9482
:1057700060258091780290917902909377028093CE
:10578000760281E080936F0262C785E792E061E074
:1057900042E02AE005C082E792E061E040E023E0D9
:1057A0000FE612E03CCF80916B2A813049F08130C6
:1057B00020F0833009F04DC709C08EE692E002C0A8
:1057C0008DE692E061E040E021E0EACF80917A024C
:1057D00090917B020090E90202C0969587950A9409
:1057E000E2F781708983CE01019661E040E021E01B
:1057F0000FE612E00E94390F89814091E902209161
:105800007A0230917B02882391F081E090E0A0E061
:10581000B0E004C0880F991FAA1FBB1F4A95D2F79A
:10582000282B392B30937B0220937A0212C781E018
:1058300090E0A0E0B0E004C0880F991FAA1FBB1F32
:105840004A95D2F7809590958223932390937B027B
:1058500080937A02FEC680916B2A813081F081307C
:1058600030F08230A9F0833009F0F3C656C08AE5E3
:105870009AE261E040E021E000E010E0D0CE8091CB
:105880005A2A90E0845D954D61E040E024E030C00C
:1058900080913F0283FF11C080915A2AE82FF0E0E7
:1058A000E45DF54D90E08289882309F491E0928BC4
:1058B00081E080935B2A8093990180915A2A282F56
:1058C00030E0F901E45DF54D82898823A1F48091EF
:1058D0002B02F901329682FF05C0CF01845D954D00
:1058E0006AE004C0CF01845D954D61E040E02EEF99
:1058F0000BE51AE294CE813009F0ABC6C901805C99
:10590000954D61E040E025E00BE51AE20E94390F79
:1059100080915A2A0E940C149CC680912B020091FF
:105920005A2A82FF11C010E0000F111F000F111F33
:10593000005D154DD8016D917D918D919C912DEC5F
:105940003CEC4CEC5DE310C010E0000F111F000FA9
:10595000111F005D154DD8016D917D918D919C9128
:105960002AE037ED43E25CE30E94AF10F801608368
:1059700071838283938380915A2AC82EDD24F60195
:10598000EE0FFF1FEE0FFF1FE05DF54DE080F18091
:1059900002811381C801B70120E030E040E050E00F
:1059A0000E94807C88235CF40F2EF0E0EF2EF0E064
:1059B000FF2EF0E00F2FF0E01F2FF02D14C0C801D4
:1059C000B70120E030E040E85FE30E94CA7D18168E
:1059D00054F40F2EF0E0EF2EF0E0FF2EF0E80F2F42
:1059E000FFE31F2FF02DCC0CDD1CCC0CDD1C20E3C5
:1059F0003AE2C20ED31ED601ED92FD920D931C9396
:105A00001397E0915A2AF0E0EE0FFF1FEE0FFF1FF1
:105A1000E20FF31FE080F18002811381C801B7011A
:105A200020910C2B30910D2B40910E2B50910F2B70
:105A30000E94807C882369F0E0920C2BF0920D2B61
:105A400000930E2B10930F2B81E080935B2A8093A1
:105A5000990180913F0283FFFCC5E0915A2AF0E052
:105A6000EE0FFF1FEE0FFF1FE05DF54D80E090E0B1
:105A7000A0E8BFE380839183A283B38381E0809316
:105A80005B2AE5C520916E1F30E08091820290E094
:105A9000DC01AA0FBB1FA80FB91F16E2E12E19E007
:105AA000F12EF901EE9D9001EF9D300DFE9D300D20
:105AB0001124A20FB31FFD01E25AF34F8081082F7A
:105AC0000F708295877089832A5A334FF9011081AC
:105AD000A45AB34F8C9186958F7190916B2A913017
:105AE000A1F1913038F0923009F40BC1933009F0F4
:105AF000B0C570C18091F103882309F465C281307B
:105B000009F0A7C5812F61E00E940E0F482F893050
:105B100008F048E080910A2B481739F040930A2B8F
:105B200081E08093EF038093990180916E1F90E054
:105B300026E239E0829FF001839FF00D929FF00DE5
:105B40001124EA5AF34F408384C50E941011302F6C
:105B5000380F402F50E0A32FB0E0CA018A1B9B0BE7
:105B60008130910579F5612F70E0CB01880F991F85
:105B7000860F971F880F991F880F991F480F591F6D
:105B800040575C4FFA012491A80FB91FA057BC4F92
:105B9000FD018491281709F43150FA018491FB0129
:105BA000EE0FFF1FE60FF71FEE0FFF1FEE0FFF1F99
:105BB000E30FF11DE057FC4FE4918E1709F032C05E
:105BC000315030C08F5F9F4F69F5612F70E0CB017E
:105BD000880F991F860F971F880F991F880F991F8D
:105BE000480F591F40575C4FFA012491A80FB91F65
:105BF000A057BC4FFD018491281709F43F5FFA01BB
:105C00008491FB01EE0FFF1FE60FF71FEE0FFF1F42
:105C1000EE0FFF1FE30FF11DE057FC4FE4918E17CD
:105C200009F43F5F3F3F41F48981815089838F3F71
:105C300009F419823BE00AC03C3040F089818F5F53
:105C40008983873010F087E0898330E0432F3C3030
:105C500008F04BE080910B2B481739F040930B2B49
:105C600081E08093EF038093990140932103809119
:105C7000350283FF24C020E030E066E279E08091C5
:105C80006E1F90E0F901EE0FFF1FE20FF31F7C0182
:105C9000E69EC001E79E900DF69E900D1124E80F40
:105CA000F91FE25AF34F909121039F708081807F0A
:105CB000892B80832F5F3F4F2034310501F780917E
:105CC000820290E020916E1F30E0FC01EE0FFF1F7A
:105CD000E80FF91F86E299E0BC01269FC001279FCB
:105CE000900D369F900D1124E80FF91FE25AF34FE3
:105CF0004F7080818078998197709295907F842BE6
:105D00008FC48091350283FF36C00E9410118093AA
:105D100022038823C9F140E050E066E279E08091F7
:105D20006E1F90E0FA01EE0FFF1FE40FF51FDC017C
:105D3000A69FC001A79F900DB69F900D1124E80F5C
:105D4000F91FE25AF34F2081822F82958F70909134
:105D50002203890F87708295807F2F78282B2083DC
:105D60004F5F5F4F40345105D1F681E08093EF03E0
:105D70008093990109C0CE01019661E040E027E0DF
:105D80000FEE13E00E94390F80913F0283FF02C0A3
:105D900083E089838091820290E020916E1F30E041
:105DA000FC01EE0FFF1FE80FF91F86E299E07C016E
:105DB0002E9DC0012F9D900D3E9D900D1124E80F4A
:105DC000F91FE25AF34F998197709295907F8081E5
:105DD0008F7826C40E94660F2091820230E04091A5
:105DE0006E1F50E0F901EE0FFF1FE20FF31F4E9DF3
:105DF00090014F9D300D5E9D300D1124E20FF31F79
:105E0000E45AF34F8F71880F9081917C982B908387
:105E100020C41C821091E60260916E1FB091820234
:105E20001031A1F58B2F90E0262F30E0FC01EE0F12
:105E3000FF1FE80FF91F86E299E0A901489F900132
:105E4000499F300D589F300D1124E20FF31FDF01E1
:105E5000A45AB34F4C91942F929596959695937022
:105E600011968C918770880F880F892B8983295A06
:105E7000334FD9016C91E35AF34F80818695869513
:105E800086958A83842F86958F7175C04B2F50E03D
:105E900070E0812F90E0FC01A6E0EE0FFF1FAA95B5
:105EA000E1F7880F991FE80FF91F83E994E0689FD5
:105EB000D001699FB00D789FB00D1124EA0FFB1F30
:105EC000E40FF51FEE0FFF1FEE5EFB4F90819295E2
:105ED00096959695937081818770880F880F892B8E
:105EE0008983212F30E084E890E0289FF001299FEA
:105EF000F00D389FF00D112486E299E07C016E9D33
:105F0000C0016F9D900D7E9D900D1124E80FF91F2B
:105F1000ED56FB4F6081F90196E0EE0FFF1F9A9559
:105F2000E1F7220F331FE20FF31FEA0FFB1FE40F0D
:105F3000F51FEE0FFF1FEE5EFB4F80818695869565
:105F40008F708A83812F90E09C01E6E0220F331F3F
:105F5000EA95E1F7880F991F280F391FA20FB31F89
:105F6000A40FB51FAA0FBB1FAD5EBB4F8C918695CA
:105F7000869586958B8390916B2A913009F44CC05D
:105F8000913038F0923009F481C1933009F061C347
:105F900072C280913F0283FF17C090E08091731F0F
:105FA000882309F491E09093731F992351F0E091B5
:105FB000E602F0E0DF01A856B04E8C91E957F04EB2
:105FC000808381E0809399018091731F882309F079
:105FD00040C38091E602082F10E00957104ED80107
:105FE000FC908F2D61E00E940E0FF801808380915C
:105FF000E602E82FF0E0E957F04E8081843008F0A7
:1060000083E08083E091E602F0E0E957F04E808182
:10601000F81609F01BC31DC3683199F0693128F4E3
:106020006C30D9F0603119F512C0603321F0603660
:1060300011F06032E1F4CE01019661E040E02FE121
:1060400011C0CE01019661E044E02BE10BC0CE010E
:10605000019661E048E027E105C0CE01019661E0CC
:106060004AE025E18E010C5F1F4F0E94390F80919D
:106070003F0283FF06C080E1898381E08C838093A7
:1060800099018C81882309F46AC04091E6026091ED
:106090006E1FB0918202A981403159F58B2F90E09B
:1060A000262F30E0FC01EE0FFF1FE80FF91F86E2FC
:1060B00099E07C012E9DC0012F9D900D3E9D900D7D
:1060C0001124E80FF91FE45AF34F9A2F9295990F74
:1060D000990F907C80818F73892B8083A695A695DC
:1060E000A7708181887F8A2B818381E08093EF0371
:1060F00036C0262F30E0842F90E0FC0106E0EE0F42
:10610000FF1F0A95E1F7880F991FE80FF91F83E930
:1061100094E0BC01269FC001279F900D369F900DF3
:106120001124E80FF91FEB0FF11DEE0FFF1FEE5EBC
:10613000FB4F9A2F9295990F990F907C80818F73C6
:10614000892B8083A695A695A7708181887F8A2B4D
:106150008183E42FF0E0EC58F04E81E08083809161
:10616000350283FF76C280916E1F90E026E239E00F
:10617000829FF001839FF00D929FF00D1124E85053
:10618000FC4F898185838091E602803199F520E07A
:1061900030E046E259E080916E1F90E0F901EE0F89
:1061A000FF1FE20FF31F849FD001859FB00D949FC6
:1061B000B00D1124EA0FFB1FE45AF34FA850BC4F57
:1061C00015969C9115979295990F990F907C8081C7
:1061D0008F73892B808315969C91969596959770D1
:1061E0008181887F892B81832F5F3F4F2034310548
:1061F00091F6F9C040E050E0E3E9EE2EE4E0FE2E37
:1062000006E219E020916E1F30E06091E602862FD1
:1062100090E0FC0176E0EE0FFF1F7A95E1F7880F22
:10622000991FE80FF91F2E9DC0012F9D900D3E9DD7
:10623000900D1124E80FF91FE40FF51FEE0FFF1F5B
:10624000EE5EFB4F209FD001219FB00D309FB00D1F
:106250001124A850BC4F15969C9115979295990FB3
:10626000990F907C80818F73892B808315969C91E8
:106270009695969597708181887F892B81834F5F52
:106280005F4F4034510509F0BDCFEFC0CE010296FB
:1062900061E040E02FE08E010C5F1F4F0E94390F3C
:1062A00080913F0283FF05C01A8281E08C83809336
:1062B00099018C81882309F458C04091E6026091CD
:1062C0006E1FB0918202AA81403111F58B2F90E0B0
:1062D000262F30E0FC01EE0FFF1FE80FF91F86E2CA
:1062E00099E07C012E9DC0012F9D900D3E9D900D4B
:1062F0001124E80FF91FE35AF34FAA0FAA0FAA0FB0
:10630000808187708A2B808381E08093EF032DC08A
:10631000262F30E0842F90E0FC0166E0EE0FFF1F97
:106320006A95E1F7880F991FE80FF91F83E994E058
:10633000BC01269FC001279F900D369F900D112410
:10634000E80FF91FEB0FF11DEE0FFF1FEE5EFB4F85
:10635000AF70AA0FAA0F8081837C8A2B8083E42FE1
:10636000F0E0EC58F04E81E080838091350283FFAD
:1063700070C180916E1F90E026E239E0829FF001AB
:10638000839FF00D929FF00D1124E850FC4F8A81FD
:1063900084838091E602803151F520E030E046E2CE
:1063A00059E080916E1F90E0D901AA0FBB1FA20F88
:1063B000B31F849FF001859FF00D949FF00D112471
:1063C000AE0FBF1FA35AB34FE850FC4F9481990FF3
:1063D000990F990F8C918770892B8C932F5F3F4F6A
:1063E00020343105F1F681E08093EF0332C140E0C3
:1063F00050E0A3E9EA2EA4E0FA2E06E219E020918B
:106400006E1F30E06091E602862F90E0DC01F6E03E
:10641000AA0FBB1FFA95E1F7880F991FA80FB91FA4
:106420002E9DC0012F9D900D3E9D900D1124A80F13
:10643000B91FA40FB51FAA0FBB1FAE5EBB4F209F95
:10644000F001219FF00D309FF00D1124E850FC4F1A
:1064500094819F70990F990F8C91837C892B8C93D9
:106460004F5F5F4F4034510551F6E62FF0E0EC5896
:10647000F04E81E0D6C00091E602003161F50E9445
:10648000660F482F80913F0283FF06C081E0809312
:10649000EF03809399014CE08091820290E020917B
:1064A0006E1F30E0FC01EE0FFF1FE80FF91F86E2C0
:1064B00099E0DC012A9FC0012B9F900D3A9F900D1F
:1064C0001124E80FF91FE45AF34F4F71440F8081F4
:1064D000817C842BA6C0E9E5F1E02CE0808168177F
:1064E00021F0215031972223C9F7215010E00C5898
:1064F000104ECE01039661E040E00E94390F80917A
:106500003F0283FF0AC01B82E091E602F0E0EC58F4
:10651000F04E81E08083809399018091350283FF62
:1065200056C080916E1F90E026E239E0829FF00114
:10653000839FF00D929FF00D1124E850FC4F8B814A
:10654000868360E070E093E9C92E94E0D92E86E25C
:10655000E82E89E0F82E40916E1F50E01091E6027F
:106560004C9DD0014D9DB00D5C9DB00D1124812F2F
:1065700090E09C0106E0220F331F0A95E1F7880F97
:10658000991F280F391FA20FB31FA60FB71FAA0FFD
:10659000BB1FAD5EBB4F4E9DF0014F9DF00D5E9D4C
:1065A000F00D1124E850FC4F9681990F990F990F27
:1065B0008C918770892B8C936F5F7F4F603471054E
:1065C00051F6E12FF0E0EC58F04E81E080834091ED
:1065D000820280916E1F90E023E934E0829FF001F7
:1065E000839FF00D929FF00D11248091E60290E0C0
:1065F0009C0166E0220F331F6A95E1F7880F991F0F
:10660000280F391FE20FF31FE40FF11DEE0FFF1FDC
:10661000ED5EFB4F9B81990F990F990F80818770D9
:10662000892B808316C08091DE2A90E061E070E0C3
:106630000E94DD0E982F873008F096E09093DE2AB6
:106640008091152B981729F09093152B81E080935A
:1066500099010F900F900F900F90CF91DF911F91A4
:106660000F91FF90EF90DF90CF90BF90AF909F90F1
:106670000895CF92EF920F938130910509F04CC0AD
:106680006F5F7F4F09F071C080E580935C2A1092A4
:106690005D2A82E79AE260E071E00E94CF7A89E7A2
:1066A0009AE260E071E00E94CF7A80E89AE260E0CE
:1066B00071E00E94CF7A87E89AE260E071E00E9480
:1066C000CF7A8EE89AE260E071E00E94CF7A85E9A5
:1066D0009AE260E071E00E94CF7A8CE99AE260E091
:1066E00071E00E94CF7A83EA9AE260E071E00E9452
:1066F000CF7A8AEA9AE260E071E00E94CF7A81EE76
:106700009AE262E143E124E105E176E1E72E57E117
:10671000C52E0E94496F29C0892B39F56F5F7F4FC5
:1067200021F58AEA9AE20E940F7C83EA9AE20E94AB
:106730000F7C8CE99AE20E940F7C85E99AE20E9424
:106740000F7C8EE89AE20E940F7C87E89AE20E9412
:106750000F7C80E89AE20E940F7C89E79AE20E940F
:106760000F7C82E79AE20E940F7C0F91EF90CF900E
:10677000089580E090E06FEF7FEF0E943933089535
:1067800081E090E06FEF7FEF0E94393308950E941F
:106790003C73209107023091080240910902509108
:1067A0000A02621B730B840B950B66307105810521
:1067B000910508F470C00E943C73609307027093C7
:1067C00008028093090290930A0240915C2A30915A
:1067D0005D2A2091202B222381F0213051F48DB3AA
:1067E0008093222B9DB38091212B809589238DBB93
:1067F00004C08FB7F8948093222B4CBD3DBD5E9AA8
:106800001EBC00000DB407FEFDCF8EB58093FD01C8
:106810001EBC00000DB407FEFDCF8EB58093FF01B6
:106820001EBC00000DB407FEFDCF8EB580930102A3
:106830001EBC00000DB407FEFDCF8EB58093030291
:106840001EBC00000DB407FEFDCF8EB5809305027F
:106850005E98222339F08091222B213011F48DBBD8
:1068600001C08FBF93B190729093612AEDEFF1E078
:10687000A2EFB1E020818181281709F42C93329690
:10688000119682E0E730F807A9F78091622A9817FD
:1068900011F49093632A40915C2A30915D2A2091F3
:1068A000202B222381F0213051F48DB38093222BB1
:1068B0009DB38091212B809589238DBB04C08FB718
:1068C000F8948093222B4CBD3DBD5E9A1EBC000007
:1068D0000DB407FEFDCF8EB58093FE011EBC0000F7
:1068E0000DB407FEFDCF8EB5809300021EBC0000E4
:1068F0000DB407FEFDCF8EB5809302021EBC0000D2
:106900000DB407FEFDCF8EB5809304021EBC0000BF
:106910000DB407FEFDCF8EB5809306025E9822234C
:1069200039F08091222B213011F48DBB01C08FBF33
:1069300083B180728093622A0895DF92EF92FF9272
:106940000F931F93CF93DF930E94C733E090F4011E
:10695000D090F6010091F50110E0B80164707070FC
:106960008BE292E00E944B08B801687070708DE273
:1069700092E00E944B08B8016170707083E492E06D
:106980000E944B08FF24B7016270707081E492E0AE
:106990000E944B08027010708BE492E0B8010E94D4
:1069A0004B08B7016470707089E392E00E944B0855
:1069B000B701687070708BE392E00E944B08B701DA
:1069C0006078707089E492E00E944B08CD2DD0E091
:1069D000BE01617070708DE492E00E944B08BE01B0
:1069E000627070708FE492E00E944B08B701607291
:1069F000707081E392E00E944B08B7016074707080
:106A000085E492E00E944B08B7016071707083E3E7
:106A100092E00E944B0821E0E222FF2485E392E00D
:106A2000B7010E944B08BE01607270708DE392E066
:106A30000E944B08BE01607170708FE392E00E946B
:106A40004B087091F30160E08091F20190E0682BB7
:106A5000792B87E392E00E944B0820912F02D69574
:106A6000C795D695C795CE018170682F267E922F47
:106A7000982B90932F02892F86958170681729F1A2
:106A800092FD0FC0613069F4296020932F020E94AB
:106A90003C7360935102709352028093530290931F
:106AA000540280912F0282FF06C080FD04C08061E5
:106AB0008F7D80932F0280912F02982F9170990FD4
:106AC000990F8B7F892B80932F0280912F02982F13
:106AD0009170990F8D7F892B80932F0282FF18C0B0
:106AE0000E943C7320915102309152024091530216
:106AF00050915402621B730B840B950B695E7340BB
:106B00008040904028F080912F02806280932F0275
:106B100020E030E0F901EE0FFF1FE55FFD4F8081BF
:106B2000877E80832F5F3F4F2031310599F7DF91BA
:106B3000CF911F910F91FF90EF90DF900895EF920A
:106B4000FF920F931F93CF93DF938C01C8E0D0E0A7
:106B500093E9E92E94E0F92EC8010C2E02C0969517
:106B600087950A94E2F780FF53C0599AFE01EC57CB
:106B7000FD4F408120916E1F30E0FE01EE0FFF1FA0
:106B8000CE01B6E0880F991FBA95E1F7E80FF91F1B
:106B90002E9DC0012F9D900D3E9D900D1124E80F5C
:106BA000F91FE40FF11DEE0FFF1FEE5EFB4F80811A
:106BB00081FF10C080917A0290917B020C2E02C05E
:106BC000969587950A94E2F780FD02C08FE311C085
:106BD0008FE70FC080917A0290917B020C2E02C049
:106BE000969587950A94E2F780FD02C08AE001C07D
:106BF00084E10E94EB0D82B18F71FE01E757FE4FD9
:106C00009081892B82B988E290E00E94A373599801
:106C10002196CC30D10509F09FCF88E290E00E9408
:106C2000A373599AC0E0D0E073E9E72E74E0F72E21
:106C3000C8010C2E02C0969587950A94E2F780FF52
:106C400053C0149AFE01EC57FD4F408120916E1FF6
:106C500030E0FE01EE0FFF1FCE0156E0880F991FB6
:106C60005A95E1F7E80FF91F2E9DC0012F9D900D59
:106C70003E9D900D1124E80FF91FE40FF11DEE0F5A
:106C8000FF1FEE5EFB4F808181FF10C080917A0272
:106C900090917B020C2E02C0969587950A94E2F79C
:106CA00080FD02C08FE311C08FE70FC080917A0290
:106CB00090917B020C2E02C0969587950A94E2F77C
:106CC00080FD02C08AE001C084E10E94EB0D82B128
:106CD0008F71FE01EF56FE4F9081892B82B988E2B9
:106CE00090E00E94A37314982196C830D10509F052
:106CF0009FCF88E290E00E94A373149ADF91CF9116
:106D00001F910F91FF90EF9008951F93CF93DF9302
:106D100010E0C0E0D0E08DEC9DE2BE0140E00E94BA
:106D2000E87221968DEC9DE2BE0143E60E94E87276
:106D300021968DEC9DE2BE0144E60E94E872219608
:106D40008DEC9DE2BE0141E00E94E87221968DEC3F
:106D50009DE2BE0143E00E94E8722196CA30D1054F
:106D6000D1F61F5F1038A9F6DF91CF911F910895DA
:106D70002F923F924F925F926F927F928F929F924B
:106D8000AF92BF92CF92DF92EF92FF920F931F9339
:106D9000CF93DF93CCE2DAE254E0A52EB12CAC0E17
:106DA000BD1EEE24FF24C82EDD2416010894211CEC
:106DB000311C42E0442E512C4C0C5D1C33E0632E00
:106DC000712C6C0C7D1C24E0822E912C8C0C9D1C53
:106DD000B7016C0D7D1D8DEC9DE248810E94E8722B
:106DE000B1016E0D7F1D8DEC9DE24A810E94E8721B
:106DF00082010E0D1F1DF50161917191819191919B
:106E00005F0120E030E048EC52E40E94CE7D0E9419
:106E1000EC7C9B01AC018DEC9DE2B801422F0E94FD
:106E2000E872B3016E0D7F1D8DEC9DE24A890E94D0
:106E3000E872B4016E0D7F1D8DEC9DE24C890E94BD
:106E4000E872219685E090E0E80EF91E9AE2CE32D3
:106E5000D90709F0BDCFDF91CF911F910F91FF901E
:106E6000EF90DF90CF90BF90AF909F908F907F90EA
:106E70006F905F904F903F902F9008958DEC9DE222
:106E800060EA7FE040E00E94E87208958DEC9DE2A8
:106E900060EA7FE04091B52A0E94E87208954F921F
:106EA0005F926F927F928F929F92AF92BF92CF929A
:106EB000DF92EF92FF920F931F93CF93DF93CCE279
:106EC000DAE2F4E0CF2ED12CCC0EDD1E00E010E093
:106ED000E82EFF2427010894411C511CE2E06E2E8D
:106EE000712C6E0C7F1C73E0872E912C8E0C9F1CD6
:106EF00064E0A62EB12CAE0CBF1CB8016E0D7F1D38
:106F00008DEC9DE20E94E172853008F084E0888378
:106F1000B201600F711F8DEC9DE20E94E1728F3F04
:106F200009F48EEF8A83B301600F711F8DEC9DE22F
:106F30000E94E172853608F084E6682F70E08827A9
:106F400077FD8095982F0E941A7D20E030E048EC74
:106F500052E40E94847CF601608371838283938370
:106F6000B401600F711F8DEC9DE20E94E1728111EE
:106F700081E08A8BB501600F711F8DEC9DE20E944C
:106F8000E172863008F085E08C8B1C861E86188A9C
:106F90000B5F1F4F219684E090E0C80ED91E0A3087
:106FA000110509F0AACFDF91CF911F910F91FF90AA
:106FB000EF90DF90CF90BF90AF909F908F907F9099
:106FC0006F905F904F90089510925A2A1092422A23
:106FD00080E00E944F3708958DEC9DE260EA7FE0EB
:106FE0000E94E1728093B52A823020F01092B52A77
:106FF0000E9446370895AF92BF92CF92DF92EF92F0
:10700000FF920F931F939091382A9F5F9093382A95
:107010008091392A8F5F8093392A8091422A882370
:1070200049F080E098E00E94290E80E098E00E94FC
:107030005E0E2FC1892F90E040912E2A20E031E092
:10704000241B3109821793070CF48BC01092382A45
:1070500080912C2A8430D9F580913A2A882309F02E
:1070600075C060E070E080E090E020E031E040E05A
:1070700050E00E945C79E090302AF090312A009133
:10708000322A1091332A0E941A7DA80197010E948A
:10709000CE7D5B016C01C801B70120E030E040E02B
:1070A00053EC0E94CE7D20E030E040E053E40E94AB
:1070B0001C7C9B01AC01C601B5010E941C7C0E9496
:1070C000EC7CB4E0660F771FBA95E1F73BC0F82F70
:1070D000E0E080913A2AE80FF11DEC5EFB4FE4916D
:1070E000E090302AF090312A0091322A1091332A10
:1070F0006E2F70E0882777FD8095982F0E941A7D6B
:10710000A80197010E94CE7D5B016C01C801B70107
:1071100020E030E040E053EC0E94CE7D20E030E003
:1071200040E053E40E941C7C9B01AC01C601B50108
:107130000E941C7C20E030E040E851E40E94CE7DBB
:107140000E94EC7C7093FB2A6093FA2A8091FA2AC1
:107150009091FB2A0E94290E80913A2A8F5F80939A
:107160003A2A8091392A90E040912F2A20E031E09C
:10717000241B3109821793070CF48BC01092392A13
:1071800080912D2A8430D9F580913B2A882309F0FB
:1071900075C060E070E080E090E020E031E040E029
:1071A00050E00E945C79E090342AF090352A0091FA
:1071B000362A1091372A0E941A7DA80197010E9451
:1071C000CE7D5B016C01C801B70120E030E040E0FA
:1071D00053EC0E94CE7D20E030E040E053E40E947A
:1071E0001C7C9B01AC01C601B5010E941C7C0E9465
:1071F000EC7CA4E0660F771FAA95E1F73BC0F82F5F
:10720000E0E080913B2AE80FF11DEC5EFB4FE4913A
:10721000E090342AF090352A0091362A1091372ACE
:107220006E2F70E0882777FD8095982F0E941A7D39
:10723000A80197010E94CE7D5B016C01C801B701D6
:1072400020E030E040E053EC0E94CE7D20E030E0D2
:1072500040E053E40E941C7C9B01AC01C601B501D7
:107260000E941C7C20E030E040E851E40E94CE7D8A
:107270000E94EC7C7093F92A6093F82A8091F82A96
:107280009091F92A0E945E0E80913B2A8F5F809335
:107290003B2A80918002882329F19091810280917C
:1072A0007E028370813041F4E0917502F0E0ED5E82
:1072B000F74FE491E69506C0E0917502F0E0ED5ECF
:1072C000F74FE491F0E09F5F909381029150892FF6
:1072D00090E08E179F0734F00E94840D1092810277
:1072E0001092800280916A028F5F80936A021F91E0
:1072F0000F91FF90EF90DF90CF90BF90AF900895E7
:107300001F920F920FB60F920BB60F9211242F936C
:107310003F934F935F936F937F938F939F93AF931D
:10732000BF93EF93FF930E94FB37FF91EF91BF91C3
:10733000AF919F918F917F916F915F914F913F910D
:107340002F910F900BBE0F900FBE0F901F901895AE
:107350002F923F924F925F926F927F928F929F9265
:10736000AF92BF92CF92DF92EF92FF920F931F9353
:10737000DF93CF9300D000D000D0CDB7DEB780919F
:107380001F038823B1F08091EE03882391F42091AC
:10739000E9033091EA038091EB039091EC038217AB
:1073A000930738F45F9810921F031092EA0310922B
:1073B000E9038091610290E0882309F491E09093C1
:1073C00061028091830260E30E94507E943041F418
:1073D0008091390190E0882309F491E0909339017C
:1073E000809183026CE00E94507E943051F4E091D1
:1073F000E602F0E0E65CFE4F10821092640210920A
:1074000063028091E002882309F496C7EAE3FAE276
:107410003CE32FEF8481882309F449C086818230C0
:10742000F1F0833030F4882359F0813009F03FC007
:1074300032C0843081F1843050F18530C1F52FC0E5
:107440008091DF02813099F58091830260E60E948D
:10745000507E992361F58081893C48F127C0809155
:10746000DF02882309F0B1C78091830260E60E94A1
:10747000507E992309F0A9C7208319C08091830207
:1074800060E60E94507E992391F4308310C0809171
:10749000830260E307C08091830260E603C08091AD
:1074A000830268E10E94507E992309F4108231968C
:1074B0004AE2EC33F40709F0ADCF80917E0283708D
:1074C000823028F580917202813059F0813028F0A5
:1074D000823059F08330D9F40CC08091830260E689
:1074E0000BC08091830260E307C08091830268E152
:1074F00003C0809183026CE00E94507E992339F48E
:1075000080917F02882309F491E090937F0210928A
:10751000DA021092D9021092F00366EB7AE27A83D3
:10752000698388E99FE19C838B830BEE802E02E0C8
:10753000902E1CEFA12E12E0B12E1B0100E010E0F6
:10754000B1E04B2E512C612C712CD02E20916E1F4E
:1075500090E1091791F4822F90E0A6E2B9E08A9FAA
:10756000F0018B9FF00D9A9FF00D1124E850FC4F15
:10757000E15AF74FC190F0801DC0822F90E024E8BF
:1075800030E0029FF001039FF00D129FF00D1124D7
:10759000AC0166E279E0469FC001479F900D569F7F
:1075A000900D1124E80FF91FE850FC4FE556FF4FEE
:1075B000C080F2903296E080809183029C2D969557
:1075C000292F30E090E06C2D70E00E945C7E8217E5
:1075D000930729F4F801E853FD4F71E0708380911F
:1075E000830290E06C2D70E00E945C7E821793070E
:1075F00009F060C0F801E954FD4F80818F5F8083FE
:107600008081F81608F4108281E0E81679F0E81617
:1076100040F092E0E916B1F0A3E0EA1609F04AC0A2
:1076200037C0F801E954FD4F808107C0F801E954E3
:10763000FD4F8081BF2DB81B8B2FF801EA55FD4F00
:10764000808338C0F801EA55FD4F80818F1509F01D
:10765000C2C6F5018081813009F0BDC6108206C026
:10766000D5018C91882311F4E1E0EC93D5018C9144
:10767000F801E954FD4FD801AA55BD4F882311F0F8
:10768000808104C08081EF2DE81B8E2F8C9312C067
:107690002F2D30E02F5F3F4F442737FD4095542F6B
:1076A00060E070E080E090E00E945C79F801EA55CB
:1076B000FD4F608320916E1F4F2D50E0F0E1DF16EB
:1076C00091F530E08091940290E0841795071CF0CA
:1076D00080E090E004C08091940290E00196FC016B
:1076E000EE0FFF1FE80FF91F46E259E0249FD0017B
:1076F000259FB00D349FB00D1124EA0FFB1FE45AF3
:10770000F34F9081929596959695937081818770AD
:10771000880F880F892B482F50E040515040A75ABE
:10772000B34FAC9152C030E0F801EC57FD4F80816F
:1077300090E0841795071CF040E050E005C0808180
:10774000482F50E04F5F5F4FF801EE0FFF1FC80159
:1077500066E0880F991F6A95E1F7E80FF91F63E962
:1077600074E0269FC001279F900D369F900D112435
:10777000E80FF91FE40FF51FEE0FFF1FEE5EFB4F42
:107780009081929596959695937081818770880FD8
:10779000880F892B482F50E04051504084E890E0FA
:1077A000089FF001099FF00D189FF00D1124A6E22B
:1077B000B9E02A9FC0012B9F900D3A9F900D112494
:1077C000E80FF91FEB56FB4FA081A15020918302D7
:1077D000F801E25FFC4FFE83ED838081EA2FF0E049
:1077E000EE0FFF1FE80FF11DEE0FFF1FE55AFE4FD2
:1077F00080819181820F911D841B950B6C2D70E00F
:107800000E94707E892B09F02CC2F801E853FD4FCD
:107810008081882309F425C21082AD81BE818C91BC
:1078200090E0882309F491E0F801E25FFC4F908337
:10783000F801E65CFE4FB1E0B083EB1691F0EB1679
:1078400040F0E2E0EE16B1F0F3E0EF1609F049C0C7
:1078500036C0F801EB56FD4F8081F801EC57FD4F23
:1078600028C0F801EB56FD4F8081F81AF801EC575B
:10787000FD4F23C0F801EC57FD4F80818F1508F4B0
:10788000B2C5D4018C91813009F0ADC51C9206C0FF
:10789000F4018081882311F421E02083D4018C91AC
:1078A000F801EC57FD4FD801AB56BD4F882319F0B6
:1078B0008C91808316C08C91F81AF08212C02F2D03
:1078C00030E02F5F3F4F442737FD4095542F60E055
:1078D00070E080E090E00E945C79F801EC57FD4F89
:1078E000608320916E1FF801EC57FD4FB0E1DB166D
:1078F000D1F4808190E030E0FC01EE0FFF1FE80F33
:10790000F91F46E259E0249FC001259F900D349F46
:10791000900D1124E80FF91FE35AF34F608166952B
:107920006695669522C0408130E0F801EE0FFF1F9A
:10793000C80166E0880F991F6A95E1F7E80FF91F03
:1079400063E974E0269FC001279F900D369F900D3C
:107950001124E80FF91FE40FF11DEE0FFF1FEE5E7B
:10796000FB4F6081669566956F70F801EC57FD4F8F
:10797000808182958F70AB81BC819C918917A9F021
:10798000908192959F709C938091731F882321F022
:10799000F801E957F04E908380917C0290917D022E
:1079A000039719F4B1E0B093990120916E1FE0E1C3
:1079B000DE16D9F48091940290E030E0FC01EE0FE5
:1079C000FF1FE80FF91F46E259E0249FC001259FE1
:1079D000900D349F900D1124E80FF91FE45AF34FD6
:1079E000808181708093F00336C0F801EC57FD4F21
:1079F000408130E0F801EE0FFF1FC801B6E0880FAC
:107A0000991FBA95E1F7E80FF91FA3E9B4E02A9F9F
:107A1000C0012B9F900D3A9F900D1124E80FF91F84
:107A2000E40FF11DEE0FFF1FEE5EFB4F808180FF24
:107A300012C02091D9023091DA0281E090E0002E4C
:107A400002C0880F991F0A94E2F7822B932B909320
:107A5000DA028093D902F801EB56FD4F80818F5FE7
:107A600080836B3008F4AAC0B0E1DB16B9F0209136
:107A7000D9023091DA02D301C201002E04C0880F6E
:107A8000991FAA1FBB1F0A94D2F780959095822355
:107A900093239093DA028093D90202C01092F003EC
:107AA0006D3091F16E3030F46B3059F06C3009F07C
:107AB000D0C010C06E3009F440C06F3009F0C9C0AA
:107AC00055C060E070E080E090E029E030E040E008
:107AD00050E054C060E070E080E090E027E030E0EB
:107AE00040E050E00E945C799B01AC01613071057F
:107AF0008105910509F0ADC060E1D61609F04BC0D3
:107B000071E07093F003A5C060E070E080E090E069
:107B100024E030E040E050E00E945C799B01AC0141
:107B2000613071058105910509F093C080E1D81697
:107B300091F591E09093F0038CC060E070E080E0FC
:107B400090E023E030E040E050E00E945C799B014F
:107B5000AC01613071058105910509F07AC0A0E1A1
:107B6000DA16C9F4B1E0B093F00373C060E070E0DE
:107B700080E090E022E030E040E050E00E945C795C
:107B80009B01AC01613071058105910509F061C06F
:107B9000E0E1DE1679F08091D9029091DA02002EB0
:107BA00004C0220F331F441F551F0A94D2F7822BA3
:107BB000932B48C0F1E0F093F0034BC0862F815027
:107BC000873058F470E06F5F7F4FD1018C9190E067
:107BD0000E94707E892BE9F113C0683041F4F101F5
:107BE000808163E00E94507E992399F516C0693028
:107BF00059F4D1018C9190E083709070892B49F5F4
:107C0000B0E1DB1669F423C06A3019F5F101808117
:107C100090E087709070892BE1F4F0E1DF16B9F005
:107C20002091D9023091DA02D301C201002E04C0A2
:107C3000880F991FAA1FBB1F0A94D2F780959095B1
:107C4000822393239093DA028093D90202C0109288
:107C5000F0038091D9029091DA029093DC02809334
:107C6000DB0220E1D21609F477C020916E1F30E0CC
:107C7000F4E8EF2EF2E0FF2EE00EF11ED7019C910A
:107C800080918302E3E9F4E02E9F60012F9FD00CE6
:107C90003E9FD00C11249801220F331FA80176E0DB
:107CA000440F551F7A95E1F7240F351FC20ED31EDE
:107CB000F601E90FF11DEE0FFF1FED5EFB4FE081B6
:107CC000E695E695E695F0E0E35BFE4FE08190E017
:107CD0006E2F70E00E945C7E892BF1F5EE23E1F1BE
:107CE0008091DB029091DC02002E02C09695879570
:107CF0000A94E2F780FF30C0D7018C91C80ED11CE6
:107D0000CC0CDD1CE2E1F4E0CE0EDF1ED6018C913E
:107D100080FF22C04091D9025091DA022091D9020D
:107D20003091DA02D301C201002E04C0880F991FDE
:107D3000AA1FBB1F0A94D2F7282B392B3093DA02E3
:107D40002093D9028091D9029091DA02842B952B4D
:107D50009093DA028093D9020F5F1F4F0894211C81
:107D6000311CEB81FC813196FC83EB830894811CF0
:107D7000911C0894A11CB11C0131110509F0E5CB3F
:107D800080917E028370823038F480917F02882354
:107D900011F02C9A01C02C988091F003882309F4EB
:107DA0008EC180912803882309F089C18091EE0358
:107DB000882309F084C180916E1FE82EFF24209152
:107DC00094026091940286E299E0E89E8001E99E27
:107DD000100DF89E100D1124D801A850BC4FA25AC6
:107DE000B74F8C91C82EDD2430E0F901EE0FFF1F54
:107DF000E20FF31FE00FF11FE25AF34F80818F7003
:107E0000F601EE0FFF1FEC0DFD1DEE0FFF1FEE0F35
:107E1000FF1FE80FF11DE057FC4FE491E150F0E047
:107E2000EE0FFF1FE450FC4F4591549170E0FB01B1
:107E3000EE0FFF1FE60FF71FE00FF11FE25AF34F9F
:107E40002081269526952695922F9E7080E0480FDA
:107E5000591F5093F3034093F203809194021296BA
:107E60002C9130E090E0821793071CF080E090E0C6
:107E700004C08091940290E00196FC01EE0FFF1F78
:107E8000E80FF91F86E299E0AC01E49EC001E59E8F
:107E9000900DF49E900D1124E80FF91FE25AF34F54
:107EA00040814F708091940290E0821793071CF0FC
:107EB00020E030E006C080919402282F30E02F5F50
:107EC0003F4FF601EE0FFF1FEC0DFD1DEE0FFF1FE4
:107ED000EE0FFF1FE40FF11DE057FC4FE491E1505E
:107EE000F0E0EE0FFF1FE450FC4F85919491F901F3
:107EF000EE0FFF1FE20FF31F06E219E0E09ED00134
:107F0000E19EB00DF09EB00D1124EA0FFB1FE25A66
:107F1000F34F4081469546954695342F3E7020E0BC
:107F2000820F931F9093F5038093F4032091F20343
:107F30003091F303A95AB34F6C91821B930B70E0FD
:107F40000E94707E7093F7036093F603C9010E944C
:107F5000B60D5F9A81E080931F039091ED038091AD
:107F60006E1F682F70E0609FF001619FF00D709FA1
:107F7000F00D1124E85AF34F8081981711F450E066
:107F800002C0592F5F5F8091940290E0FC01EE0FD8
:107F9000FF1FE80FF91F86E299E0689FD001699FF3
:107FA000B00D789FB00D1124EA0FFB1FE45AF34F78
:107FB000408146954F71A95AB34FAC912091EB0384
:107FC0003091EC038A2F90E02817390708F413C288
:107FD00080919402851709F00EC2A03671F42091A9
:107FE000EB033091EC03842F90E00196880F991FEA
:107FF000880F991F820F931F22C0242F30E0A033D7
:1080000059F48091EB039091EC032F5F3F4F220FC7
:10801000331F280F391F20C08091EB039091EC0390
:108020000196820F931F9093EC038093EB031FC084
:10803000842F90E00196880F991F880F991F9093C5
:10804000EC038093EB03DEC1242F30E0A03349F42E
:108050002F5F3F4F220F331F3093EC032093EB032E
:10806000D1C12F5F3F4F3093EC032093EB03842F5C
:1080700090E001962A2F30E08217930721F4809137
:1080800094028093ED038091940290E0FC01EE0F46
:10809000FF1FE80FF91F86E299E0DC016A9FC0012B
:1080A0006B9F900D7A9F900D1124E80FF91FE45AF1
:1080B000F34F4F71440F8081817C842B80838091AA
:1080C000940290E020916E1F30E0FC01EE0FFF1F44
:1080D000E80FF91F86E299E0AC01249FC001259FBB
:1080E000900D349F900D1124E80FF91FE25AF34FC1
:1080F000808187FF10C08091F6039091F703209153
:10810000F2033091F303820F931F9093F303809354
:10811000F2030E94B60D2091DF2A3091E02A21154A
:108120003105C1F080918302E091DE2AF0E0E7554D
:10813000FE4F608190E070E00E945C7E892B51F4DC
:108140008091D9029091DA02822B932B9093DA02DC
:108150008093D9028091D9029091DA02892B61F142
:108160008091D9029091DA02909364028093630225
:108170008091D9029091DA020E949F3580916D0220
:10818000882349F08091D9029091DA029F779093E9
:10819000DA028093D9022091D9023091DA028091DB
:1081A000292890912A2880959095822393230E94D4
:1081B0004C0D81E080938002E091861FF0E0EB5649
:1081C000FD4F808190E090934C0180934B01709122
:1081D0006E1F472F50E086E299E0489FF001499FCB
:1081E000F00D589FF00D1124EE56FB4F20E030E0CB
:1081F00061E0D901AB56BD4F9C918081891750F445
:108200001C92A981BA818C918F5F8C938150833DA0
:1082100008F06C932F5F3F4FEC57FF4F89819A8195
:1082200001969A8389832031310519F72091A5029F
:1082300086E299E0489FF001499FF00D589FF00DAC
:108240001124E85AF34F8081821768F41092A50236
:108250008091C62A8F5F8093C62A8150833D18F093
:1082600081E08093C62A20914B0130914C0186E237
:1082700099E0489FF001499FF00D589FF00D11249F
:10828000E850FC4F808190E08217930794F510929C
:10829000192B10924C0110924B018091701F882372
:1082A00041F180917C0290917D028230910541F0F4
:1082B0008530910529F08130910511F0892BC9F4A1
:1082C0001092701F10926E1F772319F481E0809333
:1082D0006E1F0E94842480E090E0FC01EB56FD4F6D
:1082E0001082FC01E25FFC4F108201968131910502
:1082F000A1F740914B0150914C0180916E1F90E08D
:1083000026E239E0829FF001839FF00D929FF00DED
:108310001124E850FC4F808190E0019748175907DD
:1083200009F06DC08091192B882309F068C081E0A5
:1083300080930D038093192B8091E002882309F527
:108340002091DF2A3091E02A21153105D1F080916A
:108350008302E091DE2AF0E0E755FE4F608190E075
:1083600070E00E945C7E892B61F4C9010E949F35F8
:108370008091DF2A9091E02A0E944C0D81E0809349
:108380008002809183028F5F8093830281508036C8
:1083900070F081E0809383028091DF02823010F0E0
:1083A0001092DF028091DF028F5F8093DF02809165
:1083B0001F03882359F18091E9039091EA03019604
:1083C0009093EA038093E90321C08091DF0281301A
:1083D00009F06DC853C8F801EA55FD4F8081882324
:1083E00009F044C93DC9F801EC57FD4F808188234D
:1083F00009F054CA4DCAA03609F026CE19CE109203
:108400000D039ACF473109F032CE39CE26960FB6FA
:10841000F894DEBF0FBECDBFCF91DF911F910F91BA
:10842000FF90EF90DF90CF90BF90AF909F908F9094
:108430007F906F905F904F903F902F900895FF92A4
:108440000F931F93F82E01EE1AE2C8016F2D41E041
:108450000E94266EC8016EE178E00E94DC77C801B8
:108460006F2D41E00E94266E1F910F91FF9008959D
:108470000F931F9301EE1AE2C80164E040E00E94EE
:10848000266EC8016CE778E00E94DC7781E080937B
:10849000682A1F910F91089581EE9AE269E878E0C9
:1084A0000E94DC7708950F931F9301EE1AE2C80132
:1084B00060E040E00E94266EC80164E378E00E941C
:1084C000DC77C80160E041E00E94266E0E944C42C9
:1084D000C80160E041E00E94266EC80163E278E0D6
:1084E0000E94DC771F910F9108950F931F9301EE67
:1084F0001AE2C80160E040E00E94266EC80166E50D
:1085000078E00E94DC77C80160E041E00E94266EBE
:108510000E944C42C80160E041E00E94266EC80102
:1085200065E478E00E94DC771F910F9108950F9326
:108530001F93CF93DF93C0E0D0E0082F10E006C078
:1085400081EE9AE261EA0E94FF772196C017D10777
:10855000BCF3DF91CF911F910F91089588E00E94A5
:108560001F42E0915A2AF0E0E45DF54D84898230A3
:1085700019F1833038F4882309F440C0813009F0C0
:1085800047C031C0843031F0843020F1853009F0AB
:108590003FC009C081EE9AE260E00E941C6E81EE4D
:1085A0009AE261E011C081EE9AE260E00E941C6EE6
:1085B00081EE9AE261E01FC081EE9AE260E00E94E3
:1085C0001C6E81EE9AE263E00E941C6E81EE9AE2DC
:1085D00062E011C081EE9AE260E00E941C6E81EEC2
:1085E0009AE263E008C081EE9AE260E00E941C6EAD
:1085F00081EE9AE266E00E941C6E089581EE9AE296
:1086000060E00E941C6E81EE9AE267E00E941C6EA0
:1086100008951F93882319F08FEF8093FC2A2091EF
:10862000E60240916E1F203171F4242F30E086E283
:1086300099E0289FF001299FF00D389FF00D11243B
:10864000E95AF34F19C030E050E084E890E0289FE9
:10865000F001299FF00D389FF00D112486E299E07A
:108660009C01429FC001439F900D529F900D112489
:10867000E80FF91FED56FB4F10818091FC2A181767
:1086800009F452C088E00E941F42183109F11931E3
:1086900030F41C3059F0103109F044C010C01033D0
:1086A00071F11036A9F11032E9F51BC081EE9AE2A2
:1086B00060E00E941C6E81EE9AE264E031C081EEBF
:1086C0009AE260E00E941C6E81EE9AE261E011C0C5
:1086D00081EE9AE260E00E941C6E81EE9AE261E017
:1086E0001FC081EE9AE260E00E941C6E81EE9AE269
:1086F00063E00E941C6E81EE9AE262E011C081EE9E
:108700009AE260E00E941C6E81EE9AE263E008C08B
:1087100081EE9AE260E00E941C6E81EE9AE266E0D1
:108720000E941C6E1093FC2A1F910895CF92DF9235
:10873000EF92FF920F931F93CF93DF93EC018B0186
:108740007A01690162E77AE20E94E979882321F5DA
:1087500081EE9AE260E041E00E94266E81EE9AE2AC
:1087600069EA78E00E94DC778C819D81029720F491
:1087700081EE9AE261E003C081EE9AE260E041E0BE
:108780000E94266E81EE9AE2BE010E94077982E77E
:108790009AE2BE010E94E27BC80169E77AE20E9488
:1087A000E9798823E1F481EE9AE264E041E00E94F5
:1087B000266E81EE9AE264EA78E00E94DC7781EE30
:1087C0009AE264E041E00E94266E81EE9AE2B801EE
:1087D0000E94077989E79AE2B8010E94E27BC7010B
:1087E00060E87AE20E94E979882361F5C70160E0D8
:1087F00070E00E949379882329F581EE9AE268E07F
:1088000041E00E94266E81EE9AE26FE978E00E94D4
:10881000DC77F70184819581029720F481EE9AE25A
:1088200069E003C081EE9AE268E041E00E94266EB2
:1088300081EE9AE2B7010E94077980E89AE2B701D7
:108840000E94E27BC60167E87AE20E94E979882308
:1088500029F581EE9AE26CE041E00E94266E81EEFD
:108860009AE26AE978E00E94DC77F60184819581DA
:10887000029720F481EE9AE26DE003C081EE9AE265
:108880006CE041E00E94266E81EE9AE2B6010E9401
:10889000077987E89AE2B6010E94E27BDF91CF91E7
:1088A0001F910F91FF90EF90DF90CF9008959F92CE
:1088B000AF92BF92CF92DF92EF92FF920F931F93EE
:1088C000DF93CF93CDB7DEB7C555D2400FB6F8943E
:1088D000DEBF0FBECDBF8091692A8823A1F081EE53
:1088E0009AE260916C2A41E00E94266E80913901E3
:1088F0008823F1F481EE9AE263E071E00E9404794A
:108900001092FF2A1EC08091FF2A8823D1F4809103
:108910006A2A90E020917C0230917D0282179307B1
:1089200081F481EE9AE260916C2A41E00E94266E09
:1089300081EE9AE26AEA7AE20E94077981E0809306
:10894000FF2A80916A2A90E020917C0230917D027A
:108950008217930711F01092692A80919901882358
:1089600011F40C947054109299018091712A88230B
:1089700009F471C081EE9AE260E040E00E94266E48
:1089800081EE9AE263EE79E00E94DC7781EE9AE272
:1089900060E041E00E94266E0E944C4281EE9AE225
:1089A00062E041E00E94266E81EE9AE261EE79E09B
:1089B0000E94DC7781EE9AE265E041E00E94266E3B
:1089C00087E00E94974281EE9AE26EE041E00E94C9
:1089D000266E81EE9AE26FED79E00E94DC772091BD
:1089E000E60240916E1F203171F4242F30E086E2C0
:1089F00099E0289FF001299FF00D389FF00D112478
:108A0000E75AF34F19C030E050E084E890E0289F27
:108A1000F001299FF00D389FF00D112486E299E0B6
:108A20009C01429FC001439F900D529F900D1124C5
:108A3000E80FF91FEB56FB4F60816C5F81EE9AE205
:108A400041E00E94266E81EE9AE26BED0E94FF7774
:108A50008BE090E078C08091702A882309F479C077
:108A600081EE9AE260E040E00E94266E80917C02F6
:108A700090917D02029729F481EE9AE26EEC79E002
:108A800004C081EE9AE26DEB79E00E94DC7781EE22
:108A90009AE260E041E00E94266E0E944C4281EE24
:108AA0009AE263E041E00E94266E2091E602409146
:108AB0006E1FDE01AD5BBD4F2031B9F4242F30E0D5
:108AC00086E299E0289FF001299FF00D389FF00D74
:108AD0001124E65AF34F8081E82FF0E0EE0FFF1FDC
:108AE000EC51FD4F6591749122C030E050E084E874
:108AF00090E0289FF001299FF00D389FF00D112480
:108B000086E299E09C01429FC001439F900D529FD5
:108B1000900D1124E80FF91FEC56FB4F8081E82FD0
:108B2000F0E0EE0FFF1FEC51FD4F65917491CD0108
:108B30000E94E40781EE9AE2BE016D5B7D4F0E94C8
:108B400004798AE090E09093E4028093E3020C942D
:108B5000705480917C0290917D028530910511F4D2
:108B60000C9436528630910594F48230910509F4C4
:108B700005C2833091050CF010C3009711F40C94DA
:108B8000A453019711F00C9470540C9479528830CE
:108B90009105B9F08930910554F48630910511F4AE
:108BA0000C94C04D079711F00C947054ACC58930EB
:108BB000910511F40C94024F0C9711F00C94705421
:108BC00010C58091E3029091E4020897A9F087E82C
:108BD0009AE268E071E00E94037BBC0180E89AE2BF
:108BE0000E94E27BBC0189E79AE20E94E27BBC0121
:108BF00082E79AE20E94E27B80916D2A813029F01F
:108C0000823011F00C947054BBC08091E3029091BB
:108C1000E402089761F480915A01813041F4809117
:108C20009A01882321F48091682A8823D1F188E071
:108C300090E09093E4028093E30280916D2A809308
:108C40005A0110929A011092682A81EE9AE260E02D
:108C500040E00E94266E81EE9AE26CEA79E00E9482
:108C6000DC7780916B2AE82FF0E0EE0FFF1FEC56C7
:108C7000FD4F659174918E010F5F1F4FC8010E94D7
:108C8000E407E0916B2AF0E0E556FE4F81EE9AE2B0
:108C9000608140E00E94266E81EE9AE2B8010E9457
:108CA000047980917E028370E82FF0E0EE0FFF1FC1
:108CB000E25CFC4F659174917E010894E11CF11C0B
:108CC000C7010E94E4078EE89AE2B7010E94037B85
:108CD0008E010B5F1F4F6091780270917902C8017D
:108CE0004AE00E941C7B85E99AE2B8010E94E27B7F
:108CF000C8010E940F7C8E01045F1F4FC801609164
:108D000075024AE00E947E7B8CE99AE2B8010E94DB
:108D1000E27BC8010E940F7C80917202E82FF0E094
:108D2000EE0FFF1FE05DFC4F65917491C7010E943B
:108D3000E40783EA9AE2B7010E94037B23E1A22EB3
:108D4000B12CAC0EBD1EC5016EE87AE20E94F97B23
:108D50009AE1C92ED12CCC0EDD1EC60165E97AE25E
:108D60000E94F97B81E2E82EF12CEC0EFD1EC7017A
:108D70006CE97AE20E94F97B8E01085D1F4FE5C025
:108D800080915A01823049F480919A01882329F414
:108D90008091682A882309F448C082E080935A01B0
:108DA00010929A011092682A81EE9AE260E040E007
:108DB0000E94266E81EE9AE26BE979E00E94DC77F0
:108DC00081EE9AE26EE040E00E94266E6091E90238
:108DD00070E06F5F7F4F81EE9AE24AE050E00E94C0
:108DE000F1788091E9028093012B80916B2AE82F22
:108DF000F0E0EE0FFF1FE456FD4F659174918E0178
:108E00000F5F1F4FC8010E94E407E0916B2AF0E05A
:108E1000E556FE4F81EE9AE2608140E00E94266EA8
:108E200081EE9AE2B8010E9404799091012B809121
:108E3000E902981709F181EE9AE26FE040E00E94A2
:108E4000266E81EE9AE269E979E00E94DC7781EE94
:108E50009AE26EE040E00E94266E6091E90270E0C6
:108E60006F5F7F4F81EE9AE24AE050E00E94F17816
:108E70008091E9028093012B80916E02E82FF0E04F
:108E8000EE0FFF1FEC57FC4F659174918E010F5F41
:108E90001F4FC8010E94E4078EE89AE2B8010E94C1
:108EA000037B80916D02E82FF0E0EE0FFF1FE85783
:108EB000FC4F65917491C8010E94E40785E99AE22C
:108EC000B8010E94037B8CE99AE26AE071E00E949B
:108ED000037BE0917A02F0917B020090E90202C0EC
:108EE000F695E7950A94E2F7E170F070EE0FFF1F38
:108EF000E457FC4F65917491C8010E94E40783EA2E
:108F00009AE2B8010E94037B7FE2A72EB12CAC0E3F
:108F1000BD1EC5016EE87AE20E94F97B66E3C62EAB
:108F2000D12CCC0EDD1EC60165E97AE20E94F97BE8
:108F30005DE3E52EF12CEC0EFD1EC7016CE97AE233
:108F40000E94F97B8E010C5B1F4FC80163EA7AE235
:108F50000E94F97BC501B601A70198010E949643C2
:108F6000C8010E940F7CC7010E940F7CC6010E94AD
:108F70000F7CC5010E940F7C0C94705481EE9AE224
:108F800060E040E00E94266E80916E2A882309F4FA
:108F900045C081EE9AE268E879E00E94DC7781EED4
:108FA0009AE260E041E00E94266E0E944C4281EE0F
:108FB0009AE264E041E00E94266EE091E602F0E071
:108FC000E957F04E608170E06F5F7F4F81EE9AE26B
:108FD0004AE050E00E94F17881EE9AE26BE041E0D5
:108FE0000E94266E80916E1F90E026E239E0829FFB
:108FF000F001839FF00D929FF00D1124E850FC4F7B
:10900000608170E06F5F7F4F81EE9AE24AE050E04E
:109010000E94F17881E080936F2A77C08091E3020B
:109020009091E402029749F480916F2A882329F4F1
:109030008091682A882309F468C082E090E09093C8
:10904000E4028093E30210926F2A1092682A81EE64
:109050009AE267E779E00E94DC7781EE9AE260E0CD
:1090600041E00E94266E0E944C4281EE9AE262E04C
:1090700041E00E94266E6091E7026F5B81EE9AE20A
:109080000E94FF776091E80270E06F5F7F4F8091F0
:10909000E70290E044E0880F991F4A95E1F7681BCA
:1090A000790B81EE9AE24AE050E00E94F1788091DB
:1090B000E8028093012B81EE9AE269E041E00E9490
:1090C000266E81EE9AE265E00E941C6E81EE9AE2C5
:1090D00061E071E00E94047980917E02837059F40E
:1090E000609176027091770281EE9AE24AE050E058
:1090F0000E948E7806C081EE9AE263E779E00E94D2
:10910000DC77809176028093002B9091E802809129
:10911000012B981719F182E00E941F426091E7022B
:109120006F5B81EE9AE20E94FF776091E80270E047
:109130006F5F7F4F8091E70290E034E0880F991FC6
:109140003A95E1F7681B790B81EE9AE24AE050E02C
:109150000E94F1788091E8028093012B8091002B8E
:1091600090E020917602309177028217930711F4F4
:109170000C9470548BE00E941F42609176027091B3
:10918000770281EE9AE24AE050E00E948E78809168
:1091900076028093002B0C9470548091E30290919E
:1091A000E4020397C1F087E89AE268E071E00E9468
:1091B000037BBC0180E89AE20E94E27BBC0189E764
:1091C0009AE20E94E27BBC0182E79AE20E94E27B83
:1091D00081E00E9409438091E3029091E4020397A9
:1091E00041F480919A01882321F48091682A882390
:1091F00081F181EE9AE260E040E00E94266E81EE0D
:109200009AE262E679E00E94DC7780916B2AE82F8F
:10921000F0E0EE0FFF1FEC52FD4F659174918E014F
:109220000F5F1F4FC8010E94E407E0916B2AF0E036
:10923000E556FE4F81EE9AE2608140E00E94266E84
:1092400081EE9AE2B8010E94047910929A0110927C
:10925000682A8E01055B1F4FE091E602F0E0E856B8
:10926000F04E608170E06F5F7F4FC8014AE00E945E
:109270004D7BCE018E5A9F4FB8010E94047C809195
:10928000731F882311F460E201C06EE792E5C92ED6
:10929000D12CCC0EDD1EC6010E94877A8C0189E597
:1092A000E82EF12CEC0EFD1EE091E602F0E0E9570D
:1092B000F04E608170E06F5F7F4FC7014AE00E940F
:1092C0004D7BC801B7010E94987ABC018E01005AFB
:1092D0001F4FC8010E94F97B8EE89AE2B8010E94F4
:1092E000E27BC8010E940F7CC7010E940F7CC6016F
:1092F0000E94157CCE01855B9F4F0E940F7C2091C0
:10930000E60240916E1F203171F4242F30E086E296
:1093100099E0289FF001299FF00D389FF00D11244E
:10932000E85AF34F19C030E050E084E890E0289FFD
:10933000F001299FF00D389FF00D112486E299E08D
:109340009C01429FC001439F900D529F900D11249C
:10935000E80FF91FEE56FB4F8081682F70E06F5FBA
:109360007F4F8E0109591F4FC8014AE00E944D7B73
:1093700085E99AE2B8010E94E27BC8010E940F7C55
:109380008CE99AE260E070E00E94037B4091E60283
:10939000403139F48E0102591F4FC8016CE071E071
:1093A00092C08091B52A882309F481C0E42FF0E0AF
:1093B000EE0FFF1FE459FC4F65917491CE010196A9
:1093C0000E94E4074091E6024C3090F580916E1FB8
:1093D00090E026E239E0829FF001839FF00D929F9A
:1093E000F00D1124E850FC4FE40FF11D8781882314
:1093F00011F460E201C06BE2BCE7CB2ED12CCC0EA5
:10940000DD1EC6010E94C97BA5E7EA2EF12CEC0EF9
:10941000FD1EC701BE016F5F7F4F0E94CF7AC6015C
:10942000B7010E94987ABC018E010D571F4F8AC068
:109430004F3041F480916D02882321F08E01065750
:109440001F4F3EC080916E1F90E026E239E0829F60
:10945000F001839FF00D929FF00D1124E850FC4F16
:10946000E40FF11D8781882311F460E201C06BE2F3
:10947000F8E9CF2ED12CCC0EDD1EC6010E94C97B8F
:10948000E1E9EE2EF12CEC0EFD1E6091E60270E09B
:109490006F5F7F4FC7014AE00E944D7BC601B70155
:1094A0000E94987ABC018E0101561F4F4BC04F306D
:1094B000A9F480916D02882389F08E010A551F4F0F
:1094C000C8016FE071E00E94CF7A83EA9AE2B801A6
:1094D0000E94E27BC8010E940F7C45C080916E1FF4
:1094E00090E026E239E0829FF001839FF00D929F89
:1094F000F00D1124E850FC4FE40FF11D8781882303
:1095000011F460E201C06BE274EBC72ED12CCC0EDB
:10951000DD1EC6010E94C97B6DEAE62EF12CEC0E21
:10952000FD1E6091E60270E06F5F7F4FC7014AE069
:109530000E944D7BC601B7010E94987ABC018E0142
:1095400005541F4FC8010E94F97B83EA9AE2B801D3
:109550000E94E27BC8010E940F7CC7010E940F7C21
:10956000C6010E94157C52ECA52EB12CAC0EBD1E7E
:10957000C5016EE87AE20E94F97B49ECC42ED12C39
:10958000CC0EDD1EC60165E97AE20E94F97B30ED62
:10959000E32EF12CEC0EFD1EC7016CE97AE20E946D
:1095A000F97B8E0109521F4FC80163EA7AE20E94DB
:1095B000F97BC501B601A70198010E949643C80135
:1095C0000E940F7CC7010E940F7CC6010E940F7C85
:1095D000C5010E940F7C80E00E94094383E090E077
:1095E000B2CA8091E3029091E4020C9721F4809139
:1095F000682A8823B9F181EE9AE260E040E00E9497
:10960000266E0E944C4281EE9AE262E040E00E94A7
:10961000266E81EE9AE26DE579E00E94DC7781EEBC
:109620009AE260E041E00E94266E0E944C4281EE88
:109630009AE262E041E00E94266E81EE9AE26AE5DB
:1096400079E00E94DC77E091DE2AF0E0E255F74F06
:10965000E49181EE9AE26E2F4AE050E00E949F78FA
:109660001092682AE091DE2AF0E0E255F74FE4918B
:109670008E0102521F4FC8016E2F4AE00E947E7B6E
:1096800082E79AE2B8010E94E979F82EC8010E94A7
:109690000F7CFF20A9F581EE9AE264E041E00E9490
:1096A000266E81EE9AE266E579E00E94DC7781EE33
:1096B0009AE264E041E00E94266EE091DE2AF0E04A
:1096C000E255F74FE49181EE9AE26E2F4AE050E0C6
:1096D0000E949F78E091DE2AF0E0E255F74FE49196
:1096E0008E010B511F4FC8016E2F4AE00E947E7BF6
:1096F00082E79AE2B8010E94E27BC8010E940F7CD7
:109700008CE090E020CA8091F103882321F0813021
:1097100009F032C2DFC18091E3029091E402079721
:1097200021F480915A018823A9F087E89AE268E041
:1097300071E00E94037BBC0180E89AE20E94E27B18
:10974000BC0189E79AE20E94E27BBC0182E79AE2CF
:109750000E94E27B8091E3029091E402079771F40A
:109760009091F10380915A01981741F480919A01E8
:10977000882321F48091682A8823A1F181EE9AE25E
:1097800060E040E00E94266E81EE9AE265E479E0B6
:109790000E94DC7780916B2AE82FF0E0EE0FFF1F2C
:1097A000EC54FD4F659174918E010F5F1F4FC801FE
:1097B0000E94E407E0916B2AF0E0E556FE4F81EE4F
:1097C0009AE2608140E00E94266E81EE9AE2B80142
:1097D0000E9404798091F10380935A0110929A01BA
:1097E0001092682A8E0104511F4FE091E602F0E0CA
:1097F000E856F04E608170E06F5F7F4FC8014AE02D
:109800000E944D7BCE018D509F4FB8010E94047C79
:109810008091731F882311F460E201C06EE793EF1B
:10982000C92ED12CCC0EDD1EC6010E94877A8C0178
:109830008AEFE82EF12CEC0EFD1EE091E602F0E03E
:10984000E957F04E608170E06F5F7F4FC7014AE0DB
:109850000E944D7BC801B7010E94987ABC018E011D
:109860000F5F1E4FC8010E94F97B8EE89AE2B80193
:109870000E94E27BC8010E940F7CC7010E940F7CFE
:10988000C6010E94157CCE0184519F4F0E940F7C1F
:1098900020916E1F30E08091820290E0FC01EE0F7B
:1098A000FF1FE80FF91FA6E2CA2EA9E0DA2E2C9DB1
:1098B000D0012D9DB00D3C9DB00D1124EA0FFB1F72
:1098C000E25AF34F90819F70AA5AB34FEC918CE00B
:1098D000E89FF0011124E90FF11DE057FC4FE491DE
:1098E000F0E0EE0FFF1FEE5AFC4F659174917E0180
:1098F0000894E11CF11CC7010E94E4078E01085F77
:109900001E4FC801B7010E94CF7A85E99AE2B801DB
:109910000E94E27BC8010E940F7C8091820290E04D
:1099200020916E1F30E0FC01EE0FFF1FE80FF91FC2
:109930002C9DC0012D9D900D3C9D900D1124E80F94
:10994000F91FE25AF34F808182958770E82FF0E08B
:10995000EE0FFF1FEC5BFC4F65917491C7010E94F5
:10996000E4078E01015F1E4FC801B7010E94CF7A44
:109970008CE99AE2B8010E94E27BC8010E940F7C48
:1099800020916E1F30E08091820290E0FC01EE0F8A
:10999000FF1FE80FF91F2C9DD0012D9DB00D3C9DA0
:1099A000B00D1124EA0FFB1FE45AF34F6081669556
:1099B0006F71262F2F5FA95AB34FAC91A03619F4BF
:1099C000220F220F03C0A03309F4220FCE018A5EBA
:1099D0009E4F2A1729F464E171E00E94CF7A06C0F5
:1099E00070E06F5F7F4F4AE00E944D7B8E010A5E00
:1099F0001E4F83EA9AE2B8010E94E27BC8010E94EE
:109A00000F7C0DE1A02E01E0B02EAC0EBD1EC501F5
:109A10006EE87AE20E94F97B14E2C12E11E0D12EA9
:109A2000CC0EDD1EC60165E97AE20E94F97BBBE23D
:109A3000EB2EB1E0FB2EEC0EFD1EC7016CE97AE2C5
:109A40000E94F97B8E010E5C1E4FC80163EA7AE228
:109A50000E94F97BC501B601A70198010E949643B7
:109A6000C8010E940F7CC7010E940F7CC6010E94A2
:109A70000F7CC5010E940F7C81EE9AE26FE041E00D
:109A80000E94266E8091820290E020916E1F30E04D
:109A9000FC01EE0FFF1FE80FF91F86E299E0AC0111
:109AA000249FC001259F900D349F900D1124E80F35
:109AB000F91FE25AF34F808187FF07C081EE9AE2D7
:109AC00063E479E00E94DC7757C081EE9AE26AE0B5
:109AD00071E050C08091E3029091E402079741F455
:109AE00080915A01813021F48091682A882391F075
:109AF00081EE9AE260E040E00E94266E81EE9AE2FA
:109B000062E379E00E94DC778091F10380935A014F
:109B10001092682A10926B2A81EE9AE260E041E08E
:109B20000E94266E0E944C4281EE9AE262E041E081
:109B30000E94266E80916E1F90E026E239E0829F9F
:109B4000F001839FF00D929FF00D1124EA5AF34F1C
:109B50008081E82FF0E0EE0FFF1FE451FD4F65918B
:109B600074918E01045B1D4FC8010E94E40781EED1
:109B70009AE2B8010E94047987E090E00C94A34532
:109B80008091E3029091E4020697A9F087E89AE2B7
:109B900068E071E00E94037BBC0180E89AE20E94C9
:109BA000E27BBC0189E79AE20E94E27BBC0182E78A
:109BB0009AE20E94E27BE0915A2AF0E0E45DF54DE2
:109BC00092898091FE2A981771F080E89AE268E005
:109BD00071E00E94037BE0915A2AF0E0E45DF54DCC
:109BE00082898093FE2A8091E3029091E402069795
:109BF00041F480919A01882321F48091682A882376
:109C0000B1F181EE9AE260E040E00E94266E81EEC2
:109C10009AE261E279E00E94DC7780916B2AE82F7A
:109C2000F0E0EE0FFF1FE455FD4F659174918E013A
:109C30000F5F1F4FC8010E94E407E0916B2AF0E01C
:109C4000E556FE4F81EE9AE2608140E00E94266E6A
:109C500081EE9AE2B8010E94047986E090E0909348
:109C6000E4028093E30210929A011092682AE09134
:109C70005A2AF0E0E45DF54D8081E82FF0E0EE0F28
:109C8000FF1FE85FFC4F659174917E010894E11C11
:109C9000F11CC7010E94E4078E01075C1E4F609112
:109CA0005A2A70E06F5F7F4FC8014AE00E944D7BE7
:109CB0008EE89AE2B8010E94E27BC8010E940F7C04
:109CC0008E01005C1E4FC801B7010E94CF7A85E962
:109CD0009AE2B8010E94E27BC8010E940F7C809149
:109CE0005A2AE82FF0E0E45DF54D82899E01295B58
:109CF0003E4F882331F0C90160E070E00E94CF7AC6
:109D000008C0628170E06F5F7F4FC9014AE00E9426
:109D10004D7B8E01095B1E4F8CE99AE2B8010E94CF
:109D2000E27BC8010E940F7C8E01025B1E4FE09116
:109D30005A2AF0E0EE0FFF1FEE0FFF1FE05DF54D1A
:109D4000608171818281938120E030E048EC52E4AF
:109D50000E94CE7D0E94EC7C9B01AC01C801622F69
:109D60004AE00E947E7B83EA9AE2B8010E94E27B8D
:109D7000C8010E940F7C35E5A32E31E0B32EAC0E56
:109D8000BD1EC5016EE87AE20E94F97B2CE5C22E69
:109D900021E0D22ECC0EDD1EC60165E97AE20E94DA
:109DA000F97B93E6E92E91E0F92EEC0EFD1EC7013A
:109DB0006CE97AE20E94F97B8E0106591E4FC801B8
:109DC00063EA7AE20E94F97BC501B601A701980116
:109DD0000E949643C8010E940F7CC7010E940F7C1D
:109DE000C6010E940F7CC5010E940F7CE0915A2A97
:109DF000F0E0E45DF54D8289882309F471C50E9485
:109E0000AE426EC58091E3029091E4020997A9F0F9
:109E100087E89AE268E071E00E94037BBC0180E879
:109E20009AE20E94E27BBC0189E79AE20E94E27B0F
:109E3000BC0182E79AE20E94E27B81EE9AE260E056
:109E400040E00E94266E8091E6022091E30230916C
:109E5000E402803109F044C02930310569F4809171
:109E60009A01882349F48091FD2A803129F4809158
:109E7000682A882309F475C081EE9AE260E179E0EE
:109E80000E94DC7780916B2AE82FF0E0EE0FFF1F35
:109E9000E453FD4F659174918E010F5F1F4FC80110
:109EA0000E94E407E0916B2AF0E0E556FE4F81EE58
:109EB0009AE2608140E00E94266E81EE9AE2B8014B
:109EC0000E94047989E090E09093E4028093E30299
:109ED0001092682A10929A0180E18093FD2A41C075
:109EE0002930310561F480919A01882341F48091F1
:109EF000FD2A803121F08091682A882391F181EE3A
:109F00009AE26FEF78E00E94DC7780916B2AE82F6D
:109F1000F0E0EE0FFF1FEC53FD4F659174918E0141
:109F20000F5F1F4FC8010E94E407E0916B2AF0E029
:109F3000E556FE4F81EE9AE2608140E00E94266E77
:109F400081EE9AE2B8010E94047989E090E0909352
:109F5000E4028093E3021092682A10929A01109210
:109F6000FD2A80916E1FA82FB0E06091E6028091DB
:109F70008202282F30E083E994E0A89FA001A99FE6
:109F8000500DB89F500D1124862F90E0FC0116E073
:109F9000EE0FFF1F1A95E1F7880F991FE80FF91FC1
:109FA000E40FF51FE20FF31FEE0FFF1FED5EFB4FF7
:109FB0009080969496949694603161F5F901EE0F35
:109FC000FF1FE20FF31F86E299E09C01A29FC001F0
:109FD000A39F900DB29F900D1124E80FF91FDF0190
:109FE000A45AB34F9C91929596959695937011961D
:109FF0008C918770880F880F892BA82EBB2440EF87
:10A000005FEFA40EB51EE35AF34FC080C694C6940A
:10A01000C6943DC0862F90E0FC01A6E0EE0FFF1F26
:10A02000AA95E1F7880F991FE80FF91FE40FF51FB4
:10A03000E20FF31FEE0FFF1FEE5EFB4F9081929534
:10A0400096959695937081818770880F880F892BDC
:10A05000A82EBB2480EF9FEFA80EB91E862F90E09C
:10A06000FC0106E0EE0FFF1F0A95E1F7880F991F2C
:10A07000E80FF91FE40FF51FE20FF31FEE0FFF1FAC
:10A08000EE5EFB4FC080C694C6949FE0C9222AE0D2
:10A090002C1590F4EC2DF0E0EE0FFF1FE851FD4F72
:10A0A000659174918E010F5F1F4FC8010E94E407F4
:10A0B0008CE99AE2B80106C0CC2039F48CE99AE226
:10A0C00068E171E00E94037B3DC038E0C31629F4CB
:10A0D0008CE99AE26CE171E0F5CF49E0C41629F40D
:10A0E0008CE99AE260E271E0EDCF5AE0C51629F4FE
:10A0F0008CE99AE264E271E0E5CFE8E7EE2EE1E078
:10A10000FE2EEC0EFD1EC70168E271E00E94E97AA6
:10A110008E010F581E4F6C2D70E06F5F7F4FC8018E
:10A120004AE00E944D7BC701B8010E94987ABC01A9
:10A130008CE99AE20E94E27BC8010E940F7CC70171
:10A140000E94157C8E0101581E4FE091E602F0E05E
:10A15000E856F04E608170E06F5F7F4FC8014AE0C3
:10A160000E944D7BCE018A579E4FB8010E94047C0D
:10A170008091731F882311F460E201C06EE776E8D6
:10A18000C72E71E0D72ECC0EDD1EC6010E94877A45
:10A190008C016DE8E62E61E0F62EEC0EFD1EE091DE
:10A1A000E602F0E0E957F04E608170E06F5F7F4FAC
:10A1B000C7014AE00E944D7BC801B7010E94987A0E
:10A1C000BC018E010C561E4FC8010E94F97B8EE81F
:10A1D0009AE2B8010E94E27BC8010E940F7CC7018D
:10A1E0000E940F7CC6010E94157CCE0181589E4FB3
:10A1F0000E940F7CB7FC23C052EAE52E51E0F52EF9
:10A20000EC0EFD1EC7016BE271E00E94E97A8E013F
:10A2100005561E4FC801B5014AE00E944D7BC7019B
:10A22000B8010E94987ABC0185E99AE20E94E27B1B
:10A23000C8010E940F7CC7010E94157C10C08E01CE
:10A2400007551E4FC801B5014AE00E944D7B85E9C4
:10A250009AE2B8010E94E27BC8010E940F7C209123
:10A260006E1F30E08091820290E0FC01EE0FFF1F34
:10A27000E80FF91F86E299E0289FD001299FB00DD1
:10A28000389FB00D1124EA0FFB1FE45AF34F608191
:10A2900066956F71262F2F5FA95AB34FAC91A036E8
:10A2A00019F4220F220F03C0A03309F4220F80916A
:10A2B000E6028031E1F4CE0180559E4F2A1729F441
:10A2C00064E171E00E94CF7A06C070E06F5F7F4F5B
:10A2D0004AE00E944D7B8E0100551E4F83EA9AE2B0
:10A2E000B8010E94E27BC8010E940F7C51C035EC8E
:10A2F000A32E31E0B32EAC0EBD1E992041F4C50152
:10A3000068E171E00E94CF7AEE24FF2428C02EEB92
:10A31000E22E21E0F22EEC0EFD1EC7016DE271E08F
:10A320000E94E97A8E0109541E4FE92DF0E0E35BAB
:10A33000FE4F608180E891E070E00E94707EC8016D
:10A340004AE00E944D7BC701B8010E94987ABC0187
:10A35000C5010E94F97BEE24E394FF24F3948E015F
:10A360000B531E4F83EA9AE2B8010E94E27BC801B8
:10A370000E940F7CFF2029F0CE0189549E4F0E943D
:10A380000F7CEE2029F0CE0182549E4F0E94157C56
:10A390009CECA92E91E0B92EAC0EBD1EC5016EE855
:10A3A0007AE20E94F97B83EDC82E81E0D82ECC0E94
:10A3B000DD1EC60165E97AE20E94F97B0AEDE02E16
:10A3C00001E0F02EEC0EFD1EC7016CE97AE20E945E
:10A3D000F97B8E010F511E4FC80163EA7AE20E9499
:10A3E000F97BC501B601A70198010E949643C801F7
:10A3F0000E940F7CC7010E940F7CC6010E940F7C47
:10A40000C5010E940F7C8091E602803109F068C28C
:10A4100081EE9AE26FE041E00E94266E8091820216
:10A4200090E020916E1F30E0FC01EE0FFF1FE80F5F
:10A43000F91F86E299E0AC01249FC001259F900D91
:10A44000349F900D1124E80FF91FE25AF34F8081D9
:10A4500087FF05C081EE9AE26DEF78E047C081EE9C
:10A460009AE26AE071E00E9404793AC29093E402B1
:10A470008093E30281EE9AE260E040E00E94266E63
:10A4800081EE9AE26CEE78E00E94DC7781EE9AE24F
:10A4900060E041E00E94266E0E944C4281EE9AE20A
:10A4A00062E041E00E94266E8091422A882329F0D2
:10A4B00081EE9AE268EE78E004C081EE9AE265EE01
:10A4C00078E00E94DC7781EE9AE26AE041E00E9447
:10A4D000266E80912803882329F081EE9AE261EEAE
:10A4E00078E004C081EE9AE26EED78E00E94DC77BD
:10A4F000F7C18091E3029091E4020197A9F087E807
:10A500009AE268E071E00E94037BBC0180E89AE275
:10A510000E94E27BBC0189E79AE20E94E27BBC01D7
:10A5200082E79AE20E94E27B8091E3029091E4024A
:10A53000019741F480919A01882321F48091682A3F
:10A54000882381F181EE9AE260E040E00E94266E6D
:10A5500081EE9AE26DEC78E00E94DC7780916B2AC4
:10A56000E82FF0E0EE0FFF1FE452FD4F659174916C
:10A570008E010F5F1F4FC8010E94E407E0916B2A14
:10A58000F0E0E556FE4F81EE9AE2608140E00E94E5
:10A59000266E81EE9AE2B8010E94047910929A0127
:10A5A0001092682A8E0108511E4F60912C2870E08D
:10A5B0006F5F7F4FC8014AE00E944D7B8EE89AE2B0
:10A5C000B8010E94E27BC8010E940F7C8E010151FC
:10A5D0001E4F60912D2870912E286F5F7F4FC8010C
:10A5E0004AE00E944D7B85E99AE2B8010E94E27B35
:10A5F000C8010E940F7CA6EFCA2EA1E0DA2ECC0E75
:10A60000DD1EE0912D28F0912E28E55DF74D618546
:10A6100062956F706F5BC6010E94B07BF4E0EF2E15
:10A62000F2E0FF2EEC0EFD1EC701B6010E94047C75
:10A63000E0912D28F0912E28E55DF74D21858E01C2
:10A6400003501E4F622F70E06F5F7F4F822F829505
:10A650008F7090E0E4E0880F991FEA95E1F7681B9E
:10A66000790BC8014AE00E944D7BC701B8010E94E6
:10A67000987ABC018CE99AE20E94E27BC8010E94B0
:10A680000F7CC7010E94157CC6010E940F7C8AEADC
:10A690009AE26CE97AE20E94E27B88E080936C2A7D
:10A6A0008E01055F1D4F60913128709132286F5FD8
:10A6B0007F4FC8014AE00E941C7B83EA9AE2B801FE
:10A6C0000E94E27BC8010E940F7C72E1A72E72E01B
:10A6D000B72EAC0EBD1EC5016EE87AE20E94F97B72
:10A6E00069E1C62E62E0D62ECC0EDD1EC60165E9FC
:10A6F0007AE20E94F97B50E2E52E52E0F52EEC0E54
:10A70000FD1EC7016CE97AE20E94F97B8E01095DAA
:10A710001D4FC80163EA7AE20E94F97BC501B601C8
:10A72000A70198010E949643C8010E940F7CC701AF
:10A730000E940F7CC6010E940F7CC5010E940F7C05
:10A7400081E090E00C94A3458091E3029091E402B3
:10A75000892BC9F480919A018823A9F48091682AF1
:10A76000882389F48091012B90E020912D2830914D
:10A770002E288217930739F49091002B80912C2872
:10A78000981709F4A9C081EE9AE260E040E00E94C7
:10A79000266E0E944C4281EE9AE260E040E00E9408
:10A7A000266E81EE9AE260EC78E00E94DC776091A0
:10A7B0002C2870E06F5F7F4F81EE9AE24AE050E014
:10A7C0000E94F17880912C288093002B81EE9AE2F0
:10A7D00060E041E00E94266E0E944C4281EE9AE2C7
:10A7E00060E041E00E94266E81EE9AE26BEB78E039
:10A7F0000E94DC7780912D288093012B60912D2879
:10A8000070912E286F5F7F4F81EE9AE24AE050E010
:10A810000E94F17881EE9AE268E041E00E94266EA3
:10A8200081EE9AE265EB78E00E94DC774EE2C42E7E
:10A8300042E0D42ECC0EDD1EE0912D28F0912E2882
:10A84000E55DF74D618562956F706F5BC6010E9493
:10A85000B07B3CE3E32E32E0F32EEC0EFD1EC7018D
:10A86000B6010E94047CE0912D28F0912E28E55D30
:10A87000F74D21858E010B5C1D4F622F70E06F5FDD
:10A880007F4F822F82958F7090E024E0880F991F70
:10A890002A95E1F7681B790BC8014AE00E944D7BBD
:10A8A000C701B8010E94987ABC018CE99AE20E9423
:10A8B000E27BC8010E940F7CC7010E94157CC60183
:10A8C0000E940F7C81EE9AE26CE97AE20E9407799D
:10A8D00010929A011092682A1092E4021092E302F8
:10A8E000CB5ADD4F0FB6F894DEBF0FBECDBFCF9170
:10A8F000DF911F910F91FF90EF90DF90CF90BF906D
:10A90000AF909F900895CF92DF92EF92FF920F93B6
:10A910001F937B018C01ADE2CA2EACE2DA2E9C01C2
:10A9200044275527205BC601622F0E94826F55275E
:10A93000412F302F2F2DC601622F0E940E70C601AD
:10A940006E2D0E940E701F910F91FF90EF90DF907F
:10A95000CF9008953F924F925F926F927F928F9225
:10A960009F92AF92BF92CF92DF92EF92FF920F939E
:10A970001F932091312830913228220F232F221F3C
:10A98000330B3195322EE82EFF2400E010E030E04A
:10A9900040E050E071E8A72E79E0B72EC12CD12C11
:10A9A000A20EB31EC41ED51ED801C70162E0880FD7
:10A9B000991FAA1FBB1F6A95D1F7A80EB91ECA1E00
:10A9C000DB1E97E0AA0CBB1CCC1CDD1C9A95D1F7B2
:10A9D00029013A0187E0440C551C661C771C8A95B6
:10A9E000D1F78824C601B5010E948354831401F570
:10A9F00099240AC0E92DF0E0E55DF74D8DE29CE277
:10AA000061850E940E709394292D30E040E050E063
:10AA10008091312890913228A0E0B0E08419950906
:10AA2000A609B709281739074A075B0718F30EC0AC
:10AA30009924E92DF0E0E55DF74D8DE29CE261851A
:10AA40000E940E70939480E8981699F78DE29CE22C
:10AA50000E9451706AE070E080E090E00E944A73CA
:10AA60008394381408F0BECFB9E0EE0CFF1C001F31
:10AA7000111FBA95D1F783E792ECA4E0B0E0E80E9D
:10AA8000F91E0A1F1B1FC801B7010E9483548DE2E3
:10AA90009CE2609131280E940E70609132288DE214
:10AAA0009CE20E940E708DE29CE20E9451706AE06E
:10AAB00070E080E090E00E944A731F910F91FF9038
:10AAC000EF90DF90CF90BF90AF909F908F907F904E
:10AAD0006F905F904F903F900895EF92FF920F9389
:10AAE0001F9360E070EC84E090E00E9483540DE2DC
:10AAF0001CE260917E026370C8010E940E70C80162
:10AB0000609178020E940E70C801609171020E94EB
:10AB10000E70C801609170020E940E70C8016091B1
:10AB200072020E940E70C801609175020E940E7040
:10AB3000C80160916E020E940E70C80160916D02A2
:10AB40000E940E70FAE7EF2EF2E0FF2EC801F70127
:10AB500060810E940E70F7016181C8010E940E7031
:10AB6000C8010E9451706AE070E080E090E00E94AD
:10AB70004A731F910F91FF90EF90089580917E028C
:10AB800082FF3BC0837090E081309105D9F0823024
:10AB90009105F1F0892B61F580917802909179020D
:10ABA000909377028093760280913E2A882319F051
:10ABB00080E00E940C1480913F2A882319F081E0E4
:10ABC0000E940C140E94932581E08093A80110C07C
:10ABD00080E293E0A0E0B0E080939F019093A00119
:10ABE000A093A101B093A2010E9493251092A80105
:10ABF00080917E028B7F80937E0280916F028823FA
:10AC000051F080912F0283FF06C00E946D55109273
:10AC10006F020E94384280917C0290917D020897D9
:10AC200011F010926F0280917E028370823051F594
:10AC300020919F013091A0014091A1015091A2016A
:10AC400027593F4F4F4F5F4F60E67AEE80E090E02C
:10AC50000E94837ECA01B9010E94187D0E94EC7C8B
:10AC6000709377026093760280913E2A882319F0D0
:10AC700080E00E940C1480913F2A882319F081E023
:10AC80000E940C1408953F924F925F926F927F92B0
:10AC90008F929F92AF92BF92CF92DF92EF92FF92EC
:10ACA0000F931F93DF93CF9300D000D000D0CDB788
:10ACB000DEB7062FC82EDD24EE24FF24603109F410
:10ACC00033C1262F30E040E050E029833A834B83A4
:10ACD0005C83C701B60123E130E040E050E00E9410
:10ACE000317E29813A814B815C81620F731F841F01
:10ACF000951FE7E0660F771F881F991FEA95D1F728
:10AD00000E9483543324402E552484E890E0489ECA
:10AD10004001499E900C589E900C11245201AA0C9F
:10AD2000BB1CC20166E0880F991F6A95E1F7A80E67
:10AD3000B91E50C043E954E0249FF001259FF00D57
:10AD4000349FF00D1124EA0DFB1DE30DF11DEE0FF4
:10AD5000FF1FDF01AE5EBB4F2C91022F06950170E5
:10AD600010E0000F111F822F869586958F7090E05E
:10AD7000880F991F880F991F082B192B822F81701C
:10AD800090E0082B192B2295269526952370119675
:10AD90008C918770880F880F822B90E0B6E0880F27
:10ADA000991FBA95E1F7082B192BED5EFB4F8081B7
:10ADB000887F8E831D828D819E81082B192B8DE2C9
:10ADC0009CE2602F0E940E708DE29CE2612F0E9437
:10ADD0000E70339480916E1F282F30E0E6E26E2EC5
:10ADE000E9E07E2E269DF001279DF00D369DF00DA9
:10ADF0001124E80DF91DEE56FB4F8081831508F0F4
:10AE000099CF8DE29CE20E9451706AE070E080E090
:10AE100090E00E944A73C701B60120E839E040E0A3
:10AE200050E00E94317E7B018C0120E038E040E060
:10AE300050E0E20EF31E041F151F69817A818B8199
:10AE40009C8126E030E040E050E00E94317EE60E3A
:10AE5000F71E081F191FC801B7010E9483548DE215
:10AE60009CE260E00E940E7080916E1F90E0869DD3
:10AE7000F001879DF00D969DF00D1124E80DF91D50
:10AE8000EE56FB4F8DE29CE260810E940E70809135
:10AE90006E1F90E0869DF001879DF00D969DF00D50
:10AEA0001124E80DF91DED56FB4F8DE29CE2608107
:10AEB0000E940E7080916E1F90E0869DF001879D2C
:10AEC000F00D969DF00D1124E80DF91DEB56FB4F8A
:10AED0008DE29CE260810E940E7080916E1F90E076
:10AEE000869DF001879DF00D969DF00D1124E80DD3
:10AEF000F91DEC56FB4F8DE29CE260810E940E70C2
:10AF000080916E1F90E0869DF001879DF00D969DCB
:10AF1000F00D1124E850FC4FE40DF51D8DE29CE28C
:10AF200067810E940E70F5C0C701B60120E839E0C4
:10AF300040E050E00E94317E6B017C016058774F09
:10AF40008F4F9F4F0E94835480916E1F90E006E2C6
:10AF500019E0809FF001819FF00D909FF00D11246A
:10AF6000E85AF34F8DE29CE260810E940E7080915E
:10AF70006E1F90E0809FF001819FF00D909FF00D7B
:10AF80001124E95AF34F8DE29CE260810E940E7019
:10AF900080916E1F90E0809FF001819FF00D909F47
:10AFA000F00D1124E75AF34F8DE29CE260810E947C
:10AFB0000E7080916E1F90E0809FF001819FF00DD8
:10AFC000909FF00D1124E65AF34F8DE29CE26081D0
:10AFD0000E940E7080916E1F90E0809FF001819F13
:10AFE000F00D909FF00D1124EA5AF34F8DE29CE290
:10AFF00060810E940E7000E076E2A72E79E0B72E05
:10B0000011C0802F90E0FC01EE0FFF1FE80FF91F29
:10B01000E20FF31FE25AF34F60818DE29CE20E943F
:10B020000E700F5F80916E1F90E08A9D90018B9D46
:10B03000300D9A9D300D1124F901E85AF34F8081AB
:10B040000817F8F28DE29CE20E9451706AE070E00D
:10B0500080E090E00E944A73C701B6016050774FCC
:10B060008F4F9F4F0E948354FF2456E2C52E59E014
:10B07000D52E3EC08F2D90E0FC01EE0FFF1FE80F94
:10B08000F91FE20FF31FDF01A45AB34F2C91022FD7
:10B0900006950F7110E0000F111F422F4295469543
:10B0A0004695437011968C918770880F880F842B7A
:10B0B00090E0B6E0880F991FBA95E1F7082B192B9D
:10B0C000217030E0022B132BE35AF34F8081A8EF5D
:10B0D0009A2E98228824082919298DE29CE2602F53
:10B0E0000E940E708DE29CE2612F0E940E70F3941C
:10B0F00080916E1F90E08C9D90018D9D300D9C9DE8
:10B10000300D1124F901E85AF34F80818F1508F0B2
:10B11000B1CF8DE29CE20E9451706AE070E080E065
:10B1200090E00E944A7326960FB6F894DEBF0FBED9
:10B13000CDBFCF91DF911F910F91FF90EF90DF90E6
:10B14000CF90BF90AF909F908F907F906F905F90C7
:10B150004F903F9008952F923F924F925F927F922F
:10B160008F929F92AF92BF92CF92DF92EF92FF9217
:10B170000F931F93DF93CF9300D000D0CDB7DEB7EE
:10B180007724C8C0003109F43FC0C701B6010E944E
:10B19000835410E08DE29CE262E00E940E708DE22A
:10B1A0009CE264E00E940E701F5F103499F78DE2FC
:10B1B0009CE20E9451706AE070E080E090E00E94A2
:10B1C0004A73C501B4010E9483548DE29CE261E0A0
:10B1D0000E940E708DE29CE26FE00E940E708DE284
:10B1E0009CE268E10E940E708DE29CE261E00E94A8
:10B1F0000E708DE29CE260E00E940E708DE29CE297
:10B2000060E00E940E7044C069817A818B819C81CC
:10B210000E9483548DE29CE26FE00E940E708DE2EA
:10B220009CE268E10E940E708DE29CE261E00E9467
:10B230000E708DE29CE260E00E940E708DE29CE256
:10B2400060E00E940E7010E08DE29CE260E30E94DC
:10B250000E701F5F1034C1F78DE29CE20E945170A6
:10B260006AE070E080E090E00E944A73C201B101A0
:10B270000E94835410E08DE29CE268E10E940E700F
:10B280008DE29CE264E00E940E701F5F103499F71B
:10B290008DE29CE20E9451706AE070E080E090E0F4
:10B2A0000E944A730F5F86E090E0A0E0B0E0880E55
:10B2B000991EAA1EBB1E80E890E0A0E0B0E0C80E78
:10B2C000D91EEA1EFB1E013109F05CCF272D269501
:10B2D0002695269581E090E0A0E0B0E004C0880FBC
:10B2E000991FAA1FBB1F2A95D2F79C01AD0180911F
:10B2F000172B9091182B822B932B9093182B8093C4
:10B30000172B60E070E040E00E94040D739490E819
:10B31000791651F1672D70E080E090E020E839E087
:10B3200040E050E00E94317E6B017C01812CA8E05E
:10B330009A2EA12CB12C860E971EA81EB91EDC01D8
:10B34000CB018058974FAF4FBF4F89839A83AB8310
:10B35000BC83212CF9E03F2E412C512C2C0C3D1CA0
:10B360004E1C5F1C00E00ECF60E070EC84E090E0CB
:10B370000E9483548DE29CE260E00E940E708DE298
:10B380009CE268E70E940E708DE29CE261E00E9400
:10B390000E708DE29CE261E00E940E708DE29CE2F4
:10B3A00061E00E940E708DE29CE20E9451706AE0A2
:10B3B00070E080E090E00E944A738DE29CE267E5D5
:10B3C00070E00E948C6F8DE29CE26FEF0E940E7025
:10B3D0008DE29CE26DEF0E940E708DE29CE260E0D7
:10B3E0000E940E708DE29CE261E00E940E708DE280
:10B3F0009CE263E00E940E708DE29CE20E9451701C
:10B400006AE070E080E090E00E944A730F900F9035
:10B410000F900F90CF91DF911F910F91FF90EF90C0
:10B42000DF90CF90BF90AF909F908F907F905F9074
:10B430004F903F902F9008953F924F925F926F925E
:10B440007F928F929F92AF92BF92CF92DF92EF92B4
:10B45000FF920F931F93A82EBB24CC24DD248601DA
:10B460007501F9E0EE0CFF1C001F111FFA95D1F7D2
:10B4700083E792ECA4E0B0E0E80EF91E0A1F1B1F60
:10B48000C801B7010E9483548DE29CE20E94517072
:10B4900078010027112790E5E90E8DE29CE26E2DE0
:10B4A00042E00E9466708DE29CE20E949F6F8C01D8
:10B4B0008DE29CE20E949F6F382F20E01070022BDB
:10B4C000132B1093322800933128045F114020F091
:10B4D0001092322810923128809131289091322890
:10B4E000880F892F881F990B9195582E282F30E0AF
:10B4F00040E050E061E8662E69E0762E812C912CC8
:10B50000620E731E841E951E92E0AA0CBB1CCC1CFE
:10B51000DD1C9A95D1F76A0C7B1C8C1C9D1C87E066
:10B52000660C771C881C991C8A95D1F7C401AA2740
:10B53000BB2710E5412E480E59016A01B7E0AA0C5D
:10B54000BB1CCC1CDD1CBA95D1F73A2CFF24C401DE
:10B55000B3010E9483548DE29CE20E945170F51465
:10B5600061F54091312843198DE29CE2642D0E94DF
:10B570006670EE240EC00E2D10E08DE29CE20E945B
:10B580009F6FF801E55DF74D8187813808F01186DE
:10B59000E3942E2D30E040E050E0809131289091EE
:10B5A0003228A0E0B0E08A199B09AC09BD09281730
:10B5B00039074A075B07F8F218C08DE29CE2642D58
:10B5C00040E80E946670EE240E2D10E08DE29CE2B1
:10B5D0000E949F6FF801E55DF74D8187813808F083
:10B5E0001186E394B0E8EB1679F7F3945F1408F052
:10B5F000AECF1F910F91FF90EF90DF90CF90BF9053
:10B60000AF909F908F907F906F905F904F903F9002
:10B6100008950F931F9360E070EC84E090E00E9427
:10B6200083548DE29CE20E9451708DE29CE264E5BD
:10B6300040E80E9466708DE29CE20E949F6F982F06
:10B640009370933009F492E0937080917E028C7F26
:10B65000892B80937E028DE29CE20E949F6F90E096
:10B660008E31910518F48EE190E005C08B3F910575
:10B6700010F08AEF90E090937902809378028DE247
:10B680009CE20E949F6F882311F481E003C0813106
:10B6900008F080E1809371028DE29CE20E949F6F2E
:10B6A000882311F481E003C0813108F080E18093A8
:10B6B00070028DE29CE20E949F6F843008F083E06C
:10B6C000809372028DE29CE20E949F6F823010F4A0
:10B6D00082E003C08B3008F08AE0809375028DE22F
:10B6E0009CE20E949F6F811181E080936E028DE247
:10B6F0009CE20E949F6F811181E080936D028DE238
:10B700009CE20E949F6F8C018DE29CE20E949F6FE1
:10B71000382F20E01070022B132B10937B02009324
:10B720007A020050104130F08FEF9FE090937B023F
:10B7300080937A021F910F9108950E94095B1092E5
:10B74000830210924C0110924B0110926D2A83E0FB
:10B7500090E090937D0280937C0280E00E94F573DC
:10B760000E947A7980916800816080936800D89AFD
:10B7700080916B00836080936B001092280380910E
:10B78000780290917902909377028093760280916B
:10B790007E02837090E08130910529F0823091051E
:10B7A00041F0892B51F40E94932581E08093A801F8
:10B7B00004C00E9493251092A80180917E028B7F85
:10B7C00080937E0280917F02882311F02C9A01C021
:10B7D0002C9880916E1F90E026E239E0829FF00164
:10B7E000839FF00D929FF00D1124DF01A25AB34FF9
:10B7F0004C91942F9F70EA5AF34FE0818CE0E89FC0
:10B80000F0011124E90FF11DE057FC4FE491E150E4
:10B81000F0E0EE0FFF1FE450FC4F859194914695A8
:10B8200046954695342F3E7020E0820F931F0E946C
:10B83000B60D80E00E940C1481E00E940C14089563
:10B840002F923F924F925F926F927F928F929F9230
:10B85000AF92BF92CF92DF92EF92FF920F931F931E
:10B86000DF93CF93CDB7DEB7A0970FB6F894DEBFC6
:10B870000FBECDBF062F90E0A0E0B0E0BC01CD012F
:10B8800020E839E040E050E00E94317E5B016C012D
:10B89000412C78E0572E612C712C4A0C5B1C6C1CDF
:10B8A0007D1CA60195012058374F4F4F5F4F2987C8
:10B8B0003A874B875C87CA01AA27BB27382F305BA2
:10B8C0003E83D601C5018050974FAF4FBF4F8A834B
:10B8D0009B83AC83BD83CD01AA27BB27E82FE05B08
:10B8E000E98310E086E299E09C01029FC001039F7A
:10B8F000900D129F900D112432E9832E34E0932E87
:10B90000880E991EAC0141505C4F58874F8322240A
:10B9100033249A8B898B88509C4FDC01A05AB74FF7
:10B92000BC8BAB8BFC01E15AF74FFE8BED8B9C017E
:10B930002F59374F388F2F8BAC014E59574F5A8F95
:10B94000498FDC01A25AB74FBC8FAB8F83E994E0DB
:10B95000089FF001099FF00D189FF00D1124FE8F34
:10B96000ED8FF0E12F16310409F4D4C0C301B20108
:10B970000E9483548DE29CE20E94517093014427FF
:10B980005527205B8DE29CE2622F46E00E946670A4
:10B990008DE29CE20E949F6F8DE29CE20E949F6F6D
:10B9A000D4018C938DE29CE20E949F6FF40181830D
:10B9B0008DE29CE20E949F6FD40113968C938DE2DE
:10B9C0009CE20E949F6FF40182838DE29CE20E94C0
:10B9D0009F6FAF81B8858C93F401E080FF240894B9
:10B9E000E11CF11CEE0CFF1C0027F7FC0095102F4A
:10B9F000C601B5010E9483548DE29CE20E94517001
:10BA0000960144275527205B8DE29CE2622F4E2D44
:10BA10000E946670EE249101220F331FC10116E0CF
:10BA2000880F991F1A95E1F7280F391F4D8D5E8DEC
:10BA3000240F351F38A32F8F67C08DE29CE20E9430
:10BA40009F6F8C018DE29CE20E949F6F8E871D8606
:10BA5000A80150708D859E85482B592B6E2D70E066
:10BA6000EF8DF8A1E60FF71FEE0FFF1FEE5EFB4F05
:10BA7000242F217030813C7FCA018270907096958E
:10BA800087958170880F322B382BCA018C73907088
:10BA900096958795969587958F70282F220F220F60
:10BAA000337C322B3083882311F4337C3083EF8D49
:10BAB000F8A1E60FF71FEE0FFF1FDF01AE5EBB4FD1
:10BAC000CA01807C977016E0969587951A95E1F7E4
:10BAD000382F3295330F330F307C2C912F73232B5B
:10BAE0002C9386958695877011962C911197287FB7
:10BAF000282B11962C93ED5EFB4F952F987F80811C
:10BB00008770892B8083E394D4018C918E1508F083
:10BB100094CFD4C069857A858B859C850E94835497
:10BB20008DE29CE20E9451708DE29CE26E8140E8C1
:10BB30000E9466708DE29CE20E949F6FEB89FC89F7
:10BB400080838DE29CE20E949F6FAD89BE898C93B9
:10BB50008DE29CE20E949F6FEF89F88D80838DE2D9
:10BB60009CE20E949F6FA98DBA8D8C938DE29CE21E
:10BB70000E949F6FEB8DFC8D8083893008F088E0F8
:10BB8000AB8DBC8D8C9300E024C08DE29CE20E94C2
:10BB90009F6F202F30E0F901EE0FFF1FE20FF31F20
:10BBA00029893A89E20FF31FE25AF34F282F30E038
:10BBB0002077307054E0359527955A95E1F7277036
:10BBC0002295207F982F90788F70282B292B208307
:10BBD0000F5FAB89BC89EC90E016B8F66A817B8177
:10BBE0008C819D810E9483548DE29CE20E94517061
:10BBF0002E2D30E02F5F3F4F220F331F442737FD9C
:10BC00004095542F8DE29CE26981422F0E9466701C
:10BC1000EE244EC08DE29CE20E949F6F8C018DE26B
:10BC20009CE20E949F6F888B1F861070EF85F889B9
:10BC30000E2B1F2B8E2D90E0AC01440F551F480F8B
:10BC4000591F29893A89420F531FFA01E45AF34FC9
:10BC5000702F7170C8018E739070969587958F7153
:10BC6000880F9801207C3770B6E036952795BA95F5
:10BC7000E1F7622F6295660F660F607C872B862B3B
:10BC8000808326952695812F869586958695FA013F
:10BC9000E35AF34F982F990F990F990F2770292B7B
:10BCA0002083815E8F71803110F027702083E394B0
:10BCB000AB89BC898C918E1508F0ACCF0894211CFF
:10BCC000311CE4E8F0E08E0E9F1E26E030E040E0FC
:10BCD00050E0420E531E641E751E4F8158854F5F03
:10BCE0005F4F58874F8380E890E0A0E0B0E0A80E57
:10BCF000B91ECA1EDB1E91E12916310409F031CEAE
:10BD0000A0960FB6F894DEBF0FBECDBFCF91DF91E6
:10BD10001F910F91FF90EF90DF90CF90BF90AF9069
:10BD20009F908F907F906F905F904F903F902F905B
:10BD300008954F925F926F927F928F929F92AF92EF
:10BD4000BF92CF92DF92EF92FF920F931F93CF9308
:10BD5000DF9381E00E947908909357028093560206
:10BD60008091E002882379F080917C0290917D029D
:10BD7000089749F483E090E090937D0280937C02E1
:10BD800081E08093990180917C0290917D020597DA
:10BD900011F01092340280917C0290917D028430E7
:10BDA000910531F00C9721F01092E50210922B2AA8
:10BDB0008091D52A882379F00E943C736093D72A1A
:10BDC0007093D82A8093D92A9093DA2A81E08093BD
:10BDD000D62A1092D52A8091D62A8823F1F0809114
:10BDE000E0028823D1F00E943C732091D72A309141
:10BDF000D82A4091D92A5091DA2A621B730B840BFE
:10BE0000950B615971408040904038F081E08093FB
:10BE1000D42A1092A8011092D62A80914D0283FF55
:10BE200008C080912B0282FD04C08091A801882364
:10BE300029F48091D32A882309F446C081E08093B5
:10BE4000E002109259011092DD2A1092D32A10922A
:10BE500083021092EA031092E9032C982C9A109214
:10BE60007F0280936C1F1092500210924C0110922E
:10BE70004B0180E090E021E0FC01EB56FD4F108289
:10BE8000FC01E25FFC4F1082FC01E551FD4F208375
:10BE9000FC01E954FD4F1082FC01EA54F54D20836A
:10BEA000FC01E853FD4F208301968131910521F774
:10BEB00080913E2A882311F010923A2A80913F2ADD
:10BEC000882311F010923B2A8091DD2A882341F0CB
:10BED0008091E002882321F01092DD2A1092500216
:10BEE00080914F0283FF08C080912B0282FD04C025
:10BEF0008091A801882341F48091B12A882321F4FC
:10BF00008091D42A8823D9F15F9810921F03109250
:10BF10007F021092E5021092EC031092EB038091E5
:10BF2000B12A882311F0109250028091D42A8823DC
:10BF300011F0109250021092D42A109150021F5FFB
:10BF400010935002113019F01230C9F40FC0109341
:10BF500059011092E00280916D02882381F080E007
:10BF600090E80E944C0D1093800209C01092590174
:10BF700081E08093E002109250021092830280913F
:10BF80002B0282FF36C08091390283FF04C080916A
:10BF9000E6020E944F1F80913B0283FF04C0809104
:10BFA000E6020E947C2180914B0283FF09C08CE055
:10BFB00090E090937D0280937C0281E080939901D0
:10BFC0008091350283FFBAC080917C0290917D02FE
:10BFD000019739F081E090E090937D0280937C029C
:10BFE00004C010927D0210927C0281E0809399013E
:10BFF000A5C080917C0290917D028230910569F408
:10C000008091390283FF02C00E94001D80913B0293
:10C0100083FF1BC00E944A1D18C00397B1F4809192
:10C02000390283FF08C08091E6020E94F3198091D3
:10C03000E6028093851F80913B0283FF06C08091BA
:10C04000E6026091851F0E940C1B8091410283FFD4
:10C0500012C080917C0290917D02039719F083E0D9
:10C0600090E002C082E090E090937D0280937C0299
:10C0700081E08093990180914B0283FF1CC08091E5
:10C080007C0290917D02049719F084E090E002C058
:10C0900083E090E090937D0280937C028091E602A1
:10C0A000803121F481E080932B2A02C010922B2A48
:10C0B00081E0809399018091330283FF26C08091B3
:10C0C00034028F5F80933402813019F08230D1F4D2
:10C0D0000FC080917C0290917D029093E202809348
:10C0E000E10285E090E090937D0280937C020AC09B
:10C0F0008091E1029091E20290937D0280937C0214
:10C100001092340281E08093990180917C02909199
:10C110007D02059711F01092340280917C0290917B
:10C120007D02089711F010926D2A80917C02909107
:10C130007D020797029710F010926D2A80914D02B0
:10C1400083FF1DC080912B0282FF19C08091E00205
:10C150008823A9F488E090E090937D0280937C028C
:10C1600080916D2A8F5F80936D2A833018F081E073
:10C1700080936D2A10926B2A81E0809399018091BF
:10C18000450283FF04C081E08093712A05C084FFCB
:10C1900005C01092712A81E0809399018091490233
:10C1A00083FF04C081E08093702A05C084FF05C02E
:10C1B0001092702A81E08093990120917C02309145
:10C1C0007D02C9010397029768F02730310551F0CD
:10C1D0002930310539F02630310521F02C30310578
:10C1E00009F01EC68091560290915702892B11F4D6
:10C1F0001092550280912D0282FF3EC0809137023D
:10C2000083FF0DC083E090E090937D0280937C02D9
:10C210000E94A70B8093E60281E0809399018091B0
:10C220002F0283FF0CC087E090E090937D02809303
:10C230007C0280E18093E60281E080939901809105
:10C240003F0283FF0CC083E090E090937D028093D7
:10C250007C0280E18093E60281E0809399018091E5
:10C260003D0283FF09C086E090E090937D028093B9
:10C270007C0281E08093990180913D0283FF1CC084
:10C280002091E6022031C1F480912D0282FD14C07C
:10C2900087E090E090937D0280937C028091672AF2
:10C2A0008093F10391E0909399018F5F8093672AC7
:10C2B000823010F01092672A80917C0290917D026A
:10C2C000079711F01092672A80913F0283FF11C0F7
:10C2D00080917C0290917D02079759F41092672A11
:10C2E00083E090E090937D0280937C0281E08093D4
:10C2F00099018091430282FFB8C08091E0028823B7
:10C3000009F4B3C0E090E60220916E1F30E1E3161D
:10C3100009F03FC08091940290E030E0FC01EE0F04
:10C32000FF1FE80FF91F86E299E0A901489F9001DD
:10C33000499F300D589F300D1124E20FF31FE45A2E
:10C34000F34F80818E7F80838091940290E0FC0186
:10C35000EE0FFF1FE80FF91FE20FF31FDF01A45AD2
:10C36000B34F8C918E7F8C93E35AF34F808187700B
:10C3700080839C9111968C911197887F846011968F
:10C380008C931197917098619C9381E08093EF0357
:10C390006CC04E2D50E08A010C571D4FD801EC9116
:10C3A00030E0DA01AA0FBB1FCA0166E0880F991FAF
:10C3B0006A95E1F7A80FB91F83E994E0289FB001BF
:10C3C000299F700D389F700D1124A60FB71F9D0176
:10C3D0002E0F311DF901EE0FFF1FEE5EFB4F808126
:10C3E0008E7F8083F801208130E0A20FB31FAA0F57
:10C3F000BB1FAE5EBB4F8C91837C8C938E2D90E0E7
:10C40000FC01A6E0EE0FFF1FAA95E1F7880F991F28
:10C41000E80FF91FE60FF71FE20FF31FEE0FFF1FE4
:10C42000EE5EFB4F80818F7380838181887F846083
:10C4300081838E2D90E0FC01B6E0EE0FFF1FBA95D0
:10C44000E1F7880F991FE80FF91FE60FF71FE20FBA
:10C45000F31FEE0FFF1FED5EFB4F8081877080831F
:10C460004C58504E81E0DA018C9380912B0282FF70
:10C470000DC08091430283FF09C08091E6028031A4
:10C4800019F00E94471C02C00E94AC1C809131022E
:10C4900082FF41C18091370283FF3DC180912B0211
:10C4A00082FF6EC080916E1F90E026E239E0829F8D
:10C4B0008001839F100D929F100D112408501C4F76
:10C4C000F801F0800E94A70BE091E602F0E0E95746
:10C4D000F04E90819295907F980FD8019C9320E028
:10C4E00030E064E870E046E259E011E080916E1FB0
:10C4F00090E0269FF001279FF00D369FF00D11244C
:10C50000DC01A49FC001A59F900DB49F900D112444
:10C51000E80FF91FEE56FB4FDC01A850BC4F8C9181
:10C520008083F901EC58F04E10832F5F3F4F20318C
:10C530003105E1F6FD01E05AF74F8C9180831093AD
:10C54000EF0380916E02813009F0E2C010E0C6E294
:10C55000D9E080916E1F90E08C9FF0018D9FF00DCF
:10C560009C9FF00D1124E850FC4F4081F41620F4FC
:10C57000812F6F2D0E94A11D1F5F113151F7C8C07F
:10C580008091E60220916E1F8031E9F4022F10E0C5
:10C590000E94A70B26E239E0029FD001039FB00D55
:10C5A000129FB00D1124A85AB34FE091E602F0E0BB
:10C5B000E957F04E90819295907F980F9C9381E07F
:10C5C0008093EF0351C030E090E044E8E42EF12C7A
:10C5D0008E9DF0018F9DF00D9E9DF00D1124C6E201
:10C5E000D9E02C9F80012D9F100D3C9F100D112430
:10C5F000E00FF11FEE56FB4FD0800E94A70B509129
:10C60000E602A52FB0E0AE9D9001AF9D300DBE9D1E
:10C61000300D1124020F131F0E561B4FFD01E95759
:10C62000F04E90819295907F980FF8019083AC58CE
:10C63000B04E81E08C9380916E028130A9F480919C
:10C640006E1F90E08C9FF0018D9FF00D9C9FF00D70
:10C650001124E20FF31FEE56FB4F4081D41620F455
:10C66000852F6D2D0E94A11D80916E1F90E026E206
:10C6700039E0829FF001839FF00D929FF00D11240D
:10C68000E850FC4F108220E030E064E870E046E2C1
:10C6900059E080916E1F90E0269FF001279FF00DDA
:10C6A000369FF00D1124DC01A49FC001A59F900DC1
:10C6B000B49F900D1124E80FF91FEE56FB4FE08157
:10C6C000DC01A850BC4F8C918E1718F4EC9320938A
:10C6D000861F2F5F3F4F20313105D9F680916E1FA5
:10C6E00090E026E239E0829FF001839FF00D929F57
:10C6F000F00D1124E850FC4FE05AF74F9081E056BE
:10C70000F8408081891720F4908380E18093861F10
:10C7100081E08093990180912B0282FF5AC0809121
:10C720002D0283FF56C04091E6024E3009F451C0FD
:10C730004F3009F44EC0403109F44BC080916E1F58
:10C7400090E026E239E0829FF001839FF00D929FF6
:10C75000F00D1124E850FC4FE40FF11D8781882370
:10C7600069F1178240E050E063E974E020916E1FA8
:10C7700030E08091E60290E0FC0106E0EE0FFF1F42
:10C780000A95E1F7880F991FE80FF91F269FC0014E
:10C79000279F900D369F900D1124E80FF91FE40F8D
:10C7A000F51FEE0FFF1FEE5EFB4F808182608083DE
:10C7B0004F5F5F4F40345105C9F602C081E0878367
:10C7C00081E080939901E091E602F0E0EC58F04EB0
:10C7D000808380917C0290917D028330910539F0B5
:10C7E0008730910521F08930910509F050C1809181
:10C7F000370284FF04C0109255021092F72A8091EC
:10C80000310282FD0DC380912D0282FD09C380910A
:10C810002B0282FD15C080917C0290917D020397CE
:10C8200079F48091E60220915602309157028031CE
:10C8300021F4C9010E94150A03C0C9010E9404091C
:10C840008091370283FF98C080917C0290917D0295
:10C850008930910519F0079709F08EC00E94A70B47
:10C86000E091E602F0E0E957F04E90819295907FDA
:10C87000980F9093820280912B0282FF7AC0809160
:10C880007C0290917D02099709F073C040E050E06E
:10C8900003E914E0C6E2D9E0809156029091570274
:10C8A000042E02C0969587950A94E2F780FF5BC03C
:10C8B0006091E60220916E1F6031E1F4822F90E0DA
:10C8C000FA01EE0FFF1FE40FF51F9C012C9FC00122
:10C8D0002D9F900D3C9F900D1124E80FF91FE45AF5
:10C8E000F34F90E0808180FF91E080818E7F892BE3
:10C8F000808339C030E0862F90E0DC01F6E0AA0F9B
:10C90000BB1FFA95E1F7880F991FA80FB91FC9013E
:10C91000809F9001819F300D909F300D1124A20FB8
:10C92000B31FA40FB51FAA0FBB1FAE5EBB4F70E0B5
:10C93000862F90E0FC0166E0EE0FFF1F6A95E1F79D
:10C94000880F991FE80FF91FE20FF31FE40FF51F7F
:10C95000EE0FFF1FEE5EFB4F808180FF71E08C9138
:10C960008E7F872B8C934F5F5F4F4031510509F0CD
:10C9700093CF81E08093990180917C0290917D0218
:10C980008930910541F0079709F062C08091E60275
:10C99000803109F05DC00E94C30B082F0E94A70BD5
:10C9A00010E0081B11090130110509F060C58091E4
:10C9B000F72A882309F05BC520916E1F30E0809133
:10C9C000820290E0FC01EE0FFF1FE80FF91F86E2E4
:10C9D00099E0DC012A9FC0012B9F900D3A9F900D9A
:10C9E0001124E80FF91F22C00E94C30B682F809109
:10C9F0006E1F90E026E239E0829FA001839F500DD8
:10CA0000929F500D1124FA01E85AF34F8081681764
:10CA1000F9F48091F72A8823D9F4862F90E0FC015D
:10CA2000EE0FFF1FE80FF91FE40FF51FE25AF34F57
:10CA300090E0808187FF91E0979599279795808175
:10CA40008F77892B808381E08093F72A80939901E7
:10CA500080912B0282FFE4C18091370283FFE0C105
:10CA600089E090E090937D0280937C020E94A70B66
:10CA7000E091E602F0E0E957F04E90819295907FC8
:10CA8000980F9093820281E080939901C9C184300C
:10CA9000910509F042C18091E002882361F0809104
:10CAA0002F0283FF08C090E08091E502882309F4FB
:10CAB00091E09093E5028091430282FF4EC0A091E5
:10CAC000E60220916E1FA031F1F48091940290E073
:10CAD00030E0FC01EE0FFF1FE80FF91F86E299E03E
:10CAE000AC01249FC001259F900D349F900D11240F
:10CAF000E80FF91FE45AF34F80818E7F808381E035
:10CB00008093EF032AC0B0E0FD01EC57FD4F408158
:10CB100030E0FD01EE0FFF1FCD0166E0880F991F89
:10CB20006A95E1F7E80FF91F83E994E0BC01269FBD
:10CB3000C001279F900D369F900D1124E80FF91F1B
:10CB4000E40FF11DEE0FFF1FEE5EFB4F80818E7F25
:10CB50008083AC58B04E81E08C938091310282FD8D
:10CB60000AC080912D0282FD06C080912B2A882365
:10CB700089F00E941A1220E030E044E8442E512C43
:10CB800096E2692E99E0792E83E9882E84E0982E2A
:10CB900001E064C0C0E0D0E001E0E02EF12C809123
:10CBA0005602909157020C2E02C0969587950A94D2
:10CBB000E2F7282F2170FE01EE0FFF1FE55FFD4F0A
:10CBC00090819E7F922B9083892F86958170281764
:10CBD00099F192FD31C0213079F587010C2E02C008
:10CBE000000F111F0A94E2F7C8010E949F35C80187
:10CBF0000E944C0D80ED97E00E94A37380E090E0CE
:10CC00000E944C0D8091E0028823B1F08091E502F2
:10CC1000813091F4FE01EA55FD4F8081FE01B6E0BE
:10CC2000EE0FFF1FBA95E1F7E80FF11DEE0FFF1FA2
:10CC3000E755F04EF182E082FE01EE0FFF1FE55F47
:10CC4000FD4F8081982F9170990F8D7F892B808364
:10CC50002196C031D10509F0A2CF8DCFF901EB5655
:10CC6000FD4F8081882309F051C010E0249D5001C0
:10CC7000259DB00C349DB00C1124790166E0EE0CBA
:10CC8000FF1C6A95E1F7B901660F771F6E0D7F1DD6
:10CC900044E7C42E4FE1D42EC20ED31E25C0412F2F
:10CCA00050E0D701A40FB51FAA0FBB1FA755B04E68
:10CCB0008D919C911197892BB1F0C89DF001C99D70
:10CCC000F00DD89DF00D1124E60FF71FE40FF51FAE
:10CCD000EE0FFF1FEE5EFB4F808183608083F601C5
:10CCE00000831D921C921F5F80916E1FC82FD0E0A1
:10CCF000C69DF001C79DF00DD69DF00D1124EA0DE3
:10CD0000FB1DEE56FB4F8081181748F22F5F3F4FF7
:10CD10002031310509F0A2CF83C00C9709F080C003
:10CD200080915602909157029093E02A8093DF2AD7
:10CD30008091E002882309F473C080912F0283FF61
:10CD400008C090E08091E502882309F491E0909377
:10CD5000E5028091E502882309F462C0A0E0B0E01A
:10CD600003E914E0FF24F39457E08091DF2A9091C7
:10CD7000E02A0A2E02C0969587950A94E2F780FF72
:10CD80004AC0ED01CC57DD4F488120916E1F30E045
:10CD9000BD01660F771FCD01E6E0880F991FEA9568
:10CDA000E1F7680F791F209FC001219F900D309FF0
:10CDB000900D1124680F791FFB01E40FF11DEE0F98
:10CDC000FF1FEE5EFB4F8081816080839091DE2AA1
:10CDD000992391F08881FB01E80FF11DEE0FFF1FF1
:10CDE000ED5EFB4F252F291B922F990F990F990F5D
:10CDF00080818770892B0AC08881FB01E80FF11DB3
:10CE0000EE0FFF1FED5EFB4F808187708083FD0179
:10CE1000EC58F04EF0821196A031B10509F0A5CF83
:10CE200080917C0290917D02029709F01AC1809155
:10CE30002D0282FF11C08091370283FF0DC083E075
:10CE400090E090937D0280937C020E94A70B8093D8
:10CE5000E60281E0809399018091310282FF54C003
:10CE60008091370283FF50C000916E1F10E00E9436
:10CE7000A70B26E239E0029FD001039FB00D129F5D
:10CE8000B00D1124A850BC4FE091E602F0E0E95744
:10CE9000F04E90819295907F980F9C9320E030E027
:10CEA000C4E8D0E066E279E041E080916E1F90E056
:10CEB0002C9FF0012D9FF00D3C9FF00D1124DC0103
:10CEC000A69FC001A79F900DB69F900D1124E80F5B
:10CED000F91FEE56FB4FDC01A850BC4F8C918083AC
:10CEE000E091E602F0E0EC58F04E40832F5F3F4FB8
:10CEF00020313105D1F6FD01E05AF74F8C91808346
:10CF00004093EF03409399018091310283FF04C065
:10CF100081E080936E2A05C084FF05C010926E2ABE
:10CF200081E0809399018091430283FF0CC080913E
:10CF3000370282FF08C09091E8028091EA029817B8
:10CF400011F40E94951D8091370284FF06C08091E4
:10CF5000310282FD02C010925502809156029091DA
:10CF60005702892B09F459C08091310282FD55C0C6
:10CF70008091350282FF18C00E94A70B873010F005
:10CF800087E002C00E94A70B8093E7028091E7022E
:10CF90008295807F2091E802922F9F70890F809365
:10CFA000EA022817B9F539C080912D0282FD35C0FB
:10CFB0000E94C30B8823B9F00E94C30B182F0E9454
:10CFC000A70B181B10936A1F0E94A70B9091E702F2
:10CFD0009295907F980F90936B1F9093EA0281E057
:10CFE000809355020FC080915502882369F40E94F6
:10CFF000A70B9091E7029295907F980F9093EA0289
:10D0000010926A1F10926C1F9091E8028091EA02C0
:10D01000981719F081E080936F1F80910D0388238A
:10D0200001F180916A1F8823E1F010920D03809135
:10D030006C1F90916B1F890F8093EA029091E80218
:10D04000981719F081E080936F1F80916C1F909169
:10D050006A1F8F5F80936C1F8150891710F01092A8
:10D060006C1F80917C0290917D02019711F40E94C7
:10D070004A2580917C0290917D02892B09F06EC037
:10D080000E944A258091292A8823C1F48091E002D8
:10D090008823A1F410922E2810922D2890913428E4
:10D0A0009093EA028091E802891719F081E0809359
:10D0B0006F1F81E0809399018093292A80910D034D
:10D0C000882309F443C0209131283091322821155A
:10D0D0003105E1F110920D0380912A2A882391F005
:10D0E00010922E2810922D28909134289093EA02C5
:10D0F0008091E802891719F081E080936F1F1092E8
:10D100002A2A21C080912D2890912E280196909353
:10D110002E2880932D2801978217930720F01092D4
:10D120002E2810922D28E0912D28F0912E28E55DD3
:10D13000F74D91859093EA028091E802891719F0E2
:10D1400081E080936F1F81E0809399018091430279
:10D1500083FF06C081E080932A2A02C01092292A08
:10D1600080917C0290917D020897D1F480916D2A84
:10D170008230B1F480916B2A833091F48091370230
:10D1800083FF07C00E94A70B8093E90281E0809390
:10D1900099018091E9028B3018F08BE08093E902CD
:10D1A0008091272A882349F080912C280E941C5ABC
:10D1B0001092272A81E08093990180916F1F882324
:10D1C000B1F110926F1F81E080939901E4E7FFE1D4
:10D1D0001192BFE1E438FB07D9F71092711F10924A
:10D1E000EF0380912B0282FF0DC08091EA026091D3
:10D1F0006E1F0E94205C8091EA028093E8020E94E8
:10D20000842411C060E080916E1F882309F461E0DE
:10D210008091EA020E94205C8091EA028093E802F9
:10D2200081E08093701F8091E8020E944F378091C7
:10D23000701F882381F08091E002882361F41092AE
:10D24000701F90E080916E1F882309F491E0909305
:10D250006E1F0E94842480912F0283FF16C080914C
:10D260002D0282FD12C0C4E7DFE110E0888188232F
:10D2700041F018828091E802612F0E9443560E947B
:10D2800038421F5F2196103189F78091EF03882380
:10D29000B9F080912F0283FF13C080912D0282FD8F
:10D2A0000FC080917C0290917D02049749F010920A
:10D2B000EF038091E80260E10E9443560E943842E9
:10D2C00080915B2A8823A1F080912F0283FF10C0F8
:10D2D00080912D0282FD0CC080917C0290917D0294
:10D2E000049731F010925B2A8091E8020E94B836D0
:10D2F0008091282A8823A1F080912F0283FF10C0FB
:10D3000080912D0282FD0CC080917C0290917D0263
:10D31000049731F01092282A80912C280E94AA5458
:10D3200080912F0284FF03C081E080939901809156
:10D330007C0290917D02059709F09FC080912D029B
:10D3400082FD5FC080915602909157020E94F20ABE
:10D3500080912B0282FF35C08091330283FD04C08F
:10D360008091430283FF07C010922A281092292837
:10D370001092422A15C080913F0283FF22C0809103
:10D38000721F882381F080912803882349F410922A
:10D390002A2810922928109228031092721F0EC07A
:10D3A000109228030BC01092280381E08093721F13
:10D3B0008FEF9FEF90932A288093292881E0809314
:10D3C000990180913D0283FF0BC090E08091422A39
:10D3D000882309F491E09093422A81E08093990197
:10D3E00080913F0283FF1EC080912B0282FD1AC0F4
:10D3F00090E080912803882309F491E0909328031A
:10D400000EC08091370283FF0DC083E090E09093BF
:10D410007D0280937C020E94A70B8093E60281E04C
:10D420008093990180910D03882339F180916A1FBF
:10D43000882319F110920D0380916C1F90916B1F3E
:10D44000890F8093EA029091E802981719F081E021
:10D4500080936F1F80916C1F90916A1F8F5F8093E4
:10D460006C1F8150891748F010926C1F06C00E94F3
:10D47000A70B882309F0ECCAB7CADF91CF911F919F
:10D480000F91FF90EF90DF90CF90BF90AF909F9063
:10D490008F907F906F905F904F9008958091E00201
:10D4A000882311F41092B12A0E949D340E94A42571
:10D4B0000E9476150E94BE550E94995E0E945744B4
:10D4C000089580ED84B982EF8AB98CEF81B989E043
:10D4D00061E00E94177412B85F980E944F6D8FEF41
:10D4E0000E942D6D8DE29CE20E946A7008951F9249
:10D4F0000F920FB60F920BB60F9211240F931F933A
:10D500002F933F934F935F936F937F938F939F934B
:10D51000AF93BF93EF93FF9380917E02837090E06F
:10D520008130910541F08230910509F46EC0892B5C
:10D5300009F0DDC017C086E09FE20E9465761816EC
:10D5400019060CF0D4C086E09FE20E949676883FD0
:10D5500008F4CDC0883F49F40E94A8390E94A83938
:10D560000E94A8390E94A839C2C08A3F09F046C06B
:10D5700081E08093E002109259011092DD2A10920E
:10D5800083021092EA031092E90380936C1F2C9897
:10D590002C9A10927F0210924C0110924B01109223
:10D5A000500280E090E021E0FC01EB56FD4F10823C
:10D5B000FC01E25FFC4F1082FC01E551FD4F20832E
:10D5C000FC01E954FD4F1082FC01E853FD4F20831C
:10D5D000FC01EA54F54D208301968131910521F734
:10D5E00080913E2A882311F010923A2A80913F2A96
:10D5F000882309F47CC010923B2A79C08C3F09F043
:10D6000076C081E08093B12A72C08091D22A8823AB
:10D6100089F11092CC2A1092CB2A1092D22A8091B2
:10D620008302843520F4809183028C3010F41092B0
:10D630008302809183028C3038F08091830284329F
:10D6400018F488E18093830280918302843238F059
:10D65000809183028C3318F480E38093830280915D
:10D6600083028C3338F080918302843518F488E487
:10D67000809383020091CB2A1091CC2A60919F0164
:10D680007091A0018091A1019091A20128E130E068
:10D6900040E050E00E94837E0217130720F01092B2
:10D6A000CC2A1092CB2A8091CB2A9091CC2A892B1C
:10D6B00011F40E94A8398091C72A9091C82AA0919C
:10D6C000C92AB091CA2A0196A11DB11D8093C72A0B
:10D6D0009093C82AA093C92AB093CA2A8091CB2AD2
:10D6E0009091CC2A01969093CC2A8093CB2AFF91DB
:10D6F000EF91BF91AF919F918F917F916F915F91CA
:10D700004F913F912F911F910F910F900BBE0F9052
:10D710000FBE0F901F901895FF920F931F9386E0F6
:10D720009FE242E15AE760E070E00E94DF750E94EC
:10D73000616AECE0F2E01082329682E0EC32F807A7
:10D74000D1F7109250021092480210923E021092AD
:10D7500034028DE29CE267E570E00E948C6F8DE2FE
:10D760009CE26FEF0E940E708DE29CE26DEF0E94D2
:10D770000E708DE29CE20E9451708DE29CE267E5A2
:10D7800070E043E050E00E9462708DE29CE20E94F3
:10D790009F6F082F8DE29CE20E949F6FF82E8DE212
:10D7A0009CE20E949F6F10E00F0D111D080F111DCC
:10D7B0000430110531F00E9475420E94AB580E945E
:10D7C00085360E94930E8091B32A843051F40E94D2
:10D7D00053428FE70E94EB0D80E094E00E94B60D6B
:10D7E000F8CF8091B22A833041F40E9475420E94A2
:10D7F000AB580E9485360E943E370E94EC378091DC
:10D80000B42A803F51F490E08091B52A882309F42E
:10D8100091E09093B52A0E9446370E949D5B8091CB
:10D820006800816080936800D89A80916B00836063
:10D8300080936B0080E060916E1F0E94205C0E94CC
:10D84000842480E090E00E944C0D0E94001D80E046
:10D850000E941C5A1092B1008091B1008093B000D8
:10D860008091B00082608093B0008091B1008260AE
:10D870008093B1008FE78093B30080917000826045
:10D88000809370000E94E437789481EE9AE260E021
:10D8900040E05AE00E945C6E81EE9AE261E048E06E
:10D8A0005AE00E945C6E81EE9AE262E040E15AE04A
:10D8B0000E945C6E81EE9AE263E048E15AE00E94C9
:10D8C0005C6E81EE9AE264E040E25AE00E945C6E97
:10D8D00081EE9AE265E048E25AE00E945C6E81EED9
:10D8E0009AE260E142E020E00E948C6E81EE9AE2D2
:10D8F00060E00E941C6E81EE9AE261E00E941C6E64
:10D9000081EE9AE262E00E941C6E81EE9AE264E08F
:10D9100040E00E94266E81EE9AE264EC0E94FF775E
:10D9200081EE9AE26EED0E94FF7781EE9AE267ED5A
:10D930000E94FF7781EE9AE261ED0E94FF7781EE0F
:10D940009AE269E040E00E94266E81EE9AE26CEB7A
:10D950000E94FF7781EE9AE260EB0E94FF7781EEF2
:10D960009AE269EB0E94FF7781EE9AE26FEB0E94E8
:10D97000FF7781EE9AE26BEB0E94FF7781EE9AE2ED
:10D9800060EB0E94FF7781EE9AE260E041E00E9446
:10D99000266E81EE9AE263E00E941C6E81EE9AE2AE
:10D9A00064E00E941C6E81EE9AE265E00E941C6EAB
:10D9B00081EE9AE266E041E00E94266E81EE9AE2F4
:10D9C00060E77AE00E94DC7760ED77E080E090E04D
:10D9D0000E944A7381EE9AE260E040E35AE00E94BE
:10D9E0005C6E81EE9AE261E048E35AE00E945C6E70
:10D9F00081EE9AE262E040E45AE00E945C6E81EEC1
:10DA00009AE263E048E45AE00E945C6E81EE9AE29A
:10DA100064E040E55AE00E945C6E81EE9AE265E0C7
:10DA200048E55AE00E945C6E81EE9AE266E040E6CC
:10DA30005AE00E945C6E81EE9AE267E048E65AE0A6
:10DA40000E945C6E81EE9AE260E142E020E00E947A
:10DA50008C6E1F910F91FF900895982F8091202B2D
:10DA60008230E0F42FB7F894913029F0913060F0D3
:10DA7000923029F402C092E008C094E006C082E02F
:10DA80008093202B2FBF089591E081E08093202B7D
:10DA90008091212B892B8093212B2FBF089584E027
:10DAA00061E00E947B7484E061E00E9417748CB591
:10DAB00080618CBD8CB580648CBD87E061E00E9484
:10DAC000177485E061E00E94177408950F931F9307
:10DAD0008C01FC01868160E00E947B7481E090E013
:10DAE0000E94A373F801868161E00E947B7481E04B
:10DAF00090E00E94A373F801868160E00E947B742D
:10DB000084E690E00E94A3731F910F910895CF9235
:10DB1000DF92EF92FF920F931F93CF93DF93D82E54
:10DB2000C92E282F392FC9018C01C0E0D0E0E62E84
:10DB3000FF24F801878161E00E941774B7010C2E61
:10DB400002C0759567950A94E2F76170F8018781C4
:10DB50000E947B7421960F5F1F4FC830D10549F793
:10DB60008D2D9C2D0E94666DDF91CF911F910F919D
:10DB7000FF90EF90DF90CF900895CF92DF92EF92D9
:10DB8000FF920F931F93CF93DF93D82EC92E282F88
:10DB9000392FC9018C01C0E0D0E0E62EFF24F80146
:10DBA000878161E00E941774B7010C2E02C0759541
:10DBB00067950A94E2F76170F80187810E947B748F
:10DBC00021960F5F1F4FC430D10549F78D2D9C2D35
:10DBD0000E94666DDF91CF911F910F91FF90EF90A2
:10DBE000DF90CF9008951F93CF93DF93EC01162F12
:10DBF0008C81642F0E947B748D818F3F19F060E0CF
:10DC00000E947B748F8584FF05C0CE01612F0E9426
:10DC1000876D0EC0612F70E084E0759567958A95D9
:10DC2000E1F7CE010E94BD6DCE01612F0E94BD6D56
:10DC3000DF91CF911F91089541E00E94F36D81E043
:10DC400090E0089540E00E94F36D0895DF93CF9334
:10DC5000CDB7DEB728970FB6F894DEBF0FBECDBFA5
:10DC60009C01FE013196A9ECB1E088E00D90019293
:10DC70008150E1F7F9018389481708F040E0E42F6B
:10DC8000F0E0EE0FFF1FEC0FFD1F8181680F606851
:10DC9000C9010E94226E28960FB6F894DEBF0FBE0F
:10DCA000CDBFCF91DF91089562E00E94226E80ED9A
:10DCB00097E00E94A3730895EF92FF920F931F9332
:10DCC000CF93DF938C017A0170E06770707023E06E
:10DCD000660F771F2A95E1F760640E94226EC0E00C
:10DCE000D0E0F701EC0FFD1F4491F801A081B18154
:10DCF0002D913C91C801642FF90109952196C830F6
:10DD0000D10579F7C8010E94546EDF91CF911F9120
:10DD10000F91FF90EF900895CF93DF93EC01423085
:10DD200018F08F8588608F874B8B1C8A222329F0FF
:10DD3000413019F48F8584608F8780E593EC0E94D1
:10DD4000A3738C8160E00E947B748E8160E00E94EE
:10DD50007B748D818F3F19F060E00E947B74CE014F
:10DD600063E00E94BD6D88E893E10E94A373CE0139
:10DD700068E00E94BD6D88E893E10E94A373CE0124
:10DD800062E00E94BD6D88E893E10E94A373CE011A
:10DD900062E00E94BD6D88E893E10E94A373CE010A
:10DDA00068E00E94BD6D88E893E10E94A373CE01F4
:10DDB00068E00E94226E88E893E10E94A373CE017E
:10DDC00061E00E94226E88E893E10E94A373CE0175
:10DDD00066E00E94226E88E893E10E94A373CE0160
:10DDE00062E00E94226E88E893E10E94A373CE0154
:10DDF0006CE00E94226E88E893E10E94A373DF9199
:10DE0000CF9108956F927F928F92AF92CF92EF92BF
:10DE10000F931F93DF93CF93CDB7DEB73C01162F3F
:10DE2000842FF301448325830683E782C086A1867D
:10DE300082869D8593879E8594879F8595879889FF
:10DE4000968761E00E941774F30185818F3F19F076
:10DE500061E00E941774F301868161E00E941774EB
:10DE6000112319F0F301178603C080E1F3018787BE
:10DE7000C30160E141E020E00E948C6ECF91DF9110
:10DE80001F910F91EF90CF90AF908F907F906F90F8
:10DE900008958F92AF92CF92EF920F931F93CF93EB
:10DEA000DF93DC01362F542F722F102FAE2C8C2CC9
:10DEB00013961C921E92129785EC91E011969C93FA
:10DEC0008E9300D000D0EDB7FEB73196CDB7DEB758
:10DED0001982118212821382CD0161E0432F2FEF4C
:10DEE000052FE72EC12E0E94026F0F900F900F900A
:10DEF0000F90DF91CF911F910F91EF90CF90AF9046
:10DF00008F90089581E080932C2C6093A72B109222
:10DF10002A2C10922B2C089581E080932C2C609356
:10DF2000A72B10922A2C10922B2C08952091A62B0F
:10DF300030E08091A52B281B3109C901089540913B
:10DF4000A52B8091A62B481718F02FEF3FEF0AC0A2
:10DF5000E42FF0E0ED5DF44D8081282F30E04F5F3D
:10DF60004093A52BC9010895E091A52B8091A62B84
:10DF7000E81718F0EFEFFFEF06C0F0E0ED5DF44DAD
:10DF80008081E82FF0E0CF01089508951092302CA1
:10DF900010922F2C88EE93E0A0E0B0E08093312C1B
:10DFA0009093322CA093332CB093342C85ED91E0D8
:10DFB00090932E2C80932D2C0895CF92DF92EF9288
:10DFC000FF920F931F93CF93DF937C016B018A0124
:10DFD00080912C2C8823A1F0C0E0D0E00DC0D701A7
:10DFE000ED91FC91D601AC0FBD1F0190F081E02DA9
:10DFF000C7016C9109952196C017D10780F304C021
:10E00000CB01642F0E941371C801DF91CF911F9142
:10E010000F91FF90EF90DF90CF900895DF93CF9313
:10E020000F92CDB7DEB7FC01698380912C2C882339
:10E03000C9F080912B2C823838F081E090E09383F6
:10E04000828320E030E015C080912A2CE82FF0E098
:10E05000E855F44D998190838F5F80932A2C8093AB
:10E060002B2C05C0CE01019661E00E94137121E0C6
:10E0700030E0C9010F90CF91DF9108950F93062FE3
:10E080008091A72B68EA7BE240912B2C21E00E9433
:10E09000BE7010922A2C10922B2C10922C2C0F91C7
:10E0A000089561E00E943E700895433808F042E808
:10E0B000862F63E27BE20E9475701092A52B8093FD
:10E0C000A62B089521E00E945570089521E00E943A
:10E0D000557008951092A52B1092A62B10922A2C01
:10E0E00010922B2C0E94C3720895382F433810F0E1
:10E0F00040E042C08091392C8823E1F791E0909371
:10E10000392C20933B2C8FEF8093CC2D1092C32C75
:10E1100041504093C42C4F5F90933A2C80913A2CFD
:10E12000330F832B80933A2C80913C2C813041F427
:10E1300010923C2C80913A2C8093BB0085EC01C05E
:10E1400085EE8093BC008091392C8130E1F3809181
:10E15000C32C841710F44091C32C20E030E00AC097
:10E16000FB01E20FF31FD901AF5BB34D8C918083AC
:10E170002F5F3F4F2417A0F3842F08950F931F9311
:10E18000582F122F433810F081E04AC08091392C6B
:10E190008823E1F782E08093392C00933B2C8FEFAA
:10E1A0008093CC2D1092C32C4093C42CA1E4BCE2EC
:10E1B000FB0102C081918D938E2F861B8417D0F3B3
:10E1C00010923A2C80913A2C550F852B80933A2C43
:10E1D00080913C2C813041F410923C2C80913A2C5F
:10E1E0008093BB0085EC01C085EE8093BC001123B9
:10E1F00021F08091392C8230E1F38091CC2D8F3F3A
:10E2000011F480E00DC08091CC2D803211F482E0B9
:10E2100007C08091CC2D803311F084E001C083E0F1
:10E220001F910F910895482F633810F081E00895F1
:10E230008091392C843011F082E008956093482D4C
:10E24000A5ECBCE2842F9C01F90102C081918D9361
:10E250008E2F841B8617D0F380E008951F920F92B3
:10E260000FB60F920BB60F9211242F933F934F933B
:10E270005F936F937F938F939F93AF93BF93EF932E
:10E28000FF938091B90090E0887F9070803691056F
:10E2900009F4F2C081369105CCF58832910509F474
:10E2A0007BC089329105B4F48031910509F46FC0C7
:10E2B000813191053CF4009709F447C1089709F0B2
:10E2C0004FC165C08831910509F466C0809709F097
:10E2D00047C182C08034910509F4A4C081349105FE
:10E2E00044F48033910509F482C0C89709F038C11D
:10E2F00089C08035910509F489C08835910509F4F4
:10E3000096C08834910509F02BC1AEC088399105BB
:10E3100009F413C189399105ECF48837910509F4A2
:10E32000ABC0893791054CF48836910509F4A4C037
:10E330008037910509F014C19FC08838910509F410
:10E34000FCC08039910509F49DC08038910509F021
:10E3500007C198C0803B910509F4C6C0813B910577
:10E360004CF4803A910509F49FC0883A910509F070
:10E37000F7C0BAC0803C910509F4E3C0883C910520
:10E3800009F4DFC0883B910509F0EAC0C2C0809162
:10E390003A2C8093BB00CFC09091C32C8091C42CA9
:10E3A000981768F49091C32CE92FF0E0EF5BF34DE0
:10E3B00080818093BB009F5F9093C32CBCC08091F1
:10E3C0003B2C882309F44BC085ED8093BC008091E1
:10E3D000BC0084FDFCCFC2C080E28093CC2D85EDD3
:10E3E0008093BC008091BC0084FDFCCFB7C080E36B
:10E3F0008093CC2D85ED8093BC008091BC0084FD82
:10E40000FCCFACC088E38093CC2D9BC08091C32C03
:10E410009091BB00E82FF0E0EF5BF34D90838F5FAE
:10E420008093C32C9091C32C8091C42C82C0809186
:10E43000C32C9091BB00E82FF0E0EF5BF34D90838D
:10E440008F5F8093C32C80913B2C882341F085ED16
:10E450008093BC008091BC0084FDFCCF7FC081E034
:10E4600080933C2C84EA6EC085ED8093BC00809143
:10E47000BC0084FDFCCF72C083E08093392C1092E5
:10E48000CB2D59C08091CB2D823808F056C0809199
:10E49000CB2D9091BB00E82FF0E0E75BF24D90832D
:10E4A0008F5F8093CB2D47C08091CB2D823830F485
:10E4B000E091CB2DF0E0E75BF24D108285ED80938B
:10E4C000BC008091BC0084FDFCCF1092392C60917F
:10E4D000CB2DE0913F2CF091402C89E49DE270E03F
:10E4E00009951092CB2D2DC084E08093392C109289
:10E4F000472D1092482DE0913D2CF0913E2C09952E
:10E500008091482D882329F481E08093482D109232
:10E51000C52C9091472DE92FF0E0EB53F34D80810E
:10E520008093BB009F5F9093472D9091472D8091E2
:10E53000482D981710F485EC01C085E88093BC0045
:10E540000FC085EC8093BC0009C01092CC2D85EDE6
:10E550008093BC008091BC0084FDFCCF1092392CCC
:10E56000FF91EF91BF91AF919F918F917F916F91AB
:10E570005F914F913F912F910F900BBE0F900FBE67
:10E580000F901F9018951092392C81E080933B2CAE
:10E5900010923C2C81E161E00E947B7480E161E09B
:10E5A0000E947B74E9EBF0E080818E7F8083808124
:10E5B0008D7F808388E48093B80085E48093BC00DD
:10E5C0000895F999FECF72BD61BDF89A80B508959E
:10E5D000F999FECF1FBA72BD61BD40BD0FB6F89468
:10E5E000FA9AF99A0FBE08951F920F920FB60F92E2
:10E5F00011242F933F938F939F93AF93BF93809159
:10E60000D22D9091D32DA091D42DB091D52D3091B4
:10E61000D62D0196A11DB11D232F2D5F2D3720F082
:10E620002D570196A11DB11D2093D62D8093D22D7B
:10E630009093D32DA093D42DB093D52D8091CE2D32
:10E640009091CF2DA091D02DB091D12D0196A11DEB
:10E65000B11D8093CE2D9093CF2DA093D02DB0934C
:10E66000D12DBF91AF919F918F913F912F910F909D
:10E670000FBE0F901F9018958FB7F8942091D22D50
:10E680003091D32D4091D42D5091D52D8FBFB9010C
:10E69000CA0108959B01AC017FB7F8948091CE2DFB
:10E6A0009091CF2DA091D02DB091D12D66B5A89B82
:10E6B00005C06F3F19F00196A11DB11D7FBFBA2F94
:10E6C000A92F982F8827860F911DA11DB11D62E0EB
:10E6D000880F991FAA1FBB1F6A95D1F7BC012DC0D7
:10E6E000FFB7F8948091CE2D9091CF2DA091D02D91
:10E6F000B091D12DE6B5A89B05C0EF3F19F001966A
:10E70000A11DB11DFFBFBA2FA92F982F88278E0FEB
:10E71000911DA11DB11DE2E0880F991FAA1FBB1F0B
:10E72000EA95D1F7861B970B885E9340C8F221507B
:10E7300030404040504068517C4F21153105410523
:10E74000510571F60895019739F0880F991F880FC8
:10E75000991F02970197F1F70895789484B5826024
:10E7600084BD84B5816084BD85B5826085BD85B575
:10E77000816085BDEEE6F0E0808181608083E1E824
:10E78000F0E010828081826080838081816080835C
:10E79000E0E8F0E0808181608083E1EBF0E080815F
:10E7A00084608083E0EBF0E0808181608083E1E938
:10E7B000F0E0808182608083808181608083E0E9F5
:10E7C000F0E0808181608083EAE7F0E0808184600E
:10E7D000808380818260808380818160808380816A
:10E7E000806880831092C1000895982F883108F0C6
:10E7F000985197708091B0018295880F880F807C26
:10E80000892B80937C0080917A00806480937A00C9
:10E8100080917A0086FDFCCF2091780040917900AC
:10E82000942F80E030E0282B392BC9010895482F20
:10E8300050E0CA018B54954FFC0124914B56554F23
:10E84000FA0184918823C1F0E82FF0E0EE0FFF1F5A
:10E85000E958F54FA591B491662341F49FB7F89418
:10E860008C91209582238C939FBF08959FB7F89435
:10E870008C91822B8C939FBF08958430C9F0853092
:10E8800038F48230F1F0833078F4813099F516C095
:10E890008730F9F0883018F4863061F516C088307A
:10E8A000F1F0893039F521C0809180008F7703C065
:10E8B000809180008F7D80938000089584B58F774C
:10E8C00002C084B58F7D84BD08958091B0008F779C
:10E8D00003C08091B0008F7D8093B0000895809137
:10E8E00090008F77809390000895809190008F7DA5
:10E8F000809390000895FF920F931F93F62E482F58
:10E9000050E0CA018B52954FFC012491CA018B54EF
:10E91000954FFC0114914B56554FFA010491002379
:10E92000C9F0222319F0822F0E943D74E02FF0E0FD
:10E93000EE0FFF1FEF57F54FA591B4919FB7F894D5
:10E94000FF2021F48C911095812302C08C91812BA2
:10E950008C939FBF1F910F91FF90089508951F9270
:10E960000F920FB60F920BB60F9211242F933F9375
:10E970004F938F939F93EF93FF934091C600209105
:10E98000172E3091182E2F5F3F4F2F7330708091CC
:10E99000192E90911A2E2817390759F0E091172E49
:10E9A000F091182EE952F24D40833093182E2093A7
:10E9B000172EFF91EF919F918F914F913F912F9142
:10E9C0000F900BBE0F900FBE0F901F9018950895DB
:10E9D0001F920F920FB60F920BB60F9211242F9326
:10E9E0003F934F938F939F93EF93FF934091CE006C
:10E9F00020919F2E3091A02E2F5F3F4F2F733070AC
:10EA00008091A12E9091A22E2817390759F0E091FC
:10EA10009F2EF091A02EE15AF14D40833093A02E0D
:10EA200020939F2EFF91EF919F918F914F913F9156
:10EA30002F910F900BBE0F900FBE0F901F90189547
:10EA4000E091F32EF091F42EE05CFF4F81919191D3
:10EA500020813181821B930B8F739070892B11F071
:10EA60000E94AE74E091122FF091132FE05CFF4FE3
:10EA70008191919120813181821B930B8F739070D2
:10EA8000892B11F00E94E77408951F920F920FB620
:10EA90000F920BB60F9211242F933F934F935F93D6
:10EAA0006F937F938F939F93AF93BF93EF93FF9356
:10EAB00020915B2E30915C2E80915D2E90915E2E88
:10EAC0002817390731F48091C1008F7D8093C100F0
:10EAD00016C0E0915D2EF0915E2EE55EF14D408115
:10EAE00080915D2E90915E2E019660E470E00E9410
:10EAF000707E90935E2E80935D2E4093C600FF91B2
:10EB0000EF91BF91AF919F918F917F916F915F91A5
:10EB10004F913F912F910F900BBE0F900FBE0F9012
:10EB20001F9018951F920F920FB60F920BB60F926F
:10EB300011242F933F934F935F936F937F938F9302
:10EB40009F93AF93BF93EF93FF932091E32E309168
:10EB5000E42E8091E52E9091E62E2817390731F4A6
:10EB60008091C9008F7D8093C90016C0E091E52E89
:10EB7000F091E62EED55F14D40818091E52E90917A
:10EB8000E62E019660E470E00E94707E9093E62E7F
:10EB90008093E52E4093CE00FF91EF91BF91AF910E
:10EBA0009F918F917F916F915F914F913F912F91A5
:10EBB0000F900BBE0F900FBE0F901F901895AF9245
:10EBC000BF92DF92EF92FF920F931F93CF93DF9349
:10EBD000EC017A018B01DD24403081EE580780E0A2
:10EBE000680780E0780711F0DD24D39491E0A92E26
:10EBF000B12CEC89FD89DD2069F0C5010E8C02C0C5
:10EC0000880F991F0A94E2F7808360E079E08DE332
:10EC100090E005C0108260E874E88EE190E0A80101
:10EC200097010E94837E21503040404050405695CD
:10EC300047953795279580E12030380720F0DD2073
:10EC400011F0DD24D6CFE889F9893083EA89FB8980
:10EC50002083EE89FF89408121E030E0C9010A8CE0
:10EC600002C0880F991F0A94E2F7482B4083EE896F
:10EC7000FF894081C9010B8C02C0880F991F0A943B
:10EC8000E2F7482B4083EE89FF894081C9010C8C53
:10EC900002C0880F991F0A94E2F7482B4083EE893F
:10ECA000FF8980810D8C02C0220F331F0A94E2F786
:10ECB000209528232083DF91CF911F910F91FF9002
:10ECC000EF90DF90BF90AF900895DC011C96ED911E
:10ECD000FC911D97E05CFF4F2191319180819181E2
:10ECE000281B390B2F733070C9010895DC011C9665
:10ECF000ED91FC911D97E05CFF4F20813181E05444
:10ED0000F040DF01AE5BBF4F8D919C9111972817AA
:10ED1000390719F42FEF3FEF07C08D919C91E80F51
:10ED2000F91F8081282F30E0C9010895DC011C966D
:10ED3000ED91FC911D97E05CFF4F20813181E05403
:10ED4000F040DF01AE5BBF4F8D919C91119728176A
:10ED5000390719F42FEF3FEF10C08D919C91119757
:10ED6000E80FF91F20818D919C91119701968F7367
:10ED7000907011969C938E9330E0C9010895FC0128
:10ED800086859785DC01A05CBF4FFC01EE5BFF4FE1
:10ED90002D913C9111978081918128173907C1F7F6
:10EDA0000895CF93DF93EC01462FEE85FF85E05C5D
:10EDB000FF4F80819181E054F040019660E470E063
:10EDC0000E94707E9C01DF01AE5BBF4F8D919C91D4
:10EDD000119728173907D1F3E05CFF4F80819181AB
:10EDE000E054F040E80FF91F4083EE85FF85E05CBA
:10EDF000FF4F31832083EE89FF89208181E090E0FD
:10EE00000D8C02C0880F991F0A94E2F7282B2083EB
:10EE100081E090E0DF91CF9108951F931092EA2E48
:10EE20001092E92E28EE33E040E050E02093EB2EE4
:10EE30003093EC2E4093ED2E5093EE2E65EE71E064
:10EE40007093E82E6093E72E87ED9DE29093F42E69
:10EE50008093F32E8BE19EE29093F62E8093F52E15
:10EE600085EC90E09093F82E8093F72E84EC90E060
:10EE70009093FA2E8093F92E80EC90E09093FC2EE4
:10EE80008093FB2E81EC90E09093FE2E8093FD2EDC
:10EE900086EC90E09093002F8093FF2E14E0109367
:10EEA000012FB3E0B093022FA7E0A093032FF5E06A
:10EEB000F093042FE1E0E093052F1092092F1092B8
:10EEC000082F20930A2F30930B2F40930C2F509331
:10EED0000D2F7093072F6093062F8FE59EE290937E
:10EEE000132F8093122F83EA9EE29093152F809325
:10EEF000142F8DEC90E09093172F8093162F8CECAD
:10EF000090E09093192F8093182F88EC90E09093C5
:10EF10001B2F80931A2F89EC90E090931D2F8093E4
:10EF20001C2F8EEC90E090931F2F80931E2F109338
:10EF3000202FB093212FA093222FF093232FE09323
:10EF4000242F1F910895CF93DF930E94AD730E94E9
:10EF50008C6BC0E2D5E70E944E6A2097E1F30E94D5
:10EF60002075F9CFCF92DF92EF92FF920F931F930C
:10EF7000CF93DF937C016B018A01C0E0D0E00FC02A
:10EF8000D6016D916D01D701ED91FC910190F08159
:10EF9000E02DC7010995C80FD91F01501040011578
:10EFA000110571F7CE01DF91CF911F910F91FF9065
:10EFB000EF90DF90CF900895EF92FF920F931F9301
:10EFC000CF93DF937C018B01C0E0D0E0F8010F5FAD
:10EFD0001F4F6491662359F0D701ED91FC91019088
:10EFE000F081E02DC7010995C80FD91FEFCFCE01E1
:10EFF000DF91CF911F910F91FF90EF900895DC0169
:10F00000ED91FC910190F081E02D09950895CF9349
:10F01000DF93DB010D900020E9F71197A61BB70BDA
:10F02000EC01E881F9810280F381E02DAD010995C1
:10F03000DF91CF9108954F925F927F928F929F922E
:10F04000AF92BF92CF92DF92EF92FF920F931F93F6
:10F05000DF93CF93CDB7DEB7A1970FB6F894DEBF9D
:10F060000FBECDBF2C01742ECB01223008F42AE054
:10F0700019A231E2C32ED12CCC0EDD1E822E992492
:10F08000AA24BB24672D752FA50194010E94837EBD
:10F0900079018A01C801B701A50194010E94317E5E
:10F0A000472D461B0894C108D1084A3014F4405D2E
:10F0B00001C0495CF6014083E114F104010511052A
:10F0C00021F07E2C5F2DC801DDCFC201B6010E9468
:10F0D0000778A1960FB6F894DEBF0FBECDBFCF91D3
:10F0E000DF911F910F91FF90EF90DF90CF90BF9035
:10F0F000AF909F908F907F905F904F900895DC012C
:10F100002115310541F4ED91FC910190F081E02D44
:10F11000642F099508950E941B780895EF92FF923D
:10F120000F931F939A017B0100E010E0B801A70143
:10F130000E947F781F910F91FF90EF900895EF92BA
:10F14000FF920F931F939A01E62EFF2400E010E038
:10F15000B801A7010E947F781F910F91FF90EF9057
:10F160000895CF92DF92EF92FF920F931F93CF9368
:10F17000DF93EC016A017B012115310541F4E8813F
:10F18000F9810190F081E02D642F09951FC02A308C
:10F190003105D1F477FF17C0E881F9810190F08142
:10F1A000E02D6DE209958C0144275527BA014C19D1
:10F1B0005D096E097F09CE012AE00E941B78980143
:10F1C000280F391F04C02AE00E941B789C01C90146
:10F1D000DF91CF911F910F91FF90EF90DF90CF9033
:10F1E0000895EF92FF920F931F937B019A010027DE
:10F1F000F7FC0095102FB801A7010E94B1781F916C
:10F200000F91FF90EF9008950E9407780895AF92B4
:10F21000BF92CF92DF92EF92FF920F931F93CF9303
:10F22000DF935C016B01EE24FF24C0E0D0E010C04E
:10F23000D501ED91FC9100811181C601BE010E94B2
:10F240008279682FC501F8010995E80EF91E21960B
:10F25000F60184819581C817D90750F3C701DF9162
:10F26000CF911F910F91FF90EF90DF90CF90BF90C3
:10F27000AF900895EF92FF920F931F937B018C0143
:10F28000611571058105910529F420E030E040E029
:10F2900050E00BC00E940107A80197010E94A57EC3
:10F2A000AC01CB01DA019C01AD01B901CA011F918A
:10F2B0000F91FF90EF900895EF92FF920F931F939D
:10F2C0007B018C01621773078407950764F4261B82
:10F2D000370B480B590BCA01B9010E943A79E60E67
:10F2E000F71E081F191FB701C8011F910F91FF904A
:10F2F000EF900895009729F0BC0180E090E00E9413
:10F3000006070895FC01848195816817790748F400
:10F310000190F081E02D309721F0E60FF71F8081FA
:10F32000089580E00895DC01FB0114968D919C9175
:10F330001597892B31F461157105A9F090E0808152
:10F3400008C00D90BC91A02D6115710529F490E0C5
:10F350008C91882349F407C0CD010E94F4079C01D9
:10F3600090E0232B09F491E0892F0895CF93DF9348
:10F370009C01FB01EC01A881B981109729F0608103
:10F38000718161157105D1F4C081D181209759F047
:10F3900084819581892B39F0888190E02227332759
:10F3A000281B390B12C0109771F0F90184819581E7
:10F3B000892B49F08C91282F30E007C0CD010E94A5
:10F3C000F4079C0102C020E030E0C901DF91CF9139
:10F3D0000895FC01DB012481358114968D919C9167
:10F3E00015972817390711F020E007C0CF010E94B8
:10F3F000B67920E0892B09F421E0822F08950F933C
:10F400001F93CF93DF93EC018B016F5F7F4F888158
:10F4100099810E940F07009711F480E005C099833D
:10F4200088831B830A8381E0DF91CF911F910F9125
:10F430000895CF93DF93EC0188819981892B29F07E
:10F440008A819B818617970760F4CE010E94FF791D
:10F45000882341F08C819D81892B19F4E881F98101
:10F46000108281E0DF91CF910895EF92FF920F9388
:10F470001F93CF93DF93EC017B016C817D81E114BD
:10F48000F104C1F04115510599F08A01060F171FCB
:10F49000B8010E94197A882369F0888199812C81AA
:10F4A0003D81820F931FB7010E94FD071D830C83CE
:10F4B00081E001C080E0DF91CF911F910F91FF901B
:10F4C000EF900895DF93CF9300D0CDB7DEB7698377
:10F4D0001A82BE016F5F7F4F41E050E00E94357A93
:10F4E0000F900F90CF91DF910895CF93DF93EC01B0
:10F4F00088819981009711F00E945606198218821E
:10F500001D821C821B821A82DF91CF9108950F9376
:10F510001F93182F092F0E94627A882321F4812FCC
:10F52000902F0E94757A812F902F1F910F9108952F
:10F530000F931F93182F092FFB0160817181448164
:10F5400055810E94357A882321F4812F902F0E94C3
:10F55000757A812F902F1F910F910895EF92FF924E
:10F560000F931F93CF93DF93EC017B018A01BA01C4
:10F570000E94197A882321F4CE010E94757A07C06F
:10F580001D830C8388819981B7010E94FD07CE01FC
:10F59000DF91CF911F910F91FF90EF900895CF933E
:10F5A000DF93EC01198218821B821A821D821C8251
:10F5B0001E826115710551F0DB010D900020E9F705
:10F5C0001197A61BB70BAD010E94AE7ADF91CF91C8
:10F5D0000895CF93DF93EC01198218821B821A825F
:10F5E0001D821C821E826115710551F0DB010D9098
:10F5F0000020E9F71197A61BB70BAD010E94AE7A68
:10F60000DF91CF9108950F931F93182F092F611544
:10F61000710559F0DB010D900020E9F71197A61B49
:10F62000B70BAD010E94AE7A02C00E94757A812F9D
:10F63000902F1F910F910895EF92FF920F931F93B8
:10F64000DF93CF93CDB7DEB761970FB6F894DEBFE7
:10F650000FBECDBF8C01CB01F80111821082138245
:10F6600012821582148216827E010894E11CF11C1C
:10F67000B70150E00E942508C801B7010E94037B32
:10F6800061960FB6F894DEBF0FBECDBFCF91DF916C
:10F690001F910F91FF90EF900895EF92FF920F93BB
:10F6A0001F93DF93CF93CDB7DEB762970FB6F89471
:10F6B000DEBF0FBECDBF8C01CB01F80111821082DD
:10F6C000138212821582148216827E010894E11C34
:10F6D000F11CB70150E00E940408C801B7010E9464
:10F6E000037B62960FB6F894DEBF0FBECDBFCF91FD
:10F6F000DF911F910F91FF90EF900895EF92FF928D
:10F700000F931F93DF93CF93CDB7DEB729970FB633
:10F71000F894DEBF0FBECDBF8C01862FF801118299
:10F7200010821382128215821482168290E07E016A
:10F730000894E11CF11CB70150E00E942508C801A3
:10F74000B7010E94037B29960FB6F894DEBF0FBE67
:10F75000CDBFCF91DF911F910F91FF90EF90089552
:10F76000DF93CF9300D0CDB7DEB7FC0111821082BA
:10F770001382128215821482168269831A82BE0154
:10F780006F5F7F4F0E94037B0F900F90CF91DF91AF
:10F790000895DF93CF9300D0CDB7DEB7FC0111827F
:10F7A00010821382128215821482168269831A8251
:10F7B000BE016F5F7F4F0E94037B0F900F90CF9130
:10F7C000DF910895CF93DF93EC01FB018617970734
:10F7D00061F0608171816115710529F04481558165
:10F7E0000E94AE7A02C00E94757ACE01DF91CF915D
:10F7F0000895FC01118210821382128215821482F4
:10F8000016820E94E27B0895FC011182108213820D
:10F8100012821582148216820E94E27B0895FC01F6
:10F82000808191810E9456060895FC01808191811A
:10F830000E94560608955058BB27AA270ED070C1C3
:10F8400061D130F066D120F031F49F3F11F41EF405
:10F8500056C10EF4E095E7FB4CC1E92F72D180F35D
:10F86000BA17620773078407950718F071F49EF5BD
:10F870008AC10EF4E0950B2EBA2FA02D0B01B90111
:10F8800090010C01CA01A0011124FF27591B99F016
:10F89000593F50F4503E68F11A16F040A22F232F22
:10F8A000342F4427585FF3CF469537952795A79572
:10F8B000F0405395C9F77EF41F16BA0B620B730B19
:10F8C000840BBAF09150A1F0FF0FBB1F661F771F8A
:10F8D000881FC2F70EC0BA0F621F731F841F48F43F
:10F8E000879577956795B795F7959E3F08F0B3CFC5
:10F8F0009395880F08F09927EE0F979587950895AF
:10F90000D4D008F481E008950CD00AC102D140F0AF
:10F91000F9D030F021F45F3F19F0EBC0511134C140
:10F92000EEC00FD198F39923C9F35523B1F3951B7A
:10F93000550BBB27AA2762177307840738F09F5F10
:10F940005F4F220F331F441FAA1FA9F333D00E2E7F
:10F950003AF0E0E830D091505040E695001CCAF7EC
:10F9600029D0FE2F27D0660F771F881FBB1F2617B1
:10F9700037074807AB07B0E809F0BB0B802DBF0184
:10F98000FF2793585F4F2AF09E3F510568F0B1C0A2
:10F99000FBC05F3FECF3983EDCF386957795679567
:10F9A000B795F7959F5FC9F7880F911D9695879535
:10F9B00097F90895E1E0660F771F881FBB1F621754
:10F9C00073078407BA0720F0621B730B840BBA0B12
:10F9D000EE1F88F7E0950895BCD088F09F5790F00F
:10F9E000B92F9927B751A0F0D1F0660F771F881F64
:10F9F000991F1AF0BA95C9F712C0B13081F0C3D07F
:10FA0000B1E00895C0C0672F782F8827B85F39F01C
:10FA1000B93FCCF3869577956795B395D9F73EF4C2
:10FA200090958095709561957F4F8F4F9F4F08956A
:10FA3000E89409C097FB3EF4909580957095619588
:10FA40007F4F8F4F9F4F9923A9F0F92F96E9BB273E
:10FA50009395F695879577956795B795F111F8CFBA
:10FA6000FAF4BB0F11F460FF1BC06F5F7F4F8F4F25
:10FA70009F4F16C0882311F096E911C0772321F01B
:10FA80009EE8872F762F05C0662371F096E8862FB3
:10FA900070E060E02AF09A95660F771F881FDAF70A
:10FAA000880F9695879597F90895990F0008550F37
:10FAB000AA0BE0E8FEEF16161706E807F907C0F0F4
:10FAC00012161306E407F50798F0621B730B840BFC
:10FAD000950B39F40A2661F0232B242B252B21F4D6
:10FAE00008950A2609F4A140A6958FEF811D811D76
:10FAF000089597F99F6780E870E060E008959FEFB0
:10FB000080EC089500240A941616170618060906B4
:10FB1000089500240A941216130614060506089583
:10FB2000092E0394000C11F4882352F0BB0F40F40B
:10FB3000BF2B11F460FF04C06F5F7F4F8F4F9F4F4B
:10FB4000089557FD9058440F551F59F05F3F71F0CD
:10FB50004795880F97FB991F61F09F3F79F0879534
:10FB60000895121613061406551FF2CF4695F1DFBD
:10FB700008C0161617061806991FF1CF869571054D
:10FB8000610508940895E894BB2766277727CB0181
:10FB900097F908958ADF08F48FEF08950BD0C0CF4E
:10FBA000B1DF28F0B6DF18F0952309F0A2CFA7CF78
:10FBB0001124EACFC6DFA0F3959FD1F3950F50E053
:10FBC000551F629FF001729FBB27F00DB11D639F0F
:10FBD000AA27F00DB11DAA1F649F6627B00DA11DB5
:10FBE000661F829F2227B00DA11D621F739FB00D5B
:10FBF000A11D621F839FA00D611D221F749F3327CB
:10FC0000A00D611D231F849F600D211D822F762F63
:10FC10006A2F11249F5750408AF0E1F088234AF060
:10FC2000EE0FFF1FBB1F661F771F881F91505040AC
:10FC3000A9F79E3F510570F05CCFA6CF5F3FECF374
:10FC4000983EDCF3869577956795B795F795E79598
:10FC50009F5FC1F7FE2B880F911D9695879597F9A9
:10FC60000895629FD001739FF001829FE00DF11D06
:10FC7000649FE00DF11D929FF00D839FF00D749F26
:10FC8000F00D659FF00D9927729FB00DE11DF91FD2
:10FC9000639FB00DE11DF91FBD01CF01112408952F
:10FCA000991B79E004C0991F961708F0961B881FCE
:10FCB0007A95C9F780950895AA1BBB1B51E107C02F
:10FCC000AA1FBB1FA617B70710F0A61BB70B881FEC
:10FCD000991F5A95A9F780959095BC01CD0108957B
:10FCE00097FB092E07260AD077FD04D0E5DF06D062
:10FCF00000201AF4709561957F4F0895F6F790955E
:10FD000081959F4F0895A1E21A2EAA1BBB1BFD01EE
:10FD10000DC0AA1FBB1FEE1FFF1FA217B307E407EA
:10FD2000F50720F0A21BB30BE40BF50B661F771F42
:10FD3000881F991F1A9469F7609570958095909522
:10FD40009B01AC01BD01CF01089597FB092E05264B
:10FD50000ED057FD04D0D7DF0AD0001C38F45095E0
:10FD60004095309521953F4F4F4F5F4F0895F6F7DF
:10FD700090958095709561957F4F8F4F9F4F089517
:10FD8000EE0FFF1F0590F491E02D09942F923F9202
:10FD90004F925F926F927F928F929F92AF92BF929B
:10FDA000CF92DF92EF92FF920F931F93CF93DF9347
:10FDB000CDB7DEB7CA1BDB0B0FB6F894DEBF0FBEA4
:10FDC000CDBF09942A88398848885F846E847D84F1
:10FDD0008C849B84AA84B984C884DF80EE80FD80F3
:10FDE0000C811B81AA81B981CE0FD11D0FB6F89469
:10FDF000DEBF0FBECDBFED0108951AE0CCEFDAE013
:10FE000004C0FE010E94C27E2296CE3FD107C9F7F0
:04FE1000F894FFCF94
:10FE1400002D0020202020007800200043560052AE
:10FE240073657400544945004F666600323A3300E6
:10FE3400333A3400373A3800313A002B002F00208F
:10FE440000292F0000010000000101000000000053
:10FE54000000000000000000000000FFFF00030499
:10FE640006080C1018203040600104000000000057
:10FE740000FFFF0000FEFF0000FDFF0000FCFF008C
:10FE840000FBFF0000FAFF03030000003F000080B6
:10FE94003F713DAA3F00000040713D2A40000080B0
:10FEA40040E0C0A0806040200001010004080C90E4
:10FEB40001000058020000010118100C0806040398
:10FEC400010C0D0E0F08090A0B04050607000102B8
:10FED40003000000001C6EB27700004000140054C0
:10FEE40000000000000E70DD6F966F9F6FB46FC549
:10FEF4006F00000000D176B277657696767676BF8D
:02FF0400760085
:00000001FF
